:020000040800F2
:10000000002000106520030839850208BD31000872
:1000100035850208318502082D85020800000000A0
:100020000000000000000000000000002985020818
:10003000258502080000000021850208052A000825
:10004000CD200308CD200308CD200308CD200308D0
:10005000CD200308CD200308F53300082135000822
:10006000E5340008A93400086D340008214E00086A
:10007000114E0008014E0008F14D0008E14D000846
:10008000CD4D0008B94D0008CD200308CD20030850
:1000900015890208CD200308CD200308313400085B
:1000A000C11E0008111F0008CD200308391F0008D9
:1000B000011F0008F11E0008CD200308CD20030811
:1000C000CD200308CD200308CD200308CD20030850
:1000D000CD200308312B0008B52A0008392A000872
:1000E000B9330008CD20030811850208CD2003088C
:1000F000D11E0008CD200308E11E0008CD20030812
:10010000000000000000000000000000CD200308F7
:10011000CD200308CD200308CD200308CD200308FF
:10012000A54D0008914D00087D4D0008694D00085F
:10013000554D0008CD20030800000000000000001D
:10014000CD200308CD200308CD20030800000000C7
:10015000000000000000000000000000000000009F
:100160000000000000000000CD200308CD2003089F
:10017000CD20030800000000000000000000000087
:0801800000000000CD2003087F
:1001880003680A7A591C01601A70704738B50B4C1D
:1001980023688BB15A68821A002A054604DA0CE0F3
:1001A8005A68AA1A002A07DB9A68226018461A6851
:1001B80090472368002BF3D138BD38BDBC2E0020F2
:1001C8000B4B002210B4027203F1DC04012102E09F
:1001D800072A09DC9979890702D5197981540132EE
:1001E8009C4203F11403F3D15DF8044B704700BF40
:1001F800107003081F230370704700BF012310B459
:1002080015211424222244704171C27003700371B5
:1002180083705DF8044B70472DE9F0410B78057B3E
:10022800DB43DFB200F1130200F11D0302F8015FA6
:100238009342FBD1DFF890E000F12701002203F898
:10024800012F9942FBD114210524002647FA04F313
:1002580003F00103002B1E4414BF4FF019084FF0A0
:100268000A0814F0010FF6B214BFAC464FF0000CA8
:100278000023CA1810FA82F20133434582F814C0E9
:10028800F7D15A1E92B20132013C8B18621C9BB204
:1002980001D01946DAE716F0010F14BF19240A2411
:1002A8000022991810FA81F10132A2420D75F8D195
:1002B80013449BB25A1C0344002192B21975AEF83C
:1002C80000200261BDE8F081301E00202DE9F04FCA
:1002D800DFF890A0BAF802300B3383B01FFA83F925
:1002E80001F1060B4FF001084FF0000C002711F840
:1002F80001EB3E464C460122A4F10B039BB201914F
:1003080005E001339BB2017B29759C4208D0C518D2
:10031800002AF6D1C51801339BB29C422A75F6D142
:1003280003190136092F019983F814C0F6B20CD0CD
:10033800092E15D008FA07F313EA0E0F14BF01228D
:1003480000220C34A4B20137D6E709F178095945DF
:100358001FFA89F9CAD1AAF802C003B0BDE8F08F24
:100368000022EEE7301E00202DE9F047DFF85C8020
:10037800B8F8043004331FFA83FC01F109094FF07F
:10038800010E11F8017B64460026231F0EFA06F2BF
:100398009BB23A40C2B1B0F80CA0C51801339BB269
:1003A8009C4285F814A0F5D101360434082EA4B275
:1003B800EBD10CF1200C49451FFA8CFCE1D100234C
:1003C800A8F80430BDE8F0879246E6E7301E002022
:1003D80010B40268047B11680223A340194209D0B3
:1003E8000649406800240C7001684FF6FE742140ED
:1003F800016053605DF8044B704700BFDC4000208B
:10040800436A826970B4D154436A0469426B013308
:10041800A34228BF00234362DAB1116811F0010139
:1004280001D070BC7047856A86699D422E44D660AB
:100438000BD3641B546081621368002143F00103ED
:1004480080F8441070BC136070475D1B5560836270
:10045800F2E7026D136843F080031360E1E700BF21
:10046800026B10B462B1036CC2684469D11A013BD3
:10047800615C5DF8044B08BF13460364C8B270475B
:10048800016A4369C4685B5C0131A14228BF114617
:1004980001625DF8044BD8B2704700BF436B13B1DB
:1004A80090F844007047836A406A181AB0FA80F0DE
:1004B80040097047416A836A99420AD3CB1A416B53
:1004C800026961B14968501E0B4483420AD2C01ABE
:1004D800704702691144CB1A416B0029F2D1501EB2
:1004E800C01A704700207047036B43B1026C5B6809
:1004F80093422FBF981AC0689B1AC0187047C269E8
:10050800036A9A422FBFD01AC0688018C01A704771
:100518000A4B30B503F1140493F900205D78072ADB
:10052800C8BF143A811804330D7313F8025C85545C
:1005380013F8012C0A76A342EED130BD444D0308CE
:1005480003682DE9F041DF691FB13B46BDE8F04182
:100558001847002A164611DD04460D460E4400E0F1
:1005680023689B68204698470028F9D0236815F827
:10057800011B1B6820469847AE42F1D1BDE8F081C7
:1005880000232822027043708370C37070472323AE
:1005980003702423C370252383712D2343702E23D6
:1005A80003712F23C371704730B4436813B11C68BB
:1005B8009B882385036840F2E93401E0002C37D09A
:1005C8001D89013C15F0020FA4B2F7D0197303F18D
:1005D8000C0540F2E93101E000294BD01C890139B2
:1005E80014F0010F89B2F7D02B78036840F2E93193
:1005F80001E000292DD01C89013914F0020F89B2BD
:10060800F7D01A7303F10C0440F2E93201E0002A32
:1006180041D01989013A11F0010F92B2F7D023782D
:10062800436813B11A689B889361012030BC7047F6
:1006380021498B4204D0A1F578418B42D6D10124BF
:100648001E4901EB04146189013189B26181618914
:10065800CCE7194A934204D0A2F578429342DFD1FD
:100668000121164B03EB01114B8901339BB24B81DE
:100678004B89D5E7104CA34203D011498B42B4D122
:1006880001210E4B03EB01114B8901339BB24B81C6
:100698004B890368AAE708498B4203D0084A93426A
:1006A800BED10122054B03EB0212538901339BB2E1
:1006B80053815389B4E700BF00300140146B002018
:1006C80000380040002870B51EDB0928044620DDEC
:1006D800012303EB83035B00B0FBF3F2092AF8D88C
:1006E8007BB10E4EB4FBF3F00928CCBF5722302261
:1006F800A6FB03E5024403FB1044EB0801F8012BB9
:10070800F0D100230B7070BD2D230B7040420131D6
:10071800DBE7303001F8010BF3E700BFCDCCCCCCE0
:10072800884230B44FF001042ED301FB04F4B0FB2F
:10073800F4F58D42F9D284B1AAB901E0B0FBF4F521
:10074800092DCCBF572230222A4404FB150003F898
:10075800012BB4FBF1F4002CF0D100221A7030BC4C
:100768007047B0FBF4F5092DCCBF372230222A445C
:1007780004FB150003F8012BB4FBF1F4002CF0D1B5
:1007880000221A7030BC70470546002AEBD1D7E723
:1007980003685A1C02601970704700BF2DE9F047C2
:1007A800089C2578002B804689460CBF4FF0200A0C
:1007B8004FF0300A661C35B3002A29DD334601E0C4
:1007C800024698B113F8011B501E0029F8D1971E54
:1007D80060B13D46013D51464046C8476B1C002B61
:1007E800F8DC257827EAE770013055B1041B294663
:1007F8004046C847301916F8015B002DF7D1BDE80F
:10080800F087BDE8F087002A04DC2846BDE8F087B9
:100818000020EBE7571EDCE70A44914251D030B480
:1008280041F2210411F8013B80EA0320430010F44F
:10083800004F84EA03059BB2ADB208BF1D466B00AA
:1008480015F4004F84EA03009BB280B208BF184633
:10085800430010F4004F84EA03059BB2ADB208BF11
:100868001D466B0015F4004F84EA03009BB280B26A
:1008780008BF1846430010F4004F84EA03059BB2F2
:10088800ADB208BF1D466B0015F4004F84EA0300A3
:100898009BB280B208BF1846430010F4004F84EAA8
:1008A80003059BB2ADB208BF1D466B0084EA030086
:1008B80015F4004F85B298B218BF28468A42B1D1C4
:1008C80030BC704783684268D0ED037A00EB83013F
:1008D8000133934281ED040A836004BF00238360DF
:1008E80000EB830393ED047A036870EE277A9A424B
:1008F800C0ED037A77EEC77AC0ED037A0CDA0133DC
:1009080007EE103AF8EEC76AB7EE007A87EEA60A45
:10091800036030EE070A704707EE102AB8EEC77A70
:1009280087EE870A704700BF90ED097A90ED004A7C
:10093800D0ED0A6AD0ED014AD0ED047A90ED035A61
:10094800D0ED025AA4EE007AB0EE406AB0EE470A43
:10095800B0EE667AA6EE247A67EEC07AA0EE457A03
:10096800E6EE257A80ED097AC0ED0A7A704700BF75
:10097800D0ED057A90ED013AD0ED003AD0ED064A77
:1009880090ED024A90ED077A90ED035A90ED086ACF
:10099800D0ED045AC0ED067AF0EE406A27EE830ADD
:1009A800C0ED056AA3EEA60A80ED087AA4EE240A33
:1009B800A5EE470AA5EEC60A80ED070A704700BFF4
:1009C800D0ED007A90ED017A30EE670AE7EE007A12
:1009D800B0EE670AC0ED007A704700BF704700BFED
:1009E8002DE9F04FDFF81CB2DFF81CE2BBF800205D
:1009F800DEF80860BBF90430BBF90250BBF90A8085
:100A0800C2EB261404FB04F424135200C2EBE602E2
:100A180003FB04F305FB02F29B1303EBE223B3F59C
:100A2800FA364FEAE37589B045F1FF373246A6FB3F
:100A38000645CDE9024502FB07F205EB4202CDE986
:100A48000467029EBBF90840039208FB02FC4FEAC8
:100A5800E87906FB09CC3A46A8FB0689049ECBF840
:100A68001830E51704FB02F206FB0522A4FB066713
:100A7800E14417444FEA182242EA096200924FEA19
:100A8800292201923D03DDE90078340345EA165531
:100A98003F19BBF80660069048EB05083C1C48F572
:100AA800004503EB8302A4FB068906FB0599803207
:100AB80013124FEA69064FEAE977079356EA0703E4
:100AC8008A4600F09280DDE90489BBF90E20DEF841
:100AD8000C40BBF910004946C4F5801ED317DDE968
:100AE800024502FB01F108FB0311A2FB08230B449A
:100AF8004FEA43492B46C11700FB03F304FB0133BC
:100B0800A0FB0401BBF90C401944E30001937346B0
:100B1800DC170023009349EAD2394FEA4248DDE95D
:100B2800002310EB080041EB0901E50712184FEA12
:100B3800CE744B4145EA5E05A41A65EB03052219FC
:100B480045EB050312196B4199019001801841EAA0
:100B5800926159418B00820043EA9073101943EB6C
:100B680005018B00820043EA90731046001919466C
:100B780032463B46694131F09DF8BBF916204C13CB
:100B8800450B45EAC14502FB04F6D31705FB03668E
:100B9800A2FB05233344BBF9146002FB04F405FBF4
:100BA800034406FB01FEA2FB0523F717234400FBC1
:100BB80007EE540EA6FB0067774444EAC3144FEAD5
:100BC800D64800194FEA636548EA473869414FEA51
:100BD800E74918EB0008BBF9124049EB01094FEA55
:100BE800182646EA096620013618069B0BB1360A14
:100BF8001E60BAF1000F02D0079BCAF8003009B096
:100C0800BDE8F08F142C0020301E0020704700BF74
:100C1800704700BF4FF40063038270474FF40063CE
:100C28000382704750F8043C012280F835201438BC
:100C380003B11847704700BF90F8493013B100223C
:100C480080F849201846704770B5044682B01830BD
:100C5800256D94F85C106B460622A847A8B19DF84C
:100C680004009DF800609DF801109DF802509DF861
:100C780003209DF8053041EA062143EA002342EAB1
:100C88000522A184E2842385012002B070BD00BF43
:100C980070B5044682B00830256A6B4606223B21AF
:100CA800A847A8B19DF804009DF800609DF80110C0
:100CB8009DF802509DF803209DF8053041EA062171
:100CC80043EA002342EA05226182A282E3820120EC
:100CD80002B070BD30B490E81200057B436902226F
:100CE800AA404A602268586A996A4FF6FE752A40F7
:100CF8008842226004D1012283F8442030BC704726
:100D08009C695A6B0C44D4600DD818690024411AA8
:100D180051609C621168002041F0010183F8440091
:100D280030BC11607047411A51609862F2E700BF09
:100D380070B40468037B2268022101FA03F31A42A3
:100D480013D042690A49582000FB02124FF6FE767A
:100D580050685289C5680068296831402960C168AF
:100D6800D24392B20A40C260636070BC704700BF51
:100D7800AC59002030B4094B1C7864B1084B0025ED
:100D880003EBC4041A6899885562D0680833014394
:100D9800A342D160F6D130BC704700BFCC5D0020C3
:100DA800D05D002010B40268047B11680223A340C0
:100DB800194209D00649406800240C7001684FF6B2
:100DC800FE742140016053605DF8044B704700BF1A
:100DD800033E0020F0B5064683B00D4600240127E7
:100DE80014E003290CBF03220122C3F3011E694644
:100DF800C3F3810330468DF805208DF806E08DF8A1
:100E080007301FF0B9F80134102C0FD02B8807FADF
:100E180004F21342F7D0AB78E9780092022903F084
:100E280003028DF80420DCD10A46DEE703B0F0BDEA
:100E3800F0B4334C00EB800004EB80046468002CB1
:100E48005BD0304E49004FF42040CDB23060A169EC
:100E5800090444D460682C4F45F08071384041F44F
:100E6800903101434FF420406160306003E0411E3F
:100E7800002838D00846A1698F07F8D54FF42040DC
:100E8800A262306002E0421E68B31046A2691106F1
:100E9800F9D562681C4945F0007545F480350A406B
:100EA80015434FF420406560306002E0421ED0B127
:100EB8001046A2699207F9D5A362A3694FF42040AE
:100EC8009B06306005D4431E68B11846A3699B068B
:100ED800F9D520233060E3610120F0BC7047411E42
:100EE80008B10846B3E7094A138801339BB24FF0AB
:100EF800FF3131601380F0BC70472046F0BC70476A
:100F0800E46A00200C6B0020009800FC106B0020A5
:100F1800134600200A4668218AE700232622036038
:100F28000270272282700122436002718371704728
:100F380070B5448806460D46C4F30B0422460021CA
:100F4800284633F046FE3369094A934209D3094AD1
:100F5800934206D2224628461946BDE8704031F031
:100F680023BB23B121462846BDE87040184770BD11
:100F7800B4B403085AB5030870B54E680546304640
:100F880030F0CEF9314604460246286831F00CFBB1
:100F98002A68131901333B212B60115570BD00BF1E
:100FA80008B51BF039FC024B024ADA60FEE700BFC5
:100FB80000ED00E00400FA05024A034B12781978A4
:100FC8001DF0C6BA8C1E00208D1E00202DE9F047AA
:100FD8000569C3681D4028D00F4606464FF00048F3
:100FE8004FF00009B5FA85F328FA03F2D2431B3B08
:100FF80032611540042B16D8DFE803F03129211996
:1010080003007B6A002B32D003F1FF3A1FFA8AFAF9
:10101800C7F824903C6A34B1236820465146984763
:101028006468002CF8D1002DDCD1BDE8F087386861
:10103800716B036889B29847002DD3D1F5E77868BA
:10104800B16B036889B29847002DCBD1EDE7B8683A
:10105800F16B036889B29847002DC3D1E5E7F868BA
:10106800316C036889B29847002DBBD1DDE7F36A7C
:101078001FFA83FACEE700BF30B50446006D6171F0
:101088000368A26823F00103036087B0A379009284
:1010980013F004023DD04FF4805213F00203019282
:1010A80044D102934FF480630022039311F00103AB
:1010B800059237D1049308238D07694648BF0493E6
:1010C80026F0F6FE6079236DA17900F00202002A6D
:1010D80015BF4FF440324FF480324FF400340024EF
:1010E80010F0010F586808BF2246CC074CBF0243D6
:1010F80020EA02025A609A6809074CBF42F00802C7
:1011080022F008029A601A6842F001021A6007B0D9
:1011180030BD13F0020301920BD04FF40055134673
:101128000295C1E7042304930C23C5E74FF4005349
:10113800B7E70293B8E700BF10B50446006DA16099
:10114800036823F001030360A37986B013F0040257
:10115800009141D04FF4805213F00203019244D120
:1011680002934FF4806362790393D1074FF0000331
:101178000493059345BF0423049308230C2369466D
:10118800920748BF049326F093FE6079236DA179F6
:1011980000F00202002A15BF4FF440324FF48032AB
:1011A8004FF40034002410F0010F586808BF22469D
:1011B800CC074CBF024320EA02025A609A6809072A
:1011C8004CBF42F0080222F008029A601A6842F006
:1011D80001021A6006B010BD13F00203019207D095
:1011E8004FF4005113460291BDE74FF40053B7E79F
:1011F8000293B8E72DE9F341056906460F467DBB22
:10120800D0F80080C8F30A0323B30023D6F800807F
:10121800019324F0BBFD042819D1224C236943F023
:1012280001032361BBB2A8F8003024F0AFFD042805
:101238002ED108F102030193019B3F0C1F8024F07B
:10124800A5FD2369042823F00103236125D06FF04D
:10125800010505E024F09AFD042805D04FF0FF357C
:10126800284602B0BDE8F0810E4C236943F0020322
:101278002361C4F81480236943F04003236124F0F8
:1012880085FD2369042823F002032361BDD0E5E727
:10129800236923F001032361D9E7336804333360FA
:1012A800DEE700BF00200240F8B504460D468E1860
:1012B8000027B54201D12069F8BDE368591CE160F7
:1012C800234415F8012B1A720429F2D1A16820468B
:1012D800FFF790FFE7602061EBE700BF00B5002152
:1012E80083B00A2021F054F80F210A2021F050F889
:1012F80001AA0321102021F06FF89DF90430DFEDD9
:10130800277ADFED275A06EE103A9DF9053006EEEA
:10131800903A9DF9063007EE103AB8EEC66AF8EE34
:10132800E66AB8EEC77A76EEE76A36EE676A37EEAF
:10133800677AF7EE007AB0EE675AA6EE255A194B8F
:101348000021B0EE456AB0EE675AA6EEA55A0A200B
:10135800E7EE257AF3EE0E5A26EE256A25EE257A73
:1013680067EEA57A83ED006A83ED017AC3ED027A10
:1013780021F00EF80DF103020121022021F02CF8D2
:101388000DF103020121092021F026F801210A208C
:1013980020F0FEFF012003B05DF804FB00000043CD
:1013A8000000803B0000002070B582B06B4606222A
:1013B800F721762029F062F99DF801209DF8043084
:1013C8009DF800609DF803509DF802409DF80500C7
:1013D800074912011B0142EA063243EA053342EA91
:1013E800141243EA1013CA608B6002B070BD00BFCC
:1013F800301E0020682029F041B900BF70B582B0C6
:1014080004466946183020F06FFFA8B19DF8050022
:101418009DF801609DF802109DF803509DF8042086
:101428009DF8063041EA062143EA002342EA0522F4
:10143800A184E2842385012002B070BD10B44C0958
:10144800012250F8243001F01F0102FA01F10B4388
:1014580040F824305DF8044B704700BF00210A4A69
:101468000B4604E00133242B0BD012F80C1C8842E5
:1014780002F10C02F6D1054803EB430300EB8300AD
:1014880070470020704700BFB44E0308A04E030801
:1014980000210A4A0B4604E00133242B0BD012F832
:1014A8000C1C884202F10C02F6D1054803EB4303F9
:1014B80000EB830070470020704700BFAC4E030864
:1014C800A04E0308022828BF022010B4084C094B7C
:1014D800207000EBC00200EB820207495DF8044B64
:1014E800013003EB4203C0B20B6022F083BF00BFA0
:1014F800683E0020F08D0020843E002038B5414B26
:101508005A899989914224BF00225A81198ADA8915
:10151800914224BF0022DA81DA788AB1072A0FD0F3
:10152800394C3A48A27801210025062A01709970A1
:10153800DD7150D92379DFED366A002B3AD138BDF9
:10154800DA79002A4CD09A783048DFED316A017890
:10155800042A38BF042207EE902AB8EEE77A07EE8D
:10156800901A27EE267AF8EEE77A9A7067EE877A6D
:10157800254CA278062A2BD8264B03EB8203D3ED01
:10158800056AF4EEE76AF1EE10FA10DDC6EE877A26
:10159800FDEEE77A17EE903A102BA8BF1023012B27
:1015A800B8BF0123DBB28B4228BF0B4603702379F7
:1015B800002BC4D0013A032AC1D8B7EE000A80EE46
:1015C800260A31F0F9F92388984238BF208038BDBF
:1015D800DFED0F6AD5E7DFED107AB0EE677ACBE77B
:1015E8009B780A48DFED0D6A017807EE103A07EE9E
:1015F800901AB8EEC77AF8EEE77A27EE267A67EE01
:10160800877AB5E71044002080590020308C0020EC
:101618006F120338444D03086F12833A6F1203396F
:1016280038B50E4C0E4DAC4206D2616820461434D3
:10163800FFF77EFCAC42F8D30A4A0B4B0B4D0C4823
:10164800106000241C702C702CF034F9094B0A4AE5
:101658006C701A60BDE838401CF0ACBC68B0030878
:10166800B4B40308843E0020D1300020683E002036
:10167800F08D002078260020E43A0020F0B50C29EF
:101688002BD8DFE801F06F2A2A2A4C2A2A2A2B2A8B
:101698002A2A0700046AB2F80CE097881668674D92
:1016A80024F480540462036A4468C16923F4005333
:1016B80043EA0E3321F4E641A84243EA073341EAFC
:1016C800062100F0B58005F50065A84200F0B0805D
:1016D80092684460C16102640362F0BD046A96893D
:1016E8009588D2F800E0554F24F480740462036AA8
:1016F8004468C16923F4007343EA062321F07301A7
:10170800B84243EA052341EA0E017ED04C4DA84277
:101718007BD092684460C161C2630362F0BD046A11
:1017280096899588D2F800E0444F24F010040462AA
:10173800036A4468816923F0200321F0807143EA39
:10174800061321F4E641B84243EA051341EA0E21A3
:1017580048D03B4DA84245D092684460816182637D
:101768000362F0BD046A9389B2F804E01768334E47
:1017780024F001040462056A4468816943EA0E039F
:1017880021F4803125F002059BB221F07301B042AB
:1017980043EA050341EA070114D0294DA84211D0B4
:1017A80005F54065A8420DD005F58065A84209D029
:1017B80005F58065A84205D092684460816142635E
:1017C8000362F0BDD689158A578A23F0080333438C
:1017D8003D43D68824F4407423F00403ADB2334368
:1017E8002C43E9E7D589178AD68823F0800343EA92
:1017F800051324F44064558A23F0400344EA87041F
:1018080043EA061344EA8504A6E7D589178AD688E9
:1018180023F4006343EA052324F44054558A23F44F
:10182800806344EA071443EA062344EA051470E790
:10183800158A24F4804444EA851449E7002C0140C1
:10184800003401402DE9F84FF02200218E488F4CDA
:10185800DFF860928E4D8F4E8F4FDFF85C8233F049
:10186800B8F98E488E49DFF854E2DFF854C20022F6
:101878001359834200F0F880B3F1804F00F0F680EE
:10188800AB4200F0F580B34200F0F480BB4200F0B8
:10189800F380734500F0F280634500F0F180434522
:1018A80000F0F080DFF81CA2534500F0A7800AF58D
:1018B800806A534508BF092300F0A1801432F02A3A
:1018C800D6D1DFF8C881774F774D08F1F0064FF091
:1018D800030A4FF0020998F804301C09013C052C52
:1018E80003F00F0300F2838037F8140040FA03F284
:1018F800D2077CD54FF0010B0BFA03F3013B1840DC
:1019080030F028FA694B1B5D184415EBC0046ED003
:1019180055F83030664898F8081003F13842920AB2
:10192800825C02F01F005209022A0BFA00FB00F049
:101938009480032A00F08A80012A05D1584A584821
:1019480052694BEA02024261B4F804E0BEFA8EF230
:10195800C2F11F0292B2D00803EB800002F0070226
:10196800046A92004FF00F0C0CFA02FC24EA0C04F3
:101978000462046A01FA02F22243002402624FF070
:10198800010C224603E0102A04F102042FD00CFABD
:1019980002F030EA0E0102F10102F4D1D3F808B0E6
:1019A8000AFA04F1C9430BEA010BC3F808B0D3F8EB
:1019B80008B0C3F808B0B3F804B01FFA8BFB2BEAE1
:1019C80000009880988880B298801868084018604D
:1019D800D3F800B009FA04F040EA0B001860D868A0
:1019E800102A01EA0001D96004F10204CFD108F1FC
:1019F800140846457FF46FAFBDE8F88F082309EB5C
:101A0800C3034FF0010B93F834A00AF01F034FEA09
:101A18005A1ABAF1020F0BFA03F30BD0BAF1030FFB
:101A28000ED0DA457FF44AAFD1F814A043EA0A038E
:101A38004B6143E7D1F818A043EA0A038B613DE7FD
:101A4800D1F81CA043EA0A03CB6137E7144A1448CB
:101A5800D2694BEA0202C26176E7114A10489269DC
:101A68004BEA020282616FE70023C8E70123C6E759
:101A78000223C4E70323C2E70423C0E70523BEE724
:101A88000623BCE70723BAE7EC3F002010700308E1
:101A9800000400400008004000100040002C0140F5
:101AA80000100240346D030850580020406D0308B0
:101AB800486D0308444D03080040014000140040ED
:101AC8000034014000440140002867D003682DE934
:101AD800F04F03F138445C4EA40A0125345D04F04C
:101AE8001F066409022C05FA06F558D0032C00F0ED
:101AF800A580012C58D08088B0FA80F4C4F11F0466
:101B0800A4B2E50803EB850504F007042E6AA400D7
:101B18000F27A74026EA07062E622E6A01F0030760
:101B2800A2407C1E3243012CC1F3810CC1F3001882
:101B38002A62C1F341113CD9C60700F189808507A3
:101B480000F19580440700F1A380020700F1B180FD
:101B5800C60600F1BF80850600F1CD80440600F17D
:101B6800DB80020600F1E980C60500F1F7808505F3
:101B780000F10581440500F11381020500F121817E
:101B8800C60400F12F81850400F13D81440400F171
:101B98004B81020400F15981BDE8F08F70472B4C4E
:101BA800A6693543A561A6E7284C66693543656192
:101BB800A1E7002422464FF0010E4FF0030904E08C
:101BC8000132102A04F10204E6D00EFA02F636EACF
:101BD8000005F5D1D3F808A009FA04F5ED430AEA9F
:101BE800050AC3F808A0D3F808B00CFA04FA4AEAC0
:101BF8000B0AC3F808A0B3F804A01FFA8AFA2AEA65
:101C080006069E80B3F804A008FA02F646EA0A0619
:101C1800B6B29E801E682E401E60D3F800A007FA58
:101C280004F646EA0A061E60D3F80CA001FA04F688
:101C380005EA0A0A46EA0A05DD60C1E7034CE669D7
:101C48003543E56157E700BF486D030800100240BF
:101C58001A6822F003021A601A683A431A60DA68AE
:101C680022F003020A438507DA607FF56BAF1A6832
:101C780022F00C021A601A6842EA87021A60DA68CF
:101C880022F00C0242EA81024407DA607FF55DAF78
:101C98001A6822F030021A601A6842EA07121A60BB
:101CA800DA6822F0300242EA0112DA6002077FF5B0
:101CB8004FAF1A6822F0C0021A601A6842EA871207
:101CC8001A60DA6822F0C00242EA8112C606DA60B7
:101CD8007FF541AF1A6822F440721A601A6842EA26
:101CE80007221A60DA6822F4407242EA0122850665
:101CF800DA607FF533AF1A6822F440621A601A6816
:101D080042EA87221A60DA6822F4406242EA8122B3
:101D18004406DA607FF525AF1A6822F440521A604B
:101D28001A6842EA07321A60DA6822F4405242EA34
:101D38000132DA6002067FF517AF1A6822F44042D2
:101D48001A601A6842EA87321A60DA6822F4404256
:101D580042EA8132C605DA607FF509AF1A6822F4D3
:101D680040321A601A6842EA07421A60DA6822F4B6
:101D7800403242EA01428505DA607FF5FBAE1A6817
:101D880022F440221A601A6842EA87421A60DA6826
:101D980022F4402242EA81424405DA607FF5EDAE42
:101DA8001A6822F440121A601A6842EA07521A6046
:101DB800DA6822F4401242EA0152DA6002057FF53D
:101DC800DFAE1A6822F440021A601A6842EA8752A3
:101DD8001A60DA6822F4400242EA8152C604DA60E4
:101DE8007FF5D1AE1A6822F040721A601A6842EA8A
:101DF80007621A60DA6822F0407242EA01628504DA
:101E0800DA607FF5C3AE1A6822F040621A601A6879
:101E180042EA87621A60DA6822F0406242EA816226
:101E28004404DA607FF5B5AE1A6822F040521A60B1
:101E38001A6842EA07721A60DA6822F0405242EAE7
:101E48000172DA6002047FF5A7AE1A6822F04042F8
:101E58001A601A6842EA87771F60DA6822F04042FF
:101E680042EA8171D960BDE8F08F00BF10B504095E
:101E7800013C052C17D80D4B33F8142000F00F0047
:101E880042FA00F313F001030DD0012303FA00F026
:101E9800013810402FF05EFF054A064B125D1044D2
:101EA80003EBC00010BD002010BD00BF346D030857
:101EB800406D03085058002001490248FFF786B8D2
:101EC8008C4000200040014001490248FFF77EB8DD
:101ED800644000200034014001490248FFF776B809
:101EE800644000200034014001490248FFF76EB801
:101EF8003C4000200004004002494FF08040FFF7BA
:101F080065B800BF1440002010B5064C06482146AD
:101F1800FFF75CF804F1C8010448BDE81040FFF77A
:101F280055B800BFEC3F0020002C014000440140A0
:101F380001490248FFF74AB8EC3F0020002C014055
:101F48002DE9F04104684E4DA30AAB427AD00AD974
:101F58004C4DAB425FD00135AB4277D0043DAB422C
:101F68005DD0BDE8F081B3F5801F67D04A3DAB4234
:101F780059D14FF0700E022647794FEA970C002985
:101F880068D0B000634685190227D4F80C809F40BA
:101F98000CEB4503BFB23C4D03F1040C47EA0807BC
:101FA80045F8231045F82C20E760EFF31181502203
:101FB80082F31288821905EBC2021369002B34D010
:101FC80013620433821905EBC202576917B11F6007
:101FD80053690433821905EBC202976917B11F6070
:101FE80093690433821905EBC202D76917B11F60E0
:101FF800D36904330027CAB21F6082F311883044C2
:1020080005EBC000036A9BB9E3684FF6FE72134004
:10201800E360BDE8F0814FF0C00E0426ACE74FF056
:10202800980E0326A8E7BDE8F08105EB0E03C9E783
:10203800E36843F00103E360BDE8F0814FF0480E28
:10204800012699E74FF0200E002695E74FF0E80E9D
:10205800052691E7BF08022306FA03F0BB40DB43DD
:10206800E768094D9BB23B4087190CEB470CE360CE
:102078000CF1040345F82C1045F8232095E700BF20
:102088004B00100050001000EC3F002030B50368F2
:102098005C4D18885C4CB4FBF2F20139013AAB4252
:1020A80094B283B089B282B266D05848834263D072
:1020B800B3F1804F60D0A0F5983083425CD000F532
:1020C8008060834258D0524883425BD000F58060DC
:1020D80083427DD022F4407200F58C3092B2834264
:1020E8001A80D9621C850ED0484A93420BD002F55B
:1020F8004062934207D002F58062934203D002F512
:102108008062934201D100221A8601225A611A88FC
:102118003C4992B242F001028B421A8062D0B3F17C
:10212800804F61D03B4A934260D002F5806293426F
:102138005ED002F5006293425CD002F58062934261
:102148005AD002F59032934258D002F54062934239
:1021580056D002F5806293421ED002F58062934207
:1021680008BF092219D002A84FF0012340F8043D06
:1021780028F074FB03B030BD254822F0700283427A
:1021880092B2A3D101201A80D9621C8558611A889D
:1021980092B202431A80C5E708221F4B03EBC20321
:1021A80001A893F835408DF80440012300228DF8EA
:1021B80005308DF807308DF8062028F04FFB1B2CD2
:1021C800D8D1164B019301A828F048FB03B030BDC5
:1021D80001201A80D9621C8558611A8892B202437C
:1021E8001A809CE70022D8E70122D6E70222D4E72A
:1021F8000322D2E70422D0E70522CEE70622CCE765
:102208000722CAE7002C014000A24A04003401401A
:102218000010004000040040444D0308190100016B
:10222800204B98422DD0B0F1804F2CD0A3F5943399
:1022380098422AD003F58063984228D003F50063BA
:10224800984226D003F58063984224D003F5903352
:10225800984222D003F54063984220D003F580636A
:10226800984207D003F58063984208BF092202D03C
:102278000020704708220C4B03EBC20393F834008C
:1022880070470022F7E70122F5E70222F3E703226D
:10229800F1E70422EFE70522EDE70622EBE7072244
:1022A800E9E700BF002C0140444D03082DE9F04F39
:1022B800013085B0C3B203938C4D8D4F8D4C8E4E3B
:1022C8000A230293DFF834921FF0A8FD4FF4FA7A3C
:1022D8004FF0100C4FF47A70D9F80430C3F30803A8
:1022E800002B40F0C580EFF31183002B40F0C08035
:1022F8002968A26800BF2B689942F9D1D7F800E095
:1023080000FB0EF39B1AB3FBFEF300FB01314FF009
:10231800010E0191D9F80430C3F30803002B40F0F3
:102328008B80EFF31183002B40F086802B68A16827
:1023380000BF2A689342F9D1D7F800B000FB0BF22E
:10234800521AB2FBFBF200FB0323019A9B1AB3F566
:102358007A7FDFD3BAF1010ABED1039B002B40F08C
:10236800C1804FF47A7ADFF8949150464FF0100C00
:10237800D9F80430C3F30803002B40F09680EFF33C
:102388001183002B40F091802968A26800BF2B6858
:102398009942F9D1D7F800E000FB0EF39B1AB3FB82
:1023A800FEF300FB01314FF0010E0191D9F8043022
:1023B800C3F3080323BBEFF311830BBB2B68A1689E
:1023C80000BF2A689342F9D1D7F800B000FB0BF29E
:1023D800521AB2FBFBF200FB0323019A9B1AB3F5D6
:1023E8007A7FE3D3BAF1010AC2D1029B013B02937F
:1023F8007FF468AF414B424ADA6005B0BDE8F08F20
:10240800EFF311888CF31288A1682368DB0344BFBB
:10241800C6F800E0A1682B6832685FFA88F888F38C
:102428001188D7F800801A4400FB08F35B1AB3FB45
:10243800F8F300FB0233D0E7EFF311888CF312882E
:10244800A1682368DB0344BFC6F800E0A1682B68D5
:1024580032685FFA88F888F31188D7F800801A4440
:1024680000FB08F35B1AB3FBF8F300FB02336CE7DD
:10247800EFF311828CF31288D4F808E02368D903AB
:1024880003D501233360D4F808E02B683168D2B251
:1024980082F311883A68194400FB02F3A3EB0E0398
:1024A800B3FBF2F300FB013131E7EFF311828CF358
:1024B8001288D4F808E02368D90303D501233360D0
:1024C800D4F808E02B683168D2B282F311883A68F0
:1024D800194400FB02F3A3EB0E03B3FBF2F300FB7A
:1024E800013160E7184628F09FFB3AE7B86A0020F8
:1024F800BC6A002010E000E0B46A002000ED00E0B3
:102508000400FA052DE9F04F013085B0C3B20393FA
:102518000B4602918B4C8C4E002B00F099808B4D12
:102528008B4FDFF830921FF079FC4FF4FA7A4FF0B6
:10253800100C4FF47A70D9F80430C3F30803002B59
:1025480040F0DE80EFF31183002B40F0D98029683A
:10255800A26800BF2B689942F9D1D7F800E000FBC8
:102568000EF39B1AB3FBFEF300FB01314FF0010E93
:102578000191D9F80430C3F30803002B40F0878099
:10258800EFF31183002B40F082802B68A16800BF15
:102598002A689342F9D1D7F800B000FB0BF2521A1F
:1025A800B2FBFBF200FB0323019A9B1AB3F57A7F77
:1025B800DFD3BAF1010ABED1039B002B40F0BD80E6
:1025C8004FF47A7ADFF88C9150464FF0100CD9F816
:1025D8000430C3F30803002B75D1EFF31183002BEC
:1025E80071D12968A26800BF2B689942F9D1D7F840
:1025F80000E000FB0EF39B1AB3FBFEF300FB013176
:102608004FF0010E0191D9F80430C3F3080313BB4E
:10261800EFF31183FBB92B68A16800BF2A689342C6
:10262800F9D1D7F800B000FB0BF2521AB2FBFBF25B
:1026380000FB0323019A9B1AB3F57A7FE3D3BAF11F
:10264800010AC4D1029B013B0293002B7FF467AFC0
:1026580005B0BDE8F08FEFF311888CF31288A168FC
:102668002368DB0344BFC6F800E0A1682B68326822
:102678005FFA88F888F31188D7F800801A4400FBBD
:1026880008F35B1AB3FBF8F300FB0233D2E7EFF36E
:1026980011888CF31288A1682368DB0344BFC6F84D
:1026A80000E0A1682B6832685FFA88F888F311881F
:1026B800D7F800801A4400FB08F35B1AB3FBF8F361
:1026C80000FB023370E7EFF311828CF31288D4F821
:1026D80008E02368D90303D501233360D4F808E060
:1026E8002B683168D2B282F311883A68194400FB2A
:1026F80002F3A3EB0E03B3FBF2F300FB01317FE718
:10270800EFF311828CF31288D4F808E02368D90318
:1027180003D501233360D4F808E02B683168D2B2BE
:1027280082F311883A68194400FB02F3A3EB0E0305
:10273800B3FBF2F300FB013118E7184628F074FAEE
:102748003EE700BF10E000E0B46A0020B86A00204D
:10275800BC6A002000ED00E0204B5B68C3F308036F
:1027680030B4BBB9EFF31183A3B91D4B1D4C1868E6
:10277800A16800BF1A689042F9D11B4B1C684FF43E
:102788007A7202FB04F3591AB1FBF4F130BC02FB74
:1027980000107047EFF31182102383F31288114958
:1027A8008C680B6813F4803F104B02D0012018602E
:1027B8008C680B49D2B20D68186882F311880A4BED
:1027C80019684FF47A72284402FB01F31B1B30BCD2
:1027D800B3FBF1F302FB0030704700BF00ED00E0EF
:1027E800B86A002010E000E0BC6A0020B46A00204B
:1027F8002DE9F84F8046FFF7AFFF254E2549DFF852
:10280800A0E0254A254D844610274FF47A7401200C
:10281800DEF80430C3F30803D3B9EFF31183BBB96F
:102828000B68D2F808A000BFD1F800904B45F7D14B
:10283800D6F800B004FB0BF9A9EB0A09B9FBFBF9C0
:1028480004FB0393A3EB0C034345E1D3BDE8F88FE6
:10285800EFF3118A87F31288D2F808B01368DB0304
:1028680044BF2860D2F808B00B68D5F800905FFA2A
:102878008AFA8AF31188D6F800A0994404FB0AF36F
:10288800A3EB0B03B3FBFAF304FB0933DAE700BF4E
:10289800BC6A0020B86A002010E000E0B46A00209A
:1028A80000ED00E008B5FFF757FF044B5B68C01A5E
:1028B800C0F5FA5020EAE07008BD00BFE43F0020F0
:1028C8002DE9F04FDFF830C1474A4849484E494D95
:1028D8008046102718F1FF38C0F08480DCF80430F7
:1028E800C3F30803002B5CD1EFF31183002B58D1FD
:1028F8000B68946800BF08688342F9D1D6F8009045
:102908004FF47A7000FB09FEAEEB040EBEFBF9FE35
:1029180000FB03EEDCF80430C3F308034FF47A74C9
:102928000120FBB9EFF31183E3B90B68D2F808A0D3
:1029380000BFD1F800904B45F7D1D6F800B004FBA2
:102948000BF9A9EB0A09B9FBFBF904FB0393A3EB09
:102958000E03B3F57A7FBDD2DCF80430C3F3080365
:10296800002BDFD0EFF3118A87F31288D2F808B072
:102978001368DB0344BF2860D2F808B00B68D5F8A9
:1029880000905FFA8AFA8AF31188D6F800A0994471
:1029980004FB0AF3A3EB0B03B3FBFAF304FB0933C1
:1029A800D5E7EFF3118487F31288D2F808901368FB
:1029B800D80303D501232B60D2F808900B68286848
:1029C800E4B284F31188D6F800A04FF47A7400EBCF
:1029D800030E04FB0AF3A3EB0903B3FBFAF304FBAE
:1029E8000E3E97E7BDE8F08F10E000E0B86A0020DF
:1029F800BC6A0020B46A002000ED00E030B4EFF3B8
:102A08001183102282F312880649074C0A68074886
:102A1800013200250A602560DBB2026883F3118861
:102A280030BC7047B86A0020B46A002010E000E0AB
:102A38001D4B70B59C68236D226BDD69C2B1636B59
:102A48002BB12B0702D5236D08221A6270BD2A0606
:102A5800F7D5A26A616A8A421FD0511CA069A16297
:102A6800825C2069266D81423285EAD3A362E8E759
:102A7800A906E4D5E26A1AB1988C80B29047DEE7DD
:102A8800E1699B8C6069DBB24E1CE6614354E169E5
:102A9800E368994228BFE261D1E7226D136823F009
:102AA80080031360CDE700BFAC6700201D4B70B5F5
:102AB8005C68236D226BDD69C2B1636B2BB12B0798
:102AC80002D5236D08221A6270BD2A06F7D5A26ABC
:102AD800616A8A421FD0511CA069A162825C206988
:102AE800266D81423285EAD3A362E8E7A906E4D5D8
:102AF800E26A1AB1988C80B29047DEE7E1699B8C54
:102B08006069DBB24E1CE6614354E169E3689942AF
:102B180028BFE261D1E7226D136823F080031360B8
:102B2800CDE700BFAC6700201D4B70B51C68236D56
:102B3800226BDD69C2B1636B2BB12B0702D5236D04
:102B480008221A6270BD2A06F7D5A26A616A8A420B
:102B58001FD0511CA069A162825C2069266D814248
:102B68003285EAD3A362E8E7A906E4D5E26A1AB196
:102B7800988C80B29047DEE7E1699B8C6069DBB294
:102B88004E1CE6614354E169E368994228BFE2615B
:102B9800D1E7226D136823F080031360CDE700BFEF
:102BA800AC67002003685B6A03B11847704700BF31
:102BB80003681B6A03B11847704700BF03682DE913
:102BC800F041DF691FB13B46BDE8F0411847002AD4
:102BD800164611DD04460D460E4400E023689B6846
:102BE800204698470028F9D0236815F8011B1B6870
:102BF80020469847AE42F1D1BDE8F08103689B6951
:102C0800184700BF0368DB68184700BF03689B6864
:102C1800184700BF03685B68184700BF03681B6854
:102C2800184700BF014B1868F8E700BF30200020A4
:102C3800054B53F8203033B11A689B88918A0B42B0
:102C480018BF1B0493617047486B00202DE9F04FB3
:102C58004A484B4B4B4C4FF090414FF0010A4FF014
:102C680002094FF004084FF0080C4FF0100E20270F
:102C78004026802530F8022B12F0010F03D019608E
:102C8800A3F804A0083312F0020F03D01960A3F8C8
:102C98000490083312F0040F03D01960A3F80480DD
:102CA800083312F0080F03D01960A3F804C00833E2
:102CB80012F0100F03D01960A3F804E0083312F0E3
:102CC800200F02D019609F80083312F0400F02D005
:102CD80019609E80083312F0800F02D019609D8021
:102CE800083312F4807F05D04FF4807B1960A3F875
:102CF80004B0083312F4007F05D04FF4007B19604C
:102D0800A3F804B0083312F4806F05D04FF4806B39
:102D18001960A3F804B0083312F4006F05D04FF41B
:102D2800006B1960A3F804B0083312F4805F05D073
:102D38004FF4805B1960A3F804B0083312F4005F05
:102D480005D04FF4005B1960A3F804B0083312F4FF
:102D5800804F05D04FF4804B1960A3F804B00833B6
:102D6800D20B04D04FF4004219609A80083301F561
:102D78008061A1427FF47EAFBDE8F08F346D030817
:102D88005058002000180048002852D0036803F16A
:102D980038422DE9F04F920A504DAA5C02F01F0507
:102DA80052090124022A04FA05F443D0032A00F048
:102DB8009080012A43D001F003077A1E012AC1F34B
:102DC800810CC1F300188088C1F341113CD9C607B2
:102DD80000F18880850700F19480440700F1A28003
:102DE800020700F1B080C60600F1BE80850600F13A
:102DF800CC80440600F1DA80020600F1E880C605BE
:102E080000F1F680850500F10481440500F1128186
:102E1800020500F12081C60400F12E81850400F12D
:102E28003C81440400F14A81020400F15881BDE864
:102E3800F08F70472A4A95692C439461BBE7284A6A
:102E480055692C435461B6E7002422464FF0010E21
:102E58004FF0030904E00132102A04F10204E6D01D
:102E68000EFA02F636EA0005F5D1D3F808A009FAF9
:102E780004F5ED430AEA050AC3F808A0D3F808B038
:102E88000CFA04FA4AEA0B0AC3F808A0B3F804A03B
:102E98001FFA8AFA2AEA06069E80B3F804A008FAFE
:102EA80002F646EA0A06B6B29E801E682E401E60EA
:102EB800D3F800A007FA04F646EA0A061E60D3F81B
:102EC8000CA001FA04F605EA0A0A46EA0A05DD60DA
:102ED800C1E7034AD5692C43D4616CE7486D030800
:102EE800001002401A6822F003021A601A683A4376
:102EF8001A60DA6822F003020A438507DA607FF570
:102F08006CAF1A6822F00C021A601A6842EA87024B
:102F18001A60DA6822F00C0242EA81024407DA6099
:102F28007FF55EAF1A6822F030021A601A6842EA2A
:102F380007121A60DA6822F0300242EA0112DA60F7
:102F480002077FF550AF1A6822F0C0021A601A68AB
:102F580042EA87121A60DA6822F0C00242EA811255
:102F6800C606DA607FF542AF1A6822F440721A602A
:102F78001A6842EA07221A60DA6822F4407242EAC2
:102F880001228506DA607FF534AF1A6822F44062C0
:102F98001A601A6842EA87221A60DA6822F44062E4
:102FA80042EA81224406DA607FF526AF1A6822F4E5
:102FB80040521A601A6842EA07321A60DA6822F444
:102FC800405242EA0132DA6002067FF518AF1A6809
:102FD80022F440421A601A6842EA87321A60DA68B4
:102FE80022F4404242EA8132C605DA607FF50AAF30
:102FF8001A6822F440321A601A6842EA07421A60D4
:10300800DA6822F4403242EA01428505DA607FF547
:10301800FCAE1A6822F440221A601A6842EA874213
:103028001A60DA6822F4402242EA81424405DA60F2
:103038007FF5EEAE1A6822F440121A601A6842EA66
:1030480007521A60DA6822F4401242EA0152DA6042
:1030580002057FF5E0AE1A6822F440021A601A6889
:1030680042EA87521A60DA6822F4400242EA815240
:10307800C604DA607FF5D2AE1A6822F040721A6090
:103088001A6842EA07621A60DA6822F0407242EA75
:1030980001628504DA607FF5C4AE1A6822F04062E6
:1030A8001A601A6842EA87621A60DA6822F0406297
:1030B80042EA81624404DA607FF5B6AE1A6822F00B
:1030C80040521A601A6842EA07721A60DA6822F0F7
:1030D800405242EA0172DA6002047FF5A8AE1A682B
:1030E80022F040421A601A6842EA87771F60DA685D
:1030F80022F0404242EA8171D960BDE8F08F00BFFA
:1031080010B1036882881A85704700BF10B1036840
:1031180082889A61704700BF38B1002983880268A5
:1031280014BF002110218B40936170470E4B1B8800
:1031380001463BB90D4B0E4A1B7810680BB981F05C
:103148000101E9E70B4B5A691AB118B91A681060FE
:1031580058747047084A18681188084A92FBF1F2B7
:103168000121026059747047546B0020566B00208F
:10317800586B00205C6B0020746B002020A10700B6
:1031880010B40A4B0A4A1C7801238340234052F8A2
:10319800200029B9B3FA83F149095DF8044BBBE76C
:1031A800191C18BF01215DF8044BB5E7446B0020DA
:1031B800486B00201C4C08B501210220FFF7E0FFF6
:1031C800237803F00502052A2AD003F00903092B06
:1031D80008D000210120FFF7D3FF00210846FFF7A0
:1031E800CFFFFEE7114A124B11681A680B68114CA1
:1031F8004FF6FE7003400B601388206823F001032C
:103208001B041B0C138018B1292200238271C3717F
:1032180002224E21FEF758FC2068FFF771FFD8E71D
:1032280019F0AAFB2378D0E7A8670020B44C002047
:10323800B84C0020BC4C002030B1036882881B8A3F
:103248001A4214BF01200020704700BF38B5044659
:1032580090F84D0000285AD104F11805636D8022BA
:103268006B21284698476420FFF72AFB636D0722E5
:103278006821284698476420FFF722FB636D0022E7
:103288006B21284698476420FFF71AFB636D0122DB
:103298006B21284698470F20FFF712FB94F8472028
:1032A800636D032A34BF18221A221B212846984727
:1032B8000F20FFF705FB636D18221C21284698474D
:1032C8000F20FFF7FDFA636D94F846201A2128466F
:1032D80098470F20FFF7F4FA636D94F848201921F6
:1032E800284698476420FFF7EBFA636D10223721D0
:1032F800284698470F20FFF7E3FA2846636D012216
:10330800382198470F20BDE83840FFF7D9BAFEF7B3
:10331800ADFD0546FFF790FF014600289CD1D5B1C9
:103328002023E871AB712846FFF72EFD2146104B8C
:1033380041F8143F28461EF077FFAB88B3FA83F3B1
:10334800C3F11F035A1C87D001229A4009490B6810
:1033580013430B6080E72946FFF716FD2146044B0F
:1033680041F8143F28461EF05FFF0122EEE700BF38
:103378002D0C00080004014010B50446806927F0B0
:103388003FFC0120FFF734FA2046FFF75FFF1022C9
:103398006A2104F11800FDF707F96420FFF790FA95
:1033A800A06927F01BFC0120BDE81040FFF720BAF8
:1033B8002DE9F0410B4E346873691C400FD0DFF8DB
:1033C80028800127B4FA84F3C3F11F0307FA03F531
:1033D80058F8230003689847AC437561F2D1BDE8FB
:1033E800F08100BF00040140983F00202DE9F04122
:1033F8000B4E346873691C400FD0DFF82880012712
:10340800B4FA84F3C3F11F0307FA03F558F823004D
:1034180003689847AC437561F2D1BDE8F08100BFFD
:1034280000040140983F00202DE9F0410B4E34681C
:1034380073691C400FD0DFF828800127B4FA84F3A1
:10344800C3F11F0307FA03F558F8230003689847E8
:10345800AC437561F2D1BDE8F08100BF00040140C2
:10346800983F00202DE9F0410B4E346873691C40E9
:103478000FD0DFF828800127B4FA84F3C3F11F03C3
:1034880007FA03F558F8230003689847AC437561B9
:10349800F2D1BDE8F08100BF00040140983F002050
:1034A8002DE9F0410B4E346873691C400FD0DFF8EA
:1034B80028800127B4FA84F3C3F11F0307FA03F540
:1034C80058F8230003689847AC437561F2D1BDE80A
:1034D800F08100BF00040140983F00202DE9F04131
:1034E8000B4E346873691C400FD0DFF82880012721
:1034F800B4FA84F3C3F11F0307FA03F558F823005D
:1035080003689847AC437561F2D1BDE8F08100BF0C
:1035180000040140983F00202DE9F0410B4E34682B
:1035280073691C400FD0DFF828800127B4FA84F3B0
:10353800C3F11F0307FA03F558F8230003689847F7
:10354800AC437561F2D1BDE8F08100BF00040140D1
:10355800983F0020084A094808B5936943F00103D9
:1035680093610021402231F034FB054B4FF0FF32CC
:103578001A60C3F8032008BD00100240983F0020DD
:10358800D83F00202DE9F041044618460D4616465E
:1035980098462DF0C5FE2768E6722844A072294691
:1035A8007D69434632462046AC46BDE8F041604757
:1035B800036810B504461B689847236820469B6833
:1035C8009847A37B0133A37310BD00BF10B50368F0
:1035D80004469B689847FF2301226373227310BD3A
:1035E80008B5FEF743FC40B12C2282710022C2715B
:1035F8002021BDE80840FFF7C7BB08BDF0B48489A7
:103608004FF6FF764FF47A743BB3002A37D0177819
:10361800013201E0B44219D00589013C15F00205D8
:10362800A4B2F7D007734FF47A7402E0BCB2B44284
:103638000CD0058915F0010504F1FF37F6D0057B9C
:10364800EDB209B10D700131013BDDE70D4B984238
:1036580007D0A3F57843984202D00120F0BC704708
:103668000125094B03EB05156B8901339BB26B816F
:10367800688980B2003018BF0120F0BC7047FF276E
:10368800CAE700BF00300140146B0020F8B50446BB
:1036980040681F4610B103688088188541F0800192
:1036A800206840F2E93300E003B30589013B15F0D7
:1036B800020F9BB2F8D0017300F10C0640F2E93317
:1036C80000E01BB30589013B15F0010F9BB2F8D050
:1036D80033782068134639460022FFF78FFF636866
:1036E80013B11A689B8893610120F8BD104988427C
:1036F80003D0104B9842EDD101230F4901EB03137E
:103708005989013189B259815B89E3E708498842BF
:1037180003D0084B9842DCD10123074901EB03137E
:103728005989013189B259815B892068D2E700BF84
:103738000030014000380040146B002038B50B4CB5
:103748002378054653B90A4B6278186849212B46F5
:1037580000252570FFF79AFF012038BDFFF7A2F872
:103768000028F0D0FFF744F8EDE700BFE43F002061
:10377800E03F0020F0B54A4C257C012D83B013D0E2
:1037880028D3022D0DD1474B1B780646002B77D145
:103798006846FFF7D3FF20B19DF8063013F0030009
:1037A80022D0002003B0F0BD3E4E3378002B62D10A
:1037B8006846FFF7C3FF9DF8003008B1DB0764D403
:1037C8000023237433784BB1002301330020237482
:1037D80003B0F0BD334E3378002BF5D10121022020
:1037E8001EF024FE237CF0E79DF801E09DF8001010
:1037F8009DF803709DF802209DF805509DF804304F
:10380800207441EA0E2142EA072243EA052309B25D
:1038180012B21BB2494252425B42234806EE901A4A
:1038280007EE102A07EE903A90ED005AD0ED015AB3
:1038380090ED026AF8EEE66AB8EEC77AF8EEE77A33
:1038480066EE856A27EE257A67EE867AFDEEE66AE9
:10385800BDEEC77AFDEEE77A16EE901A17EE102A3B
:1038680017EE903A31807280B38001210A201EF051
:103878008FFD03B0F0BDFFF715F8002898D090E74A
:10388800FFF710F800288CD182E7337823B9072195
:1038980003201EF0CBFD257C0135257481E700BF90
:1038A800301E0020E43F002000000020F8B505018C
:1038B8005A4C5B4B625961199A4204EB050704BFE5
:1038C80001230B730646387A26F03EFD3B7A03F057
:1038D8001F015B090122022B02FA01F278D0032BA7
:1038E80071D0012B67D0631901361879FEF7BEFA3B
:1038F800F6B2074610B11223C6718371631958795D
:10390800FEF7B4FA10B11323C6718371631998795D
:10391800FEF7ACFA10B11423C671837166190E2133
:10392800F2793846FEF7D0F87079FEF79FFAF27907
:103938000E21FEF7C9F8B079FEF798FAF2790E2150
:10394800FEF7C2F86359374A934251D0344A93423A
:1039580059D0354A934240D02C44227B002A2FD19B
:10396800012002249A8822F480521204120C9A80B0
:10397800998889B241F4805199801A8802F4415299
:1039880042F44572024322431A809A8822F47062F4
:103998001204120C42F4E0629A809A8B22F40062BC
:1039A8001204120C07219A8319821A8892B242F0E3
:1039B80040021A80F8BD1D4B996A0A439A6292E741
:1039C80000200446CEE7194B19690A431A618AE7B1
:1039D800164BD9680A43DA6085E702F5EA321169BD
:1039E80041F400411161116921F400411161B3E70B
:1039F80002F56042D16841F48051D160D16821F468
:103A08008051D160A8E702F5EC32116941F4804198
:103A18001161116921F4804111619DE7146B002047
:103A28000038004000300140003C004000100240D7
:103A3800427A02B9704710B504460368406804F139
:103A48000A0198470023637210BD00BF437A5A1CCD
:103A58000344D2B242729972037A934200D802B9EF
:103A6800704710B504460368406804F10A01984796
:103A78000023637210BD00BF30B40B4D002305F165
:103A8800800101E0272B0CD011F8132082424FEA65
:103A9800430403F10103F5D12C4494F8810030BCB0
:103AA8007047002030BC7047444D0308064B074957
:103AB8008B4202D30023184670471A88C2F30B02C0
:103AC8009042F8D01433F3E768B00308B4B403089D
:103AD800024A136823EA000010607047008F002034
:103AE8002DE9F047A84FA94E15F010FEBE421ED290
:103AF800DFF82083DFF820934446258862197DB1DA
:103B08004A450DD2052D0BD933886188C3F30B03C1
:103B1800994200F0D880144625886219002DEFD10B
:103B2800716830461436FDF703FABE42E4D3984A6A
:103B38005378022B40F2EC80002396495370137897
:103B48009548022B016000F2DF8003EBC301934A22
:103B580003EB810302EB4303914C1846236029F0E1
:103B6800A9FE904A1378A3F1170102290FD98E49AB
:103B780011F83300002840F0D180D800014449787A
:103B880029B18A4911F83330002B00F0F580884BB1
:103B98009A78042A00F0E78032B91A88B2F5F07FE3
:103BA80084BF4FF4F0721A808249834A0B681A4026
:103BB800002A00F0E480DE0700F1D0805D0400F107
:103BC800C880180700F1C0809A0100F1B7809B04F3
:103BD80000F1AD8023689A8CD98C914224BF0022D1
:103BE8009A84FDF78BFC21F04BFE10B973481FF047
:103BF800EFFB10F0E9FF00213022714830F0E9FFB7
:103C0800704B266803F1500102E00433994279D0E1
:103C18001A78002AF9D19C78D8788442F5D26A4972
:103C28006A4B91F800E06A486A4D1C6B6A4B286041
:103C3800C827642111FB0E71DFF8E0E15960674F76
:103C480030F8041C664DAEF8001000219960D96068
:103C5800196159619961D96183F8201083F821109D
:103C68003A702E600CB114F053FB5E4B9FED5E5A18
:103C78001B885E4A9FED5E6A557E5E4C5E495F48D2
:103C8800086006EE903AF8EEE66A938AC5EE265A80
:103C980007EE103AD38A127EC4ED005A07EE903A26
:103CA800B8EEC77A564BF8EEE77A1D725A7227EECD
:103CB800067A67EE867ABDE8F04783ED017AC3EDB0
:103CC800007A15F00BBD63799B077FF424AF716808
:103CD80094F804A03046FDF72BF93388BAEB133F6C
:103CE8000BD173887068AA1FC3F30B039A4204F1BF
:103CF8000601A8BF1A462EF057FC1436BE42FFF440
:103D0800FBAE14E701228AE700231370234B23E755
:103D1800204903EB430301EB830110E7D8000D189A
:103D28006D68002D7FF42AAF1725157026E73548F2
:103D3800FFF7CEFE4020FFF7CBFE4BE746F2090027
:103D4800FFF7C6FE0B6842E72F48FFF7C1FE0B6876
:103D58003AE72E48FFF7BCFE0B6832E72C48FFF71E
:103D6800B7FE0B682AE71A8BB2F57A7FBFF41CAF4F
:103D78004FF47A721A8317E71823137007E743F092
:103D880001030B6017E700BFB4B4030868B0030869
:103D9800683E0020E43A002078260020F08D0020BC
:103DA800843E00208C2B002034710308BC74030867
:103DB80080590020008F002009600002DC430020A9
:103DC800F41F0020902B0020F4370020083B00202F
:103DD8001C290020B8950020303E00202C0000202F
:103DE80028200020BC1E0020C0C9FB48301E00202F
:103DF80017B7D138C01E0020B83000203661023D08
:103E080094300020094000020160000209200002ED
:103E18000860000207F003080000040826290020B3
:103E2800F8B51A4D2B789F2B2ED16B78BE2B2BD142
:103E380005221749A81C30F017FF28BB072229467E
:103E48004FF6FF70FCF7E8FC124FEC1D22884AB1D0
:103E5800A618BE4218D2052A16D92146FCF7DCFC62
:103E68003446F3E721460222FCF7D6FC0222A118C9
:103E7800FCF7D2FC0634084B641B1C8041F60F5338
:103E8800C31A58425841F8BD0020F8BD00F0030895
:103E98000079030800000408BC2700202DE9F04F32
:103EA800DFF854914F4F8DB00326A7EB090718226E
:103EB8000DEB0200002130F08CFE4B4BCDF8189032
:103EC80007971A69120604D5484A5A6002F18832DF
:103ED8005A6001228DF82C203422DA60444B454C7C
:103EE80018689A8804909B79ADF8142004A90722D1
:103EF80006A88DF81630FDF7D7F9072204A94FF662
:103F0800FF70FCF789FCDFF8F4B080464FF0000A38
:103F18005C4536D30CAC002524F82C5D02222146E2
:103F280006A8FDF7C1F9022221464046FCF774FCB9
:103F380040BAC043ADF80800022202A906A8FDF75E
:103F4800B3F9099860B108ABC0F1040229461844D6
:103F580030F03FFE089906A8FDF74CF909950A903C
:103F68009DF82C300A9A23B11F490B6943F080034E
:103F78000B61013E2DD0002A99D1FFF751FF50B3B4
:103F88002CE065888DF80DA0C5F30B05AA1DADF8CA
:103F980008202288C2F30B01120BADF80A108DF825
:103FA8000C2002A9062206A8FDF77EF9062202A91E
:103FB8004046FCF731FC616880462A4606A8FDF7B2
:103FC80073F9616840462A46FCF726FC143480469B
:103FD8009EE7002AD1D00520FEF768F90DB0BDE8AC
:103FE800F08F00BF0000040800200240230167454D
:103FF800124E030868B0030800F00308B4B40308BD
:1040080008B515F083FBFFF749FF15F067FBFFF7CD
:1040180067FD0120BDE8084020F0ECB908B5FDF7C0
:10402800FFFA15F073FBFFF739FFBDE8084015F0FC
:1040380055BB00BF08B515F069FBFFF72FFFBDE8BA
:10404800084015F04BBB00BF0378202B024600F157
:104058000100F9D0092BF7D02D2B2CD02B2B03BF27
:104068005378B7EE000A0246B7EE000AA3F1300112
:10407800C8B209289FED467A10D8F2EE046A07EE16
:10408800901AF8EEE77A12F8013FE7EE267AA3F1E4
:104098003001C8B20928B0EE677AF0D92E2B4CD07F
:1040A80003F0DF03452B0BD0F7EE007A67EE276AA3
:1040B80020EE260A70475378BFEE000A0246D5E77D
:1040C80010B451782D2959D02B290ABF9178501C4A
:1040D800901C0024A1F13003092B53D8002303EBD3
:1040E800830301EB430310F8011FA1F13002092AF1
:1040F800A3F13003F3D9B3F59A7F28BF4FF49A732D
:10410800072B42D9DFED236A1A46F7EE007A083A00
:10411800072A67EEA67AFAD803F007032BB1F2EE66
:10412800046A013B67EEA67AFBD124B3C7EE276A7F
:104138005DF8044B20EE260A70475378A3F130014E
:10414800C8B2092802F10102AAD8F2EE046AF0EE18
:10415800665A07EE901AF8EEE77A12F8013F87EEF2
:10416800A66AA3F13001C8B2092866EEA56A37EE3F
:10417800067AEED994E767EE276AD9E7901C91781A
:104188000124A7E7F7EE007ACFE7F7EE007AC5E754
:104198000000000020BCBE4CB5EEC00ADFED317A4D
:1041A800F1EE10FACCBF30EE270A30EE670ADFEDE9
:1041B8002E7A20EE270A30B5FDEEC07A87B017EECA
:1041C800904A054684EAE470002303A9A0EBE47052
:1041D80001930093029328F099F8002CACBF202398
:1041E8002D2303A88DF800302DF09AF8012803A993
:1041F80024D002282DD0032805BF302368466846FE
:104208008DF8013030F00BFD68462DF089F8033841
:10421800C4B222466946284630F05FFD00232B557C
:1042280028462DF07DF82E22431C2A540DEB04015C
:10423800E81830F011FD284607B030BD3023684635
:104248008DF801308DF802308DF8033030F0E7FC3E
:10425800DAE7302368468DF801308DF8023030F007
:10426800DEFCD1E76F12033A00007A442DE9F041F1
:10427800064615460846B6FBF2F43CB905FB14643D
:10428800124B1B5D00F8013BBDE8F081B4FBF2F76F
:1042980067B90E4B05FB174705FB1464DA5D00F898
:1042A800012B1B5D00F8013BBDE8F081B7FBF2F87C
:1042B800B8F1000F02D04046FFF7D8FF05FB187889
:1042C800024B13F8082000F8012BE3E708790308EC
:1042D8000368591C1A46016012F8021B02605878DC
:1042E80041EA0020704700BF38B50446006815460B
:1042F8002EF05AF922682A44226038BD036810B4A7
:104308000A0A5C1C04601A7003685A1C026019705F
:104318005DF8044B704700BF03685A1C026010B474
:10432800197003680A0A5C1C04601A7003680A0C96
:104338005C1C04601A700368090E5A1C026019702C
:104348005DF8044B704700BF03685A1C026019707F
:104358000368090A5A1C0260197070472DE9F04772
:10436800002488B080460F461E46A14605AD531C62
:104378000393117839B3252933D1931CCDF81090C4
:104388000393507830284ED04FF0000AA0F1300344
:10439800DBB2092B42D96C2819D0642800F093802D
:1043A80024D825281CD063D9582876D063281BD157
:1043B80031784046B847039A531C03931178043662
:1043C80001340029D7D1204608B0BDE8F087039B07
:1043D8005A1C03921B78642B7CD02AD8252B54D1E5
:1043E800252140460134B847039AC0E7732833D0E3
:1043F80044D975284FD106F1040E30682B460022A7
:104408000A217646FCF78CF9049A009553463946FA
:104418004046FCF7C3F9039A0444A8E704AA03A991
:104428001EF04AFCB7E7D31C039390784FF0010ABB
:10443800ACE7732B10D05BD9752B3AD0782B96D17B
:10444800A3F15802B2FA82F2306852092B461021C1
:104458000436FCF765F9D7E73368049A00933946C0
:1044680000234046FCF79AF904360444039A7EE791
:104478000028B9D1204608B0BDE8F0876E28B3D12E
:10448800039A336804361C6071E72AD9582BD7D0B1
:10449800632B8DD06BE77828A6D1A0F15802B2FA29
:1044A80082F2306852092B461021FCF739F904369C
:1044B800AAE706F1040E30682B4600220A21764648
:1044C800FCF72EF9A0E7331D306829461E46FCF795
:1044D800F9F899E7331D306829461E46FCF7F2F8CB
:1044E80092E7002B7FF443AF204608B0BDE8F08781
:1044F8006E2BC6D03BE700BF0EB400B584B005AB49
:10450800019053F8042B0649039301A8FFF726FFEF
:10451800019B00221A7004B05DF804EB03B07047E9
:10452800990700080FB430B583B006AB0B490C48A7
:1045380053F8042B096800680193FFF70FFF094C33
:104548000546206803685B6998470028F9D0284623
:1045580003B0BDE8304004B0704700BFA06700203A
:10456800A467002030200020DFED2B7AB4EEE70AA4
:10457800F1EE10FA4ADDDFED296A9FED297A01E0B4
:10458800B0EE670AB4EEC70AF1EE10FA70EE667A7A
:10459800F6DC9FED247AF4EEC77AF1EE10FA38D5FE
:1045A800DFED1E6A9FED207A01E0F0EE407AF4EE2E
:1045B800C77AF1EE10FA37EEA60AF6D4DFED1B7AC9
:1045C800B4EEE70AF1EE10FA14DDDFED137A37EEF8
:1045D800C00A60EE006A9FED166A9FED167ADFED5D
:1045E800167AA6EE867A20EE266AE6EE877AA6EE98
:1045F800270A7047DFED117AB4EEE70AF1EE10FAF8
:1046080044BFDFED087A37EEC00AE2E7F0EE407A01
:10461800BFE7B0EE670AD1E7DB0F4940DB0FC940BF
:10462800E4CB1641DB0F49C0E4CB16C1DB0FC93F11
:1046380092E741B99730083C15A82ABEDB0FC9BFDD
:1046480041404A0011F0800F82F0D503D2B2DBB2AC
:1046580008BF1346590013F0800F81F0D502C9B284
:10466800D2B208BF0A46510012F0800F81F0D5037C
:10467800C9B2DBB208BF0B46590013F0800F81F0B6
:10468800D502C9B2D2B208BF0A46510012F0800F53
:1046980081F0D503C9B2DBB208BF0B46590013F04D
:1046A800800F81F0D502C9B2D2B208BF0A465100C4
:1046B80012F0800F81F0D503C9B2DBB208BF0B46F8
:1046C8005A0082F0D50013F0800FD2B2C0B208BFF2
:1046D8001046704780EAE073A3EBE0738B4205DB7A
:1046E800002801DD401A704702D17047002070474A
:1046F8000844704709B909E0194690FBF1F301FB3A
:1047080013030846002BF7D1084670470146FBE71C
:1047180010B507EE901A2DED028BB8EE678ADFED23
:10472800227A28EE008A044628EE278AB0EE480A44
:104738002EF08EF9F0EE408AB0EE480A2EF0EAF834
:10474800F7EE007A9FED197AF0EE675AE8EE875A8D
:104758000023A361B0EE676AC7EEA56A63612362AE
:10476800E361A3626362A8EEC76ABDEC028B77EED1
:10477800C07AB6EE007AF8EE005A27EE877A20EE75
:10478800250A27EE267A26EE266A67EEA67A20EE16
:10479800260A84ED046AC4ED017A84ED007A84ED7A
:1047A800027A84ED030A10BD27D4D236F304353FCC
:1047B8004B0901F01F0150F82320012303FA01F1EE
:1047C800114214BF18460020704700BFF0B5484B8F
:1047D80048491A68096883B00123560200935CBFF0
:1047E80003F180530093D4005CBF43F0100300939F
:1047F800880744BF43F0C60300934F0744BF43F004
:10480800080300930E073C4948BF43F0200309788A
:1048180048BF0093D40548BF43F0006301F0EF00A0
:1048280048BF009308286D4655D00E2953D0D003B1
:104838003248009B00784CBF43F4204343F40053B4
:10484800D7044CBF43F0C84343F0884300280CBF4B
:1048580007200F20960648BF43F48073540748BFCB
:1048680043F4003343F400245205009402D5244A4B
:104878001279A2BB182936D00190002701263946A3
:104888002846FCB2FFF794FF60B11E4B002203F5E7
:10489800D87103E08B420FD013F80C2CA24203F11D
:1048A8000C03F7D10137242FE9D195E80300164B03
:1048B80083E8030003B0F0BD7A0904F01F0455F83B
:1048C800223006FA04F4013723EA0404242F45F8B9
:1048D8002240D4D1E9E743F480530093A7E743F497
:1048E800C0130093C6E7009B43F060730093C3E7CF
:1048F800686C0020D45100208C2B0020A85900207F
:1049080034690020AC4E0308841E00202DE9F84FBE
:104918004E014FF0000B174D8146904606F12007D7
:104928005C46594628465FFA8BFAFFF741FFC0B14B
:10493800A64215D8A74213D900200F4A014604E021
:104948000131242914D012F80C0C504502F10C0244
:10495800F6D10A4B01EB410103EB81014846C04700
:1049680001340BF1010BBBF1240FDAD1BDE8F88F4C
:104978000021F3E7841E0020AC4E0308A04E030874
:10498800B0F1FF3F0AD0022810B403DC5DF8044BF5
:10499800FCF74EBA00205DF8044B704700207047C2
:1049A8003123F42276210020EAE700BFF0B5574B07
:1049B800574A97B01968914200AF00F09C8055495A
:1049C800554A00234FF47000C1F888003B607B60B3
:1049D800136843F48033136003E03B68B3F5A04FDA
:1049E80009D0136803F400337B603B6801333B60F4
:1049F8007B68002BF1D0484B1B6813F4003318BFB9
:104A080001237B607B68012B4BD0424D424B434ACC
:104A1800EA60434A596A11605A6A424E42F080720B
:104A28005A625A6907F1580442F4FC0241F6FF71D0
:104A38005A6124F8501D032321464FF09040BB7261
:104A4800FCF7C8F94FF6FF73214637483B81FCF75E
:104A5800C1F921463548FCF7BDF921463448FCF731
:104A6800B9F921463348FCF7B5F921463248FCF735
:104A7800B1F920461BF08CF8BB683049304AA1FBDD
:104A8800031330499B0CF02400204FF0070E5C37CD
:104A98000B60566085F823409060C2F800E0BD4680
:104AA800F0BD294A1C4B122111605A685A605A6895
:104AB8005A605A6842F480625A605A6822F47C123A
:104AC8005A605A6842F4E8125A601A6842F08072D2
:104AD8001A601A689201FCD559680F4A21F003013F
:104AE8005960596841F002015960536803F00C039A
:104AF800082BFAD189E700221A6062B6134B1B68AB
:104B080083F30888124B1B689847FEE7FC9F002038
:104B1800EFBEADDE00ED00E0001002400005FA0532
:104B2800646C00203F190100000400480008004898
:104B3800000C0048001000480014004883DE1B43A6
:104B480010E000E0BC6A00200020024000D8FF1FEF
:104B580004D8FF1F064A00235168814202F11C0253
:104B680004D001330C2BF7D100207047D8B270471E
:104B78003000002070B50F4C0F4DC0EBC00004EBA7
:104B88008004686926693043686182B09209667B4F
:104B9800A1600025012101A863618DF804608DF8EA
:104BA80005208DF806508DF8071025F057FE02B045
:104BB80070BD00BF3000002000100240074BC0EB62
:104BC800C00030B403EB8000054C056963692B43D2
:104BD80063610176427630BC704700BF3000002028
:104BE800001002402DE9F04F554C54F8204083B096
:104BF800002C60D0656D1F469046524B6A6822654E
:104C0800A160236004F15A014FF4807304F5AD727A
:104C18006161A261E36023610646287E25F094FB6A
:104C2800E86858B1FFF796FF721CD2B20C21FFF763
:104C3800C5FF236DEA6822632433E364A86890B152
:104C4800FFF788FF721C8146D2B20B21FFF7B6FF2F
:104C58002346EA7E3C494846FFF78CFF236DAA6845
:104C680062632833A36494F85900FDF7FFF881467E
:104C780094F85800FDF7FAF83A07824695F819B003
:104C88001DD5B9F1000F1AD017F0110F4FF00B0313
:104C980006F1010614BF4E213E2189F8063089F835
:104CA80007605A464846FCF70FFFFB0743D5236BBE
:104CB8006BB3636B5BB3204603B0BDE8F08F17F0AE
:104CC800010F0CBF2E274E2718F0020F0DD0B9F197
:104CD800000F0AD00B22731C89F8062089F80730C8
:104CE80048465A463946FCF7EFFE18F0010FDED069
:104CF800BAF1000FDBD001360C238AF807605A4658
:104D080039468AF806305046FCF7DEFECFE72B7F9F
:104D1800AA7E8DF804209B090021012201A88DF8A4
:104D280005308DF806108DF8072025F097FD2046F0
:104D380003B0BDE8F08F4846FEF7E2F9B7E700BFD9
:104D4800AC6700201C4E0308DD0C00080348D0F8AF
:104D58003C3113B100F59A701847704730000020B5
:104D68000348D0F8203113B100F58C70184770470C
:104D7800300000200348D0F804310BB1FC3018474C
:104D8800704700BF300000200348D0F8E8300BB16E
:104D9800E0301847704700BF300000200348D0F8C3
:104DA800CC300BB1C4301847704700BF300000202A
:104DB8000348D0F8B0300BB1A8301847704700BF8F
:104DC800300000200348D0F894300BB18C301847DD
:104DD800704700BF300000200248836F0BB170306D
:104DE80018477047300000200248C36D0BB154309B
:104DF80018477047300000200248036C0BB1383068
:104E080018477047300000200248436A0BB11C3035
:104E180018477047300000200248836803B11847DC
:104E2800704700BF300000201749184B184A19482E
:104E380010B4D1F8884044F47004C1F888401C6864
:104E480044F001041C605C6822405A601A6822F031
:104E5800847222F480321A601A6822F480221A605E
:104E68005A6822F4FE025A60DA6A22F00F02DA6205
:104E78001A6B002410404FF0006218639C608A602F
:104E88005DF8044B704700BF00ED00E000100240E1
:104E98000CC07FF8CCFC00FF38282DE9F04700F063
:104EA80097810C462ED9802800F0F68074D85228B5
:104EB80000F0898040F24C81542800F0B2816E28BD
:104EC80040F0AC81B04B0A681B88B04DFF2BA8BFDF
:104ED800FF23511C21601370A96881F3100120463B
:104EE80089B2FFF731FAAA4B20461988FFF72CFA46
:104EF800296801F30F01204689B2FFF725FA01203E
:104F0800BDE8F087042800F03F8240F2EE802028B8
:104F180000F0A18040F22481242800F0D2812828C2
:104F280040F07C810B68DFF89C829A4E591C022263
:104F380021601A70236806275A1C22601F70236894
:104F48000A22591C21601A70236801255A19226007
:104F58001D70B8F800102046FFF7F6F9B8F80210EF
:104F68002046FFF7F1F923685A1922601F70236859
:104F78005022591921601A7023680022591921609A
:104F88001A7031882046FFF7DFF920467188FFF74D
:104F9800DBF92846BDE8F08782282FD0C0F0AB8126
:104FA800A02800F09681FE2840F038817A4D05F15E
:104FB800080635F8021B2046FFF7C6F9AE42F8D1BD
:104FC8000120BDE8F0870A68744E531C0321236052
:104FD80006F10C0711703346062001212268551C82
:104FE8002560117022689F4202F101012160107052
:104FF80000F0DB819979D8790633EFE70B68684AC6
:10500800624D1178674A581C20601970D188204673
:10501800FFF79AF95C4B22681B88FF2B02F101010C
:10502800A8BFFF2321601370A96881F310012046EF
:1050380089B2FFF789F9296801F30F01204689B27F
:10504800FFF782F92368584A591C127821601A70B0
:105058000120BDE8F0870B68524D591C6A78216021
:105068001A7023682A78591C21601A702368AA7854
:10507800591C21601A70E9882046FFF765F92368F2
:105088002A79591C21601A7023686A79591C216091
:105098001A700120BDE8F087DFF82C81434F444E99
:1050A800DFF828A108F10D090A2515E0322D34D0C2
:1050B800A5F13C00C0B2132835D900232268511C41
:1050C800216015702268C84502F101012160137042
:1050D8003FF476AF18F8015B0A2DE7D1BAF8003033
:1050E800FF2BA8BFFF23DBB2E8E7022800F08D8181
:1050F80000F27A81012840F091800B680022591C47
:1051080021601A7023685A1C2260187023682422B0
:10511800591C21601A70BDE8F0873388FF2BA8BF9F
:10512800FF23DBB2CAE724F097FB0028C5D0037839
:105138000A2B00F27281B0F9023087FB0312DB17E9
:10514800C3EBA2039BB2FF2BA8BFFF23DBB2B5E7DB
:10515800442863D1002A3FF433AF164B13602FE77E
:1051680005285BD120460B221349FFF7BDF82046DE
:1051780008221249FFF7B8F8204607221049FFF71E
:10518800B3F80120BDE8F0871C69002020690020E1
:10519800089400207C600020886800207C6B03084D
:1051A80073690020DC930020189400206766666607
:1051B800485F0020A90F0008407903084C790308CC
:1051C80058790308201F0020554E0308785F0020F7
:1051D8000B689E4A01205C1C0C6018700B68052443
:1051E8001D180D601C700B680A241D180D601C70BA
:1051F8000B6800241D180D601C700B6814781D18AE
:105208000D601C700B6854781D180D601C700B68BD
:1052180092781C180C601A70BDE8F0870020BDE871
:10522800F0870B688A4F591C012221601A70236885
:1052380000259A1822601D70236897F85C20591C75
:1052480021601A70236897F85620591C21601A703B
:10525800B7F858102046FFF777F829462046FFF799
:1052680073F8B7F85A102046FFF76EF8BD1E07F11D
:10527800480635F8021F2046FFF766F8AE42F8D117
:105288002268744B0C21501C20605D181170226834
:1052980013F8011F501C9D4220601170F7D123683C
:1052A8000222591C21601A70B7F85E102046FFF7D9
:1052B8004BF82046B7F86010FFF746F80120BDE824
:1052C800F087654B08461968FFF726F80120BDE806
:1052D800F087624B08461968FFF71EF8604B2046B6
:1052E8001968FFF719F85F4B20461968FFF714F89B
:1052F8000120BDE8F087DFF88C915B4F09F10F06BC
:105308004FF00A0820E0B8F1500F35D0B8F15A0F25
:1053180034D0B8F1320F34D0A8F13C00C0B2132811
:105328007DD90025294623685A1C2260204683F827
:105338000080FFF709F829462046FFF705F84E4593
:105348003FF43EAE19F8018BB8F10A0FDBD1474B99
:105358009D68196805EB85054FF6FF736D009D4242
:10536800A8BF1D469942A8BF194625EAE57521EA56
:10537800E171ADB289B2D6E73D4BE9E73D4B5D68D7
:10538800E7E797E82200E5E702463B492046FEF7B3
:10539800ABFF20460021FEF7D7FF23680022591CE7
:1053A80021601A700120BDE8F087344B21681A7813
:1053B800481C20600A70002A3FF402AE013AD2B2BB
:1053C80002EB420206EB42025278002A3FF4F8ADA3
:1053D8000132D5180133226813F8011F501C9D4271
:1053E80020601170F7D1EBE50B680222591C21608F
:1053F8001A70236801201A18226018702368002286
:10540800191821601A70BDE8F087084604221C4963
:10541800FEF76AFF0120BDE8F087002396E624F036
:105428001BFA00283FF47DAF03780A2B3FF679AFCB
:10543800B0F90430B0F9061003EB830383F3500589
:1054480021EAE171ADB289B26DE700BFDF8D0020BE
:1054580070930020B9930020008F0020ACF7FF1F45
:10546800B0F7FF1FB4F7FF1F80600020B05F002077
:10547800EC5F0020F85F002038790308E040002046
:1054880030790308454E03082DE9F04F80462DED8D
:10549800048BB0F908000881C5B28FB028460C46C5
:1054A8009146FFF7F9FC40B101231A46184662817C
:1054B8000FB0BDEC048BBDE8F08FA5F10A03E72B14
:1054C80000F2EA80DFE813F0D105E800E800E80020
:1054D800E800E800E800E800E800E800E800E80084
:1054E800E800E800E800E800E800E800E800E80074
:1054F800E800E800E800E800E305E800E800E80064
:105508003206E800E800E800CF04E800D304E80029
:105518001305E8002C05E8003805E8003C05E8001C
:105528006205E800E800E800BB01D801E800C20114
:10553800E800E800D001E800E800E800E800E8003A
:10554800AE01E800E800E800E800E001E800FB013F
:10555800E8001C024202E800E800E800E800E80071
:10556800E800E800D402E8005902E800A602E800D2
:105578001703E8009F06E800E800E800E800430693
:105588006C068C049504BD04E800E800B006AE0380
:10559800E800BB03F403E800E800E800E80024049E
:1055A800E800E8003004E800E800E800520463047A
:1055B8007C046003E800E800E8009E03E8001406A5
:1055C800E800E800E800E800E800E800E800E80093
:1055D800E800E800E800E800E800E800E800E80083
:1055E8004306E800E800E800E800E800E800E80012
:1055F800E800E800E800E800E800E800E800E80063
:10560800E800E800E800E800E800E800E800E80052
:10561800E800E800E800E800E800E800E800E80042
:10562800E800E800E800E800E800E800E800E80032
:10563800E800E800E800E800E800E800E800E80022
:10564800E800E800E800E800E800E800E800E80012
:10565800E800E800E800E800E800E800E800E80002
:10566800E800E800E800E800E800E800E800E800F2
:10567800E800E800E800E800E800E800E800E800E2
:10568800E800E800E800E800E800E800E800E800D2
:10569800E800E8002506A605742D44D0772D53D0E0
:1056A800F52D62D098E84800A5F12102F61A362AAD
:1056B80000F2BE86DFE812F05206BC06BC06BC0645
:1056C800BC06BC06BC06BC061206BC06BC06BC066C
:1056D800BC06BC06BC06BC06BC06BC06BC06BC06B2
:1056E800BC06BC06BC06BC06D105BC06BC06BC068E
:1056F800BC06BC06BC06BC06BC06BC06BC06BC0692
:10570800BC06BC06BC06BC06BC06BC06BC06BC0681
:10571800BC06BC06BC06BC06BC06BC067906BC06B4
:10572800EC05BC06E705D8F80030D8F804209A4202
:105738001EBF5A1CC8F800201978A54A08BF0021C6
:105748002046FFF7E3F8AFE6D8F80030D8F8042091
:105758009A421EBF5A1CC8F8002019789D4A08BFF3
:1057680000212046FFF7D2F89EE6D8F80030D8F896
:1057780004209A4241F09D86974BFF221A724FF0FF
:105788000008964D15F004FF41463022944885F8EC
:1057980000802FF01EFA8DF814809DF814300B2B22
:1057A80001F248878F4F8E4E42469DF8143003EB26
:1057B800430307EBC3035B7CE3B19DF8143003EBB1
:1057C800430307EBC3035B69A3B19DF8143003EBF4
:1057D800430307EBC3032021586946F82200FDF76D
:1057E800D3FA2B7856F82300FDF790FC2A7801327B
:1057F800D2B22A709DF814300133DBB28DF8143020
:105808009DF814300B2BD0D92368591C21601A70CD
:10581800B9F1000F3FF448AE734BC9F800300123CB
:105828001A4643E6236800255A1C2260294620466A
:105838001D70FEF771FD29462046FEF76DFD00211B
:105848002046FEF769FD01231A462FE62268674BBA
:10585800501C997820601170216858784A1C0123DF
:1058680022601A46087021E6082261492046FEF7A0
:105878003BFD01231A4619E6216801200A18226017
:1058880003460246087011E623685A4D591C2A78C7
:1058980021601A7023686A78591C21601A70698817
:1058A8002046FEF751FD23682A79591C21601A7099
:1058B800E9882046FEF748FD2168287ACEE74E4E53
:1058C8003378002B3FF4F0AD4C4F0025B8462368E1
:1058D80017F81520591C21601A7098F8011001EB6F
:1058E800810101EB810101F2EE2189B22046FEF728
:1058F8002BFD337801359D4208F10208E7DBD3E53B
:1059080023683F4D01269A1922601E7021F0D4FFAA
:10591800002841F0C5853B4B2268511C216010705E
:10592800226841F2B410511C185C216041F27811D0
:10593800107059582046890AFEF7EEFCE96B20469C
:105948004908FEF7E9FC01231A46AFE521682E4A0B
:105958000123481C20600B7021689078CD182560C1
:10596800087021681078CD18256008702168507873
:10597800CA1822601A46087098E5244EF378002B5E
:1059880001F03C8523680822591C21601A7023689D
:105998000122991821601A7023681D4D591C2A7913
:1059A80021601A702368AA78591C21601A70298806
:1059B8002046FEF7C9FC698A2046FEF7C5FC236825
:1059C800F279591C21601A702168E87846E700BF0F
:1059D800810F000889010008841E0020E189002049
:1059E8004C2F002060560020C1D00208241F002040
:1059F800805E0020F4370020903B00202C300020EF
:105A080008870020E0740020E8930020104400205C
:105A180080590020B54D23686A79B54E591C21601C
:105A28001A7033682046198CFEF78EFC33682046BE
:105A3800598CFEF789FC69892046FEF785FCA989FF
:105A48002046FEF781FC33682046998CFEF77CFCE3
:105A580033682046D98CFEF777FCE9892046FEF7A3
:105A680073FC298A2046FEF76FFC01231A461DE5C0
:105A780018F052FDFF28064601F06A850EA9002598
:105A880001F82E5D0DF109008DF8095018F024FD7C
:105A98000EA800F82D5D18F013FD0EA800F82C5D77
:105AA80018F002FD0EA820F8245D18F0F1FC236818
:105AB8005A1C22601E7023689DF80920591C216019
:105AC8001A7023689DF80A20591C21601A702368EF
:105AD8009DF80B20591C21601A7023689DF80C2032
:105AE800591C21601A70BDF814102046FEF72CFCD2
:105AF80001231A46DAE400212046FEF725FC00219E
:105B08002046FEF721FC00212046FEF71DFC2268F6
:105B1800774D0023511C2160137022682968501C9E
:105B280091F82F102060117022682968501C91F894
:105B38003A102060117022682968501C91F83B10B7
:105B4800206011702268511C216013702268511C5A
:105B5800216013702268511C216013702B68204645
:105B6800D98FFEF7F1FB2B682046998FFEF7ECFBE7
:105B780023682A68591C92F8312021601A702B6812
:105B8800216893F8320069E6DFF880E10027FEB269
:105B9800714600232268501C206016702268501C31
:105BA80020601370226811F8010F0133551C062B71
:105BB80025601070EED10137062F0EF1060EE6D1E2
:105BC8004C4900232268501C206017702268501C22
:105BD80020601370226811F8010F0133551C0B2B3C
:105BE80025601070EED12368434A581C07212060B5
:105BF800197023680021581C20601970216892F8D8
:105C0800F0002BE63D4D2046A98AFEF79DFBE98A68
:105C18002046FEF799FB298B2046FEF795FB0123CA
:105C28001A4643E4364B20461968FEF775FB354B98
:105C380020461988FEF788FB01231A4636E4324DC0
:105C480023682A68591C127821601A702B68226808
:105C58009978531C2360002311702A6821681A441C
:105C680001335279481C032B20600A70F5D1236850
:105C78002A68591C127A21601A7023682A68591CEC
:105C8800D27821601A7023682A68591C1279216019
:105C98001A702B6820465989FEF756FB23682A6834
:105CA800591C527A21601A702B6821685878D5E5FA
:105CB8000F4D00232268286803EB4301561C405C03
:105CC800266010702A6820680A44461C52782660AC
:105CD80002702A6820680A4401339278411C0A2B12
:105CE80021600270E6D1FFF7DFBB00BF104400203F
:105CF800843E0020E33D0020003D00208059002024
:105D08000C940020883E002078260020BF3D00200B
:105D1800A84952232268501C2060137011F8013FD3
:105D2800002BF7D1FFF7C0BBA34D05F16006A9888A
:105D38002046FEF709FBE9882046FEF705FB29897E
:105D48002046FEF701FB2368AA7A591C21601A70C5
:105D58002368EA7A591C21601A7055F80C1B2046F2
:105D6800FEF7DAFAAE42E2D1FFF79EBB934D20462A
:105D78002988FEF7E9FA69882046FEF7E5FAA98836
:105D88002046FEF7E1FA01231A46FFF78FBB226887
:105D98008B4B8A491878551C2560107022685878F2
:105DA800551C2560107022689B78501C2060137069
:105DB800C9882046FEF7C8FA01231A46FFF776BBC2
:105DC8002368804A80491078804A5D1C25601870D5
:105DD80023688978581C20601970216890783DE5FF
:105DE80010227B492046FEF77FFA01231A46FFF767
:105DF8005DBB784D784EDFF81482DFF81492DFED42
:105E0800778ADFED779A9FED779A05F1200708E00A
:105E180020460435FEF798FABD4206F118063FF40D
:105E280043AB717C0029F3D095ED008AB0EE480AA7
:105E38002CF0C2FD98F80030002B41F0EC8281B2C2
:105E4800E6E7694E3378002B3FF42EAB674F002509
:105E580037F8021F2046FEF777FA337801359D425E
:105E6800F6DBFFF721BB624B21681878F6E4614D39
:105E780023682A7A591C21601A70A98B2046FEF7DC
:105E880063FA298B2046FEF75FFA698B2046FEF7F6
:105E98005BFA2368EA7C591C21601A70E98C204659
:105EA800FEF752FA298D2046FEF74EFA2368AA7F9C
:105EB800591C21601A70236895F82020591C21600C
:105EC8001A70A98C2046FEF73FFA2368EA7A591C13
:105ED80021601A70E9682046FEF71EFA23682A7CBA
:105EE800591C21601A70216895F82100B6E4424DCA
:105EF80005F14006B5F880102046FEF725FA23681C
:105F080095F88220591C21601A70236895F883201F
:105F18000435591CAE4221601A70EBD1FFF7C4BAA0
:105F2800364D05F1800655F8041F2046FEF7F4F9B2
:105F3800B542F8D1FFF7B8BA2E4B2168587D8DE4E9
:105F48002F4B03F15A0522685979501C20601170B3
:105F580022681978501C2060117022685978501CEA
:105F68002060117022689978501C20601170226896
:105F7800D978501C20601170226819790633501C9A
:105F88009D4220601170DED1FFF78EBA1D4D1E4E66
:105F980005F1300795F902100023F2568A4201F004
:105FA80074810C33482BF8D10835BD42F2D1FFF784
:105FB8007BBA00BF644E03080C8D0020DC3700203C
:105FC800941E00201044002018290020F82B0020DF
:105FD800D8280020E8280020605600200000404211
:105FE8000040744400E08244903B0020AA880020CE
:105FF8008C2B0020805E0020003D0020FC3C00200F
:10600800E4300020DC430020145E0020A859002062
:10601800686C0020BD4B03F1700522681978501C8C
:106028002060117022685978501C20601170226815
:106038009978501C206011702268D978501C206013
:10604800117022681979501C2060117022685979E2
:10605800501C20601170226899790733501CAB429C
:1060680020601170D9D1FFF71FBAA9482BF058F951
:1060780000287FF719AAA64B1D18226813F8011BE0
:10608800501CAB4220601170F7D1FFF70DBAA14D3B
:10609800A14F05F1500600212878A04A0B4607E0D9
:1060A8000133242B02F10C0201F0EC8012F80C1CD5
:1060B8008842F5D103EB4303226807EB8303511CA5
:1060C80093F864302160137023686A78591C216042
:1060D8001A702368AA78591C21601A702368EA7814
:1060E8000435591CB54221601A70D4D1FFF7DCB9C8
:1060F8008B4B8C49B3F9003081FB0321DB17C3EBD1
:10610800A10189B22046FEF71FF901231A46FFF7BD
:10611800CDB9854D2046A989FEF716F9698920462B
:10612800FEF712F901231A46FFF7C0B97F4D204642
:106138002988FEF709F9A9882046FEF705F9298973
:106148002046FEF701F901231A46FFF7AFB90DF112
:10615800140900220592DFF800A2754B03920492FD
:10616800C9F80420904601214FF6FF7B07E008F1AB
:106178000108B8F10B0F01F0A6801AF9011F4E1C97
:10618800F5D04BFA08F2D007F1D51A8842FA08F28E
:10619800D207ECD548460193FBF750F9019BE6E797
:1061A800644E338AB3F5007F06F1340594BF0127A6
:1061B8000427403655F8041B91FBF7F1204689B2B5
:1061C800FEF7C2F8B542F5D15B4D5C4F05F10C0600
:1061D800B5EC010AD7ED087A80EE270A2CF0ECFB23
:1061E80081B22046FEF7B0F8B542F1D1544D05F121
:1061F8000C0655F8041B204689B2FEF7A5F8AE42F6
:10620800F7D1FFF751B92368474A4E49D078444A35
:106218005D1C2560187023680978581C2060197067
:106228002168D078FFF71ABB474D20462988FEF72A
:106238008BF869882046FEF787F8B5F904303949A4
:10624800DA1781FB0313C2EBA30399B22046FEF7CA
:106258007BF801231A46FFF729B95A1CC8F8002011
:106268001A780A2A0FD19A1CC8F80020374A597898
:106278001170D91CC8F8001099785170191DC8F808
:106288000010DB7893704FF0FF331A46FFF70EB912
:106298005A1CC8F800201D78FF2D01F0E581FE2D5D
:1062A80001F07C814046FEF713F8D8F80030D8F8A2
:1062B8000420D21A002A07DD5A1CC8F800201B78CF
:1062C80013B90B2D41F2FA81242DDCD8204A4FF066
:1062D800FF3322F815001A46FFF7E8B85A1CC8F829
:1062E80000201B780A2B01F04B81502BCBD1404664
:1062F800FDF7EEFF174D28804046FDF7E9FF4FF008
:10630800FF3368801A46FFF7D1B800BF448B0020DE
:106318006C3E0020902B0020444E0308AC4E03082E
:10632800F82B00206766666618290020D4670020CD
:10633800283E0020083B00204C4C0020244400202C
:106348004C3B0020082C0020603E0020DF8D002000
:10635800709300207C600020944E03081A46591C54
:10636800C8F800102E4D12F8021B6970C8F80020FA
:106378005A782A70DA1CC8F800209B78AB7040461F
:10638800FDF7A6FFD8F80030E8801A46591CC8F86F
:10639800001012F8021B2971C8F800205B786B7195
:1063A8004FF0FF331A46FFF781B85A1CC8F800208F
:1063B8001878721E0328D2B23FF665AF411EC9B2E3
:1063C800184D194B01EB410105EB41011870497853
:1063D80000283FF458AF8A427FF455AF0021C3F834
:1063E8000610C3F8021099726AB10132D8F8001089
:1063F8001A4401330131C8F8001011F8010C03F8F0
:10640800010F9A42F6D1094B1B78002B3FF43BAFA2
:106418001CF036FC4FF0FF331A46FFF747B800BFB1
:10642800DC9300207C6B0308E0400020FC67002020
:10643800A5F10B00EF283FF626AF01A252F820F095
:10644800656E00088F6200088F6200088F6200087E
:106458008F6200088F6200088F6200088F62000850
:106468008F6200088F6200088F6200088F62000840
:106478008F6200088F6200088F6200088F62000830
:106488008F6200088F6200088F6200088F62000820
:106498008F6200088F6200088F6200088F62000810
:1064A800F76D00088F620008DD6D00088F62000834
:1064B800BB6D00088F6200088F6200088F620008B9
:1064C800A76D00088F620008F16C00088F62000851
:1064D800B96C00088F620008916C00088F62000890
:1064E8007D6C00088F6200081B6C00088F62000832
:1064F800D16B00088F6200088F6200088F62000865
:106508008F620008B15400088F620008B16B000860
:106518008F6200088F620008956B00088F62000880
:106528008F6200088F6200088F6200088F6200087F
:106538008F6200088F6200088F6200088F6200086F
:106548008F620008FF6A00088F620008B16A0008BD
:106558008F6200088F6200087D6A00088F62000859
:106568008F6200088F6200088F6200088F6200083F
:106578008F6200088F620008817100088F6200082E
:10658800CF7000088F620008897000088F620008C9
:10659800297000088F620008FB6F00088F620008EE
:1065A8008F6200088F6200088F6200088F620008FF
:1065B8008F6200088F6200088F6200088F620008EF
:1065C8008F6200088F6200088F6200088F620008DF
:1065D8008F6200088F6200088F6200088F620008CF
:1065E8008F6200088F6200088F6200088F620008BF
:1065F8008F6200088F6200088F6200088F620008AF
:106608008F6200088F6200088F6200088F6200089E
:106618008F6200088F6200088F6200088F6200088E
:106628008F6200088F6200088F6200088F6200087E
:106638008F6200088F6200088F6200088F6200086E
:106648008F6200088F6200088F6200088F6200085E
:106658008F6200088F6200088F6200088F6200084E
:106668008F6200088F6200088F6200088F6200083E
:106678008F6200088F6200088F6200088F6200082E
:106688008F6200088F6200088F6200088F6200081E
:106698008F6200088F6200088F6200088F6200080E
:1066A8008F6200088F6200088F6200088F620008FE
:1066B8008F6200088F6200088F6200088F620008EE
:1066C8008F6200088F6200088F6200088F620008DE
:1066D8008F6200088F6200088F6200088F620008CE
:1066E8008F6200088F6200088F6200088F620008BE
:1066F8008F6200088F6200088F6200088F620008AE
:106708008F6200088F6200088F6200088F6200089D
:106718008F6200088F6200088F6200088F6200088D
:106728008F6200088F6200088F6200088F6200087D
:106738008F620008A16F00088F620008636F00086D
:106748008F620008D56E000873720008577200083F
:106758008F620008636A00088F620008396A0008BF
:10676800276A0008C76900088F6200089F69000847
:106778008F6200088F6200087D6900084969000877
:106788003569000807690008E1680008BF68000863
:106798008F620008A76800088F6200088F620008EF
:1067A8008F6200088F6200088F6200088F620008FD
:1067B8008F6200088F6200088F6200088F620008ED
:1067C8008F6200088F6200088F6200088F620008DD
:1067D8008D6800088F6200088F620008236800082F
:1067E8008F6200088F6200088F6200088F620008BD
:1067F8008F6200088F6200088F620008096800082D
:10680800D04B1B78DB073FF53EADFDF713FCFDF7DA
:1068180067F901231A46FEF749BE5A1CC8F800203A
:106828001A780F2A3FF62FAD991CC8F80010C2EB52
:10683800C202C54958788854D81CC8F800000A44D0
:1068480099785170191DC8F80010D9789170591DA0
:10685800C8F800101979D170991DC8F80010597935
:106868001171D91DC8F800109979517103F1080107
:10687800C8F80010DB79937126F088FF01231A46C7
:10688800FEF714BE4046FDF723FDB04DA8814046F3
:10689800FDF71EFD012368811A46FEF707BE404634
:1068A800FDF716FDAA4900EB8000420001230A808B
:1068B8001A46FEF7FBBD4046FDF70AFDA54DA88226
:1068C8004046FDF705FDE8824046FDF701FD01233E
:1068D80028831A46FEF7EABD1A46591CC8F8001064
:1068E80012F8020BC8F80020DA1C5978C8F8002002
:1068F8009A781BF021FA00287EF4D6ADC3E41A4634
:10690800591CC8F80010944912F8020B0870C8F80E
:1069180000208E495A788A70DA1CC8F800208C4A00
:106928009B78937001231A46FEF7C0BD8B4B8C49A8
:1069380018684A222BF038FE01231A46FEF7B6BD26
:1069480019465A1CC8F80020864A11F8020B107024
:10695800C8F8001059785170D91CC8F800109B78F5
:1069680093704046FDF7B4FC7F4A0123D0801A4655
:10697800FEF79CBD4046FDF7ABFC7B4D28804046AA
:10698800FDF7A6FC68804046FDF7A2FC0123A8801D
:106998001A46FEF78BBD754F3B78002B3EF484AD4D
:1069A800734E00254046FDF793FC15F0FFFE3B783B
:1069B800A6EC010A01359D42F4DBFEF775BD0F2EEA
:1069C8007FF461AC5A1CC8F800201D78072D3FF6EB
:1069D8005AAC684F40460C26FDF77AFC06FB05F6D4
:1069E800BD19A8804046FDF773FCE8804046FDF7D6
:1069F8006FFCD8F8003028811A46591CC8F80010D6
:106A080012F8021BA972C8F800205B78EB724046A6
:106A18002BF059FB0123B8511A46FEF747BD4046F3
:106A2800FDF756FC544A012310801A46FEF73EBD76
:106A38005A1CC8F800201878060600F13486414B25
:106A48001B78DD073EF530AD032828BF0020FAF794
:106A580039FD01231A46FEF729BD3A4B1B78D807A2
:106A68003EF522ADFDF7DAFAFDF73AF801231A46AA
:106A7800FEF71CBD414A1278012A3EF615AD1946AB
:106A88005A1CC8F800203E4A11F8020B9070C8F84A
:106A9800001059781170D91CC8F800109B785370F1
:106AA80001231A46FEF702BD5A1CC8F800201E78BA
:106AB800112E3FF6E8AB9A1CC8F80020314D5B78E0
:106AC80005F816304046FDF703FC40F6CA03984225
:106AD800A8BF184640F2EE23984205EB4605B8BF1A
:106AE80018460123A0F2EE211A46192091FBF0F175
:106AF8006970FEF7DBBC1A46591CC8F80010224D15
:106B080012F8021B2970C8F800205B786B704046A9
:106B1800FDF7DEFBD8F8003068805A1CC8F8002062
:106B28001B782B714046FDF7D3FBD8F80030E8807E
:106B38005A1CC8F800201B782B7201231A46FEF74E
:106B4800B5BC00BFEB3C0020448B00201829002076
:106B5800F82B00208059002010440020843E00209B
:106B680024550308941E0020DC3700207568002097
:106B7800E03600200C8D0020901E0020048F00209D
:106B8800E89300202C300020F4370020C14A03F19C
:106B980008010133C8F8003013F8010C02F8010F9E
:106BA8009942F6D1FEF780BC1A46591CC8F8001065
:106BB800B94912F8020B8870C8F800205B784B704E
:106BC80001231A46FEF772BC0722B6FBF2F2C2EBAB
:106BD800C201711A7FF457ABD2B2571EFFB2002A16
:106BE8003EF462ACDFF8B49201378A465A1CC8F802
:106BF800002093F90010A94B002593F902208A423E
:106C080000F0E0840135062D03F10803F5D1FFF704
:106C18003ABB5A1CC8F800201A780E2A3FF633AB44
:106C2800991CC8F800105D78032D3FF62CAB9C48E2
:106C3800062101FB02F14218DE1C5571C8F80060FC
:106C48009D784554191DC8F80010D9785170591D00
:106C5800C8F8001019799170991DC8F80010597971
:106C6800D170D91DC8F800109B79137101231A46F9
:106C7800FEF71CBC5A1CC8F800208A4A1B785375BA
:106C880001231A46FEF712BC5A1CC8F800201D78CA
:106C98001F2D3FF6F8AA052E7FF4F5AA40462BF0E3
:106CA80012FA814B43F8250017F084F9FEF7FCBB74
:106CB8007D4D05F140064046FDF70AFBD8F8003047
:106CC800A5F88000591C1A46C8F8001012F8021BD3
:106CD80085F88210C8F800205B7885F88330043581
:106CE800AE42E8D1FEF7E0BB5A1CC8F800206D4D53
:106CF8001B782B724046FDF7EBFAA8834046FDF758
:106D0800E7FA28834046FDF7E3FAD8F800306883AD
:106D18005A1CC8F800201B78EB74082E7EF6C4AB0A
:106D28004046FDF7D5FAE8844046FDF7D1FA0C2E27
:106D380028857EF6B9ABD8F800301A46591CC8F831
:106D4800001012F8021BA977C8F800205B7885F8B4
:106D580020304046FDF7BCFA102EA8847EF6A4AB7E
:106D6800D8F800305A1CC8F800201B78EB7240464F
:106D78002BF0A9F9D8F80030E8605A1CC8F80020B0
:106D88001A782A74162E7EF68FAB9A1CC8F8002043
:106D98005B7885F8213001231A46FEF787BB5A1C19
:106DA800C8F80020414A1B78137001231A46FEF7E1
:106DB8007DBB4046FDF78CFA3D4D28604046FDF707
:106DC80087FA68604046FDF783FA0123A8601A46EF
:106DD800FEF76CBB374D00232B6040462BF073F950
:106DE8002A68012302432A601A46FEF75FBB5A1C31
:106DF800C8F80020187813283FF645AA9A1CC8F846
:106E080000205D782C4A002105E00131242902F197
:106E18000C023FF438AA167AAE42F6D1274D284A1A
:106E28000C2606FB0151DD1C91F85C1002F82010BD
:106E3800C8F8005002EB800299785170191DC8F803
:106E48000010D8789070581DC8F800001D491B79AB
:106E58000868D3702BF054F9FEF726BB1A4B102E96
:106E68004FF0000228BF10261A605A609A60DA6054
:106E78001A74002E3EF418ABD8F8002016440132DC
:106E8800C8F8002012F8011C03F8011BB242F6D121
:106E9800FEF70ABB7F5E0020241F0020DC43002091
:106EA800E4300020805E0020003D00208C2B002074
:106EB800D4670020008F0020A04E0308444E03082A
:106EC800902B0020843E00206C3E0020092E7FF687
:106ED800DAA99E4F1A46591C3D68C8F8001012F8E6
:106EE800021B2970C8F800205A78AA70DA1CC8F862
:106EF80000209A78642A03F10401A8BF64226A7109
:106F0800C8F80010DA78642A03F10501A8BF6422E2
:106F1800AA71C8F800101A79EA719A1DC8F80020F9
:106F28005A79642A28BF6422D91D2A72C8F8001029
:106F38009A79EA7003F10802C8F80020DB792B710E
:106F48004046FDF7C5F90A2E688140F0C3830DF06D
:106F58003BFE01231A46FEF7A9BA7D4A1068DA1CDF
:106F680001462133951EC8F8005012F8035C0D70D5
:106F7800551EC8F8005012F8025C4D70C8F8002081
:106F880012F8015C8D7003329A4201F10301E9D1D4
:106F980026F0D4FDFEF788BAC6F34706122E3FF650
:106FA80072A9B6B10EAB0DF1120703EB4605B9464F
:106FB800263D4046FDF78CF929F8020F4D45F8D1DA
:106FC800644B37F8022F23F8022F4F45F9D1112EC1
:106FD80009D8614A7300023B13440021223223F886
:106FE800021F9A42FBD15D49012213460A70FEF73F
:106FF8005DBA1A46591CC8F80010594912F8020B14
:10700800C870C8F8002057495A780A70DA1CC8F8BE
:107018000020554A9B78D37001231A46FEF746BADA
:107028004046FDF755F94046FDF752F94046FDF751
:107038004FF9D8F80030464D9A1C2F68C8F8002040
:107048005A7887F82F20DA1CC8F800209A7887F831
:107058003A201A1DC8F80020DA7887F83B20073351
:10706800C8F800304046FDF733F9F88740462F68E6
:10707800FDF72EF9112EB88700F23D83286887E7BF
:107088005A1CC8F80020324D384F1B78D5F80090AC
:107098007B714046FDF71CF9A9F820004046D5F859
:1070A8000090FDF715F9052EA9F8220000F23483A7
:1070B800FAF724FA1BF07EFE286815F0ABF90123D5
:1070C8001A46FEF7F3B91A46591CC8F80010274E9D
:1070D80012F8021BB170C8F8002025495A780A70C6
:1070E800DA1CC8F80020234D9A782A711A1DC8F8AE
:1070F8000020DB78092BA8BF09234046AB70FDF7B9
:10710800E7F8D8F80030D8F804202880D11A0129E7
:1071180007DD4046FDF7DCF8D8F80030D8F8042041
:1071280068829A4240F01A83FAF7E8F9D8F80030F2
:10713800D8F804209A423EF4B7A95A1CC8F800208F
:107148001B78EB7001231A46FEF7B0B978260020A9
:10715800843E00200E2E0020102E0020342E002009
:1071680018290020082C0020F82B002010440020AB
:10717800308C0020805900204046FDF7A9F80546CC
:1071880017F0CAF9FF283EF48FA9B5F57A7F80F089
:1071980054820DF13809002309F8243DEE084946C8
:1071A80003A88DF80C30013617F096F99DF80C30CD
:1071B800F6B205F00705B34205F1010503D19DF8C4
:1071C8001430AB4203D02946304617F091F9D8F86D
:1071D8000030D8F80420D21A012A7EF765A95A1C73
:1071E8000EA8C8F8002000221D7800F82C2D17F0F2
:1071F80067F99DF80C30AB420AD0C44B1B683BB111
:107208009A79AA4204D31B681B690BB12846984790
:10721800D8F800305A1CC8F80020484600221D78CB
:107228008DF8142017F040F99DF81430AB423EF465
:107238003BA9B64B1B68002B3EF436A91B685B695B
:10724800002B3EF431A928469847FEF72DB9B04BDC
:107258001B78DA073EF528A9AE490A78012342F0DF
:1072680004020A701A46FEF721B9A94B1B78D90700
:107278003EF51AA9A84A4FF4C871012311801A468D
:10728800FEF714B900231B7AFFDE23685A1C22601C
:10729800197029882046FDF757F82368EA78591CA1
:1072A80021601A7023682A79591C21601A70236892
:1072B800AA79591C21601A7023686A79591C2160BF
:1072C8001A70FEF771BEDFF884B24FF000084FF075
:1072D800080A08F10108B8F1240F1BD0C8F12002F0
:1072E8000AFA02F22BFA08F6A8F1200316432AFA42
:1072F80003F31E4306F0010200231343E9D05FFAAB
:1073080088F00DF00FFC0028E3D041464846FAF714
:1073180095F8DEE77E4B1B78DF0700F12181002618
:107328007E4FB04602E00136242E0ED03146384654
:10733800FDF73EFA0028F6D031464846FDF738FA00
:10734800002856D108F10108EDE7754B754EB3F8E2
:1073580050102046FCF7F8FF734B1988204689B275
:10736800FCF7F2FF714B1A68530103F02001C2F3D6
:1073780040030B43C2F3800143EA4103C2F3C00157
:1073880043EA8103C2F3401143EAC10102F010024B
:1073980011432046FCF7D8FF03A904222046FCF736
:1073A800A3FF23683178624A581C2060197011883D
:1073B8006429A8BF64212046FCF7C6FF962D00F07B
:1073C800D48000212046FCF7BFFF2168B8F11903DB
:1073D80048BFA8F11203A3F3C4034A1C2260204645
:1073E8001A460B7004A9FCF77FFF01231A46FEF723
:1073F8005DB8414603A8FAF721F8A3E72368B178F6
:107408004C4A581C2060197023681278591C216056
:107418001A70FEF7C1BAD9F8003013F48053B4EEED
:10742800E88A00F0B380F1EE10FAC0F2FA80B4EE08
:10743800C98AF1EE10FA0DD8DFED3F7A9FED3F7A59
:1074480077EEC87AB4EEC78AF1EE10FAB0EE678A22
:1074580000F2E780F7EE007A78EE677AB6EE007A07
:10746800F0EE696AE7EE876A40F2E932FDEEE67A05
:1074780017EE901AB1F5FA6FA8BF4FF4FA6191426E
:10748800B8BF114689B2002B3EF4C2ACB5EE408AB3
:10749800F1EE10FA40F2DC5308BF1946FEF7B8BC0B
:1074A80095F82420264B002A40F0B2803046FEF79B
:1074B80033BA5A1C1946C8F80020184811F8022B8C
:1074C8000272C8F800105B784372042A06D9FF2AB2
:1074D8003EF455A921680020FEF7C0B9194909787A
:1074E800994203D8022AF5D1FF2BF3D12268012350
:1074F800D11821601370B9F1000F3DF4D5AF124ACD
:10750800C9F800201A46FDF7D1BF00BF803E002011
:10751800EB3C0020D893002096260020841E0020F3
:1075280094090020683E0020106B0020D4510020F0
:10753800BE270020308C002000C0884400C0824450
:10754800E074002075680020C10F000890E33FF444
:1075580021680123CA1822601A460870FDF7A6BFE1
:10756800059B43F001030593D9E623680322591CC0
:1075780021601A7023687278591C21601A7024E7F8
:107588004046FCF7A5FE7A4DFEF7B5BEF1EE10FABF
:10759800BFF660AF4FF47A71FEF73ABC9A1CC8F890
:1075A80000205D78022D3EF66EAE4046FCF790FE58
:1075B800704A02EB45024FF0FF33A2F85E001A460C
:1075C800FDF774BF09EBC5064046B170FCF780FEB5
:1075D800D8F8002029F835001346511CC8F80010C7
:1075E80013F8021BF170C8F8003053783371D31CBC
:1075F800C8F800309378B371131DC8F800300AF149
:10760800010AD278727157457FF4F0AAFDF74CBF92
:107618005978022908D003290CBF04203046FEF708
:107628007BB94FF47A7131E7042A34BF0220032072
:10763800FEF772B94246FEF7E7B80DF1140948465D
:1076480016F026FFBDF81430AB423FF4C0AD4A4BEC
:107658001B68002B3FF4BBAD1B689B69002B3FF4F4
:10766800B6AD28469847B2E5DA1CC8F80020414D67
:107678009A7885F85C201A1DC8F80020DB7885F810
:1076880056304046FCF724FEA5F858004046FCF763
:107698001FFE4046FCF71CFE4FF0FF33A5F85A00CA
:1076A8001A46FDF703BF00F07F00032828BF00201B
:1076B80013F0CAFF01231A46FDF7F8BE2D4B003020
:1076C8001D4418BF01204FF0FF3385F84A001A46C1
:1076D800FDF7ECBED8F800303A68591CC8F800101D
:1076E800197851720B2E3FF432AC991CC8F800106F
:1076F8005B7853702BE4D8F800302968581C1A4678
:10770800C8F8000012F8020B81F83100C8F8002010
:107718005B7881F83230B1E44046FCF7D9FD7881D6
:107728004046FCF7D5FDB8814046D5F80090FCF7F7
:10773800CFFDA9F824004046D5F80090FCF7C8FD15
:107748000D2EA9F826007FF6B3AC4046FCF7C0FD25
:10775800F8814046FCF7BCFD3882A9E45A1CC8F8F9
:1077680000201B78003318BF0123F371DCE400BF4D
:10777800201F002070930020803E00202DE9F04F4C
:107788002DED028BC54B1B7891B0072B059001F0AE
:107798007D8200230793C24BD3F800B01BF4806F9F
:1077A80040F05486BF4B1B6806931C0700F1F88510
:1077B800BD4BBE4DB3F80090BD4CBE4BBE491F68D3
:1077C800B1F906807A89904580F29184BB4B4FF0DD
:1077D8007E521A60DFF8F8A294F90820B1F900C0C7
:1077E800BAF81860207994F805E0002AACEB060393
:1077F80014BF01224FF0FF32002B40F3E384B3F5AE
:10780800FA7FC0F2E5844FF4FA731B1A07EE903A38
:10781800F8EEE77AB445C5ED007A03DAF1EE677A57
:10782800C5ED007AB1F902C0ACEB0603002B40F3BA
:10783800D684B3F5FA7FC0F2D8844FF4FA731B1AD2
:1078480007EE903AF8EEE77AB445C5ED017A03DA27
:10785800F1EE677AC5ED017AB1F90430991B002978
:10786800D8BFF11AB1F5FA7F80F23B847145D8BFD1
:107878004FF0000E00F3378402FB0EF207EE902A59
:10788800F8EEE77AB342C5ED027ABCBFF1EE677A4B
:10789800C5ED027A1BF48053049300F0E980B8F533
:1078A800FA6F4246A8BF4FF4FA62B2F57A7FB8BFC2
:1078B8004FF47A72A2F57A728149DFF818E281FBF7
:1078C8000230D317C3EB6013581C6FF0630C3EF9FA
:1078D80010003EF913E00CFB0323A0EB0E0003FBA2
:1078E80000F381FB0321DB17C3EB61139E440FFAFE
:1078F8008EFE07EE90EA049BB8EEE78A85ED038AD0
:10790800002B40F0B08519F04003089340F0B9848B
:10791800069B13F0140F03D019F4027F40F02A8657
:10792800684B1B7823B1BAF81A30434580F29A8421
:1079380094F82E601EB119F0030F40F0598794F89F
:1079480034209AF81F30002A40F0BA859AF81E6051
:10795800002E00F0C380022E00F04487032E00F0B2
:107968002687594949880233DBB2002A00F02C8760
:10797800002900F0298755480668B1FBF6F10EB2D8
:10798800A4F86460ABB307EE906AF8EEE77AF7EE16
:10799800006A86EEA77A012BD5ED007AD4ED1E6A2F
:1079A80077EEE67A67EE877AC4ED1A7A21D0D5EDBC
:1079B800017AD4ED1F6A77EEE67A022B67EE877AB2
:1079C800C4ED1B7A15D0D5ED027AD4ED206A77EE96
:1079D800E67A032B67EE877AC4ED1C7A09D0D5EDD9
:1079E800037AD4ED216A77EEE67A67EE877AC4EDFA
:1079F8001D7A2A490978092901F00185002E72DDCE
:107A080093B394ED1E7AD4ED1A7A77EE877A012B28
:107A1800C4ED1E7AC5ED007A21D094ED1F7AD4ED1D
:107A28001B7A77EE877A022BC4ED1F7AC5ED017AAF
:107A380015D094ED207AD4ED1C7A77EE877A032B53
:107A4800C4ED207AC5ED027A09D0D4ED217A94EDFF
:107A58001D7A77EE877AC4ED217AC5ED037A013B6A
:107A6800022BB8BF0223DBB2002A18BF02233BE077
:107A7800BAF81A108845C0F2F383B8F5FA6FD4BF84
:107A8800C1EB0803C1F5FA634FF47A7202FB03F203
:107A9800C1F5FA61B2FBF1F20EE700BF856800207C
:107AA800686C0020D4510020283E00207469002012
:107AB800901E002078260020AC880020E0250020B9
:107AC8001F85EB512C000020903B0020742B0020D8
:107AD800805E00207C2600200AD7233CA4F864603E
:107AE800002A00F06F8102233A785FED056AB978C1
:107AF80007EE902AF8EEE77AB0EE007A67EEA67AFB
:107B0800D34AF4EEC77AF1EE10FA107840F34484C1
:107B1800DFEDD06A37EEC77AB0EE676AA7EE266A5D
:107B2800F0EE466A95ED007A9FEDCB6ADFF84CE3FC
:107B3800DFF84CC327EE066AF0EEC65ACEED005ABF
:107B48008CED006A99B107EE101AB8EEC75A9FED8E
:107B5800C37A66EE064A25EE075AB7EE007A37EE84
:107B6800457A64EEA54AA5EE247A26EE076A9FEDCB
:107B7800BC7A7A7926EE877A27EE067AAAB1DFED03
:107B8800B76A9FEDB86A65EEA65A06EE902AF8EE37
:107B9800E66A66EEA56AF4EEC66AF1EE10FA40F3FC
:107BA800D9859FEDB16A27EE067A0C289FEDAF8A3A
:107BB800DFEDAF6ADFF8CC8200F0A785B4EEC87AB3
:107BC800F1EE10FA98BFB0EE478AB4EEE68AF1EE0D
:107BD80010FAB8BFB0EE668A88ED008A002B00F074
:107BE800E680B0EE007AF4EEC77AF1EE10FA05DD21
:107BF80037EEC77ADFED976AE7EE267A95ED017AD8
:107C0800DFED956A27EE267AF0EEC75A8CED017AF9
:107C1800CEED015A99B106EE901A9FED906AF8EEF2
:107C2800E66A27EE075A66EE866AB7EE006A36EE0F
:107C3800666A25EE255AA6EE856A27EE067ADFEDF6
:107C4800886ABA7967EEA67A67EE877AFAB107EE9C
:107C5800102AB8EEC77A9FED816ADFED826A27EEB7
:107C6800257A27EE067AB4EEE67AF1EE10FA00F3FA
:107C78006D85B5EEC07AF1EE10FA01F16380B7EECA
:107C8800006A36EE477AC6EE076A67EEA67A0C28CF
:107C980000F01C85DFED756A9FED757AF4EEE67AE3
:107CA800F1EE10FA88BFF0EE667AF4EEC77AF1EEDC
:107CB80010FAB8BFF0EE477A012BC8ED017A76DDED
:107CC8007B78DFED666A07EE903AF8EEE77AB0EE79
:107CD800007A67EEA67A7B7AF4EEC77AF1EE10FAAC
:107CE80005DD37EEC77ADFED5B6AE7EE267A95EDBC
:107CF800027ADFED596A27EE267AF0EEC75A8CED44
:107D0800027ACEED025A9BB106EE903A9FED536A85
:107D1800F8EEE66A27EE075A66EE866AB7EE006A5C
:107D280036EE666A25EE255AA6EE856A27EE067AAD
:107D3800DFED4B6AFB7967EEA67A67EE877AFBB1CF
:107D480007EE103AB8EEC77A9FED446ADFED456A50
:107D580027EE257A27EE067AB4EEE67AF1EE10FAE7
:107D680000F3F084B5EEC07AF1EE10FA00F1E68780
:107D7800B7EE006A36EE477AC6EE076A67EEA67A6D
:107D88000C2800F09B84DFED396A9FED397AF4EE18
:107D9800E67AF1EE10FA88BFF0EE667AF4EEC77A6A
:107DA800F1EE10FAB8BFF0EE477AC8ED027A09286A
:107DB80000F07B849AF82150002D40F03184002394
:107DC80084F834302B4D2C4F95F82420DFF8B880F8
:107DD800531E082B00F20381DFE813F01F019D01F9
:107DE800A500010158000900B20101019F0198F89E
:107DF8000030002B40F0B6842B68297A4FF480724B
:107E080003EB0121002022F02BFE2B7A0133DBB299
:107E1800022B2B7240F05481002022F063FE0020D8
:107E280022F060FEFF2022F05DFE00F01F00052812
:107E380001F06A831FF00EFBEE68002E00F09783B6
:107E480000222B6969680120B04795F82420BFE714
:107E580085680020D7A368416F12033B0AD7233CEB
:107E680000004843A4707D3F0000C84200C0F944A8
:107E780000C0F9C408870020B86A00200C2600203A
:107E880000260020E82500202A6800204FF4007111
:107E980028681FF091FA012800F0DF84C0F0D88527
:107EA800022840F00D811FF0FDFA1FF0D3FAEE68AA
:107EB800002E00F05C83002210462B696968B047E9
:107EC80095F8242084E71021D3481FF075FA8346DB
:107ED800002840F0F38001217F2024F053FD012881
:107EE800814640F0EB805846022124F04BFD0028E3
:107EF80001F0AE81012840F0E18016213A2024F0FB
:107F080041FD431C9B02EB631FF0CCFA3068FBF782
:107F1800F7F800210A201FF06DFA002840F0D886F3
:107F2800032385F8243010210CA81FF045FA0028F7
:107F380040F0C6809DF83A209DF839009DF83C1025
:107F48009DF83D309DF83B60120442EA00620A4306
:107F58001B019DF83E109DF83100DBB243EA111376
:107F680042EA062203F5FA636A632B879DF83220FA
:107F78009DF8383042EA002201F00F01180903F099
:107F88000F0385F83A106A859DF830109DF8332064
:107F980085F832309DF8343085F8281085F82C2083
:107FA8009DF835109DF8362085F82D309DF837302E
:107FB80085F8303085F8310085F82E1085F82F20A7
:107FC8001FF070FAAB7E002B00F01681934822F068
:107FD80005FE002304222B6285F824200323DBB24C
:107FE800022B73D9042A00F0C780082A00F0C48045
:107FF8008B4B1B7823B98B4EB278002A40F03C8516
:1080080005981BF057F9884B1B78072B00F07C84E8
:1080180011B0BDEC028BBDE8F08F844E3068FBF7E1
:108028006FF8002108461FF0E5F981461FF03AFA7B
:10803800B9F1010F44D130684FF0000B85F819B041
:10804800FBF75EF840F2AB1108201FF0D3F90528C2
:1080580000F00F84012800F01E861FF023FA6B7EC3
:10806800002B01F04D82022385F824303068FBF79D
:1080780047F86B7E022B14BF4FF000094FF0804980
:10808800002137201FF0B6F9494629201FF0B2F920
:1080980081461FF007FAB9F1000F11D16B7E022B50
:1080A80000F0068685F81A903068FBF729F8002159
:1080B80009201FF09FF900283FF405AF1FF0F2F9DF
:1080C80095F82420531EDBB2022B8BD8584B6969D4
:1080D8001B685B1AC82B88D91FF0BCF995F82420B7
:1080E80080E74FF4FA71A1EB0E0EFFF7C5BBB8F5A8
:1080F800FA6FC0F2A9803B7AC3F1640307EE903AA5
:108108009FED4C7A4C4BF8EEE77A67EE877AC3ED31
:10811800007AFFF75FBB454EA8E70826FF2022F04C
:10812800E1FCFF2800F0FB83013EF7D16B693A6858
:10813800FA339342C4D21FF08DF995F8242047E60C
:10814800FF2022F0CFFCFF284FF0080606D0013EA2
:10815800ECD0FF2022F0C6FCFF28F8D12B6A0022C1
:10816800012B2A7641F27B84EA69013B01322B62BA
:108178000823EA6185F82430304D1FF047FD6B78FD
:10818800022B00F0D883032B7FF432AF41F2B813EF
:10819800EB5C002B41F07D8041F2A403EB5C002BEB
:1081A80041F0728041F2E803EB5C002B41F07680ED
:1081B80041F22C13EB5C002B3FF41AAF204820F05F
:1081C80011FB15E7A6EB0C03B3F5FA7FBFF61BAB63
:1081D8009842FFF61AABDFED1B7AFFF71BBBA6EB45
:1081E8000C03B3F5FA7FBFF628AB9842FFF627AB2E
:1081F800DFED147AFFF728BB0C4E3068FAF780FFE2
:108208004FF4007110201FF0F5F806461FF04AF9E8
:10821800002E3FF4DBAE8EE7488700200038004090
:10822800DE3A0020E8930020856800202C680020B2
:10823800B86A00200AD7233CE0250020E07400201B
:108248000C86002000000000387AA8EB020303FB2C
:1082580000F3C2F5FA6293FBF2F3C3F164034DE74E
:108268001A4615E4D14B1B78012B00F04283192BD9
:1082780000F03F830E2B3FF45BAB082B3FF458AB69
:108288003CE3CB4BCB49B3F904306289DFEDCA6AD2
:108298009FEDCA7A81FB0301DB17C3EBA1039B1A8D
:1082A8001BB207EE903AF8EEE77A67EEA67A77EE19
:1082B800876ABDEEE66A16EE103A2033402B40F28C
:1082C8004D83DFEDBF6ABDEEE77A17EE103A203333
:1082D800402B00F240839FEDBB7AF4EEC77AF1EEB3
:1082E80010FA40F3EF87DFEDB85A9FEDB86A01E066
:1082F800F0EE477AF4EEC67AF1EE10FA37EEE57A48
:10830800F6DCDFEDB37AB4EEE77AF1EE10FA40F17D
:10831800DD87DFEDAD5A9FEDAF6A01E0B0EE677A19
:10832800B4EEC67AF1EE10FA77EE257AF6D49FED20
:10833800A37AF4EEC77AF1EE10FA00F395829FED76
:10834800A67AF4EEC77AF1EE10FA44BF9FEDA07A50
:1083580077EE677A67EEA75A9FEDA05A9FEDA06A5D
:108368009FEDA07AA5EE856A27EEA55AA5EE867A36
:10837800E5EE077A95ED016AD5ED005A27EEC67A43
:1083880065EEA77AA5EEA67AE6EE267A85ED007A5E
:10839800C5ED017AFFF7BCBAF0EE676AFFF7C2BB1A
:1083A800914D924BD5ED027AB3F80090804B814AFB
:1083B800B3F904308E4CB2EE0E7AF0EEE76AF4EEC2
:1083C800C76AF1EE10FA82FB03124FEAE37338D55D
:1083D80019F0040F35D02188C3EBA2035B1A9BB2B6
:1083E8001AB212F1B30FBCBF03F5B4731AB2B32AB1
:1083F800C8BFA2F5B4737F49C8BF1AB2237A0978F7
:10840800002B4FF6FF7318BF012308077FF5D5A986
:108418007949096812FB03F30A7E78499BB212FB7B
:1084280003F381FB03121A44DB17C3EB221307EE95
:10843800103AB8EEC77A77EEC77AC5ED027AFFF739
:10844800BCB9C3EBA2032380FFF7B7B96C488368B4
:10845800002B3FF4A7A900F144019847694BD3F8D2
:1084680000B0FFF79FB91D216748FCF7A1F9002864
:108478003FF449AA654BDB78002B7FF444AADFED73
:10848800647A644938EE678AC6F5FA63FDEEC87AFD
:108498001BB2CDED087ABDF92020120381FB020141
:1084A800D217C2EBA11203FB02F343F30F33334499
:1084B80007EE903AF8EEE77AC5ED037AFFF723BAAC
:1084C80055485149D0F8EC00096844F62066B04296
:1084D800A8BF3046B0F57A7FB8BF4FF47A7080B243
:1084E800C906E08640F1C9810499002900F02E846C
:1084F8004149D1F800C0BCF836E04FEA5E0E454E5F
:10850800A16BD5ED037AA6FB00608609642090FB79
:10851800F6F01428BDEEE77A04EB4108A8BF142052
:1085280001318142A16317EE109AA4BF0021A16313
:1085380004EB4101A8F83C90B1F93C1007EE101A81
:10854800B8EEC77A77EEC77AFDEEE77ACDED047A12
:10855800BDF9100080EAE071A1EBE071714500F30C
:10856800A2862E494FF07E500860FFF7EFB995F8C4
:1085780024202DE41F4B1B7813F0100300F08D818D
:10858800227B236995ED017A002A0CBF01224FF066
:10859800FF3203FB02F307EE903AF8EEE77A77EE44
:1085A800877AC5ED017AFFF7BBB900BF8C2B002095
:1085B800603E00206766666635FA8E3CDB0FC93F71
:1085C80000000000DB0F4940DB0FC940E4CB164137
:1085D800DB0F49C0E4CB16C1DB0FC9BF92E741B935
:1085E8009730083C15A82ABE74690020283E002050
:1085F800901E0020D8930020843E00208988888817
:1086080024440020686C00201C940020303E002088
:1086180000007A44D34D62109409002028000020FD
:108628001E21D448FCF7C4F800283FF4C8AB089BC7
:10863800002B7FF4C4AB94F88830AB4240F07086CE
:10864800CD4BD4ED237AD3ED006A98ED025ADFEDD5
:10865800CB5A9FEDCB6A27EEC57A68EE277AA8EE4B
:10866800267AE5EE267AB4EEE57AF1EE10FA88BFBE
:10867800B0EE657AB4EEC67AF1EE10FAF4EEE57A69
:10868800B8BFB0EE467AF1EE10FA88BFF0EE657A20
:10869800F4EEC67AF1EE10FAB8BFF0EE467A88ED3D
:1086A800007AC8ED027AFFF78ABBFDEEC87AB54AB0
:1086B80017EE903A9680D380FFF77CBBBDEEE77A41
:1086C800B04B17EE102A9A80FFF75DBB9FEDAB7A8F
:1086D800DFEDAB6AAB49F4EEC77AF1EE10FA98BF5A
:1086E800B0EE677AFDEEE77AB4EEE67AF1EE10FACC
:1086F80017EE902AB8BFB0EE667A012B88ED017AA2
:108708004A803FF7DDAAFFF755BBB4EEC87AF1EE11
:1087180010FA98BFB0EE478ABDEEC77AB4EEE68A83
:10872800DFF86092F1EE10FA17EE102AB8BFB0EE3B
:10873800668A88ED008AA9F80020002B7FF451AAE8
:10874800FFF738BBDFED906AFFF718BBDFED8E6AE5
:10875800FFF79BBAF7EE005A75EEE66A85EEA66A51
:10876800FFF721BA894B19688E037FF53EAC4FF4A9
:1087780000325A60864B1A68864B4FF6FE710A40E3
:1087880083490A601A89D2077DD41AF06BFA002847
:10879800FBD1804A938823F002031B041B0C9380AF
:1087A80098F80030002B7FF437ABFFF725BB9AF819
:1087B8002010C1EB411001EB8001C900023389B2DE
:1087C800DBB2002A7FF4D4A8B4F86460013E36B264
:1087D800002EA4F864603FF713A9002A7FF483A948
:1087E800FFF7F0BAE18E01F57A7189B2FFF7BBB8ED
:1087F800694BDFED6A7A93ED080AB4EEE70AF1EE09
:1088080010FA40F282822AF06DF9D4ED0C7A20EE4B
:10881800270A2AF0D1F8B0F5617F00F39E8207EEAF
:10882800900AF8EEE76ADFED5E7A66EEA76A07EE71
:10883800906AB8EEE77AFDEEE67A17EE903A2033C2
:10884800402B40F2B9869FED570A2AF0B5F800B2DE
:1088580007EE900AB8EEE77A59E26B693A68643332
:108868009342FFF420AB2BE49FED577A77EE677ABB
:1088780070E585F81990FFF7F0BB1BF0805F7FF477
:1088880033AEFFF763B89A891A89D007FBD41AF078
:10889800E9F900287FF479AF7BE7E279002A40F014
:1088A8009782B4F91460A179A8EB060383EAE37010
:1088B800A0EBE370884240F3278503EBD3730122D2
:1088C8005B10636284F82820227723691E44B6F57A
:1088D800FA6FA8BF4FF4FA66B6F57A7FB8BF4FF4BF
:1088E8007A7607EE906AF8EEE77AC5ED037AFFF735
:1088F80017B82D4B9B7B002B7FF41AA82B4A00231B
:10890800AB609360FFF714B8F9F726FF079A1D4B81
:10891800801A988011B0BDEC028BBDE8F08F1EF074
:10892800C1FD042385F82430214D1FF06FF96B78C1
:10893800022B7FF428ACAB784FF0010B072B3FF6E6
:1089480057ABDFE813F0480461043C043104C30367
:108958008D0397035B03DFED137A0BE5F4EEC77A1B
:10896800F1EE10FA40F3C485DFED145A9FED116A59
:1089780034E000BF1C9400202000002000C0F9440F
:1089880000C0F9C4886800200000C8420000024006
:1089980058000240003800406C3000208FC2753CFF
:1089A800D06D393A0000000080570020E8250020EB
:1089B800E0740020E4CB1641DB0F49C0DB0FC9404F
:1089C800E4CB16C1DB0FC93FDB0F494092E741B941
:1089D8009730083C15A82ABEF0EE476AF4EEC66A3E
:1089E800F1EE10FA36EEE57AF6DC5FED0D6AB4EEDC
:1089F800E67AF1EE10FA40F177855FED105A1FED37
:108A0800106A01E0B0EE667AB4EEC67AF1EE10FABA
:108A180077EE256AF6D41FED157AF4EEC76AF1EE03
:108A280010FA40F366811FED187A77EE666A66EEF3
:108A3800A65A1FED1A5A1FED1A6A1FED1A7AA5EEEB
:108A4800856A26EEA55AA5EE867AE5EE076A3AE427
:108A58001EF028FDEE680423002085F824302876CF
:108A6800002E3FF489AB2B692A686968B04795F8EE
:108A78002420531EFFF727BBC44F3B78013B0A2B2A
:108A880059D8DFE813F015020702FB013902580034
:108A9800580024025402D901C3010B00022A38D11C
:108AA800BB4BDFF828831B78002B40F0DF87D8F812
:108AB800005045B32B7833B395F82820002A40F0AE
:108AC8002E812B7EAA6385F83C20042285F8282075
:108AD80013F008036A6AEA622A6303D0AD4A41F2D6
:108AE8009413D3586B634FF00009C5F82490C5F868
:108AF8000890C5F80C90284623F0F6FE0523C5F823
:108B0800409085F8283000220423C8F8002088F80F
:108B18001430A14BA14A5B681268C833934204D34E
:108B280022F0FAFF002800F0B381B278032A01F09E
:108B3800638001233B70022A00F0F180F378002B58
:108B48003FF45EAA964B1B68D90440F17B85954B90
:108B58009B8807EE903AF8EEE77A934991ED012A5F
:108B6800D1ED022A91ED033AD1ED043A91ED054A8F
:108B7800D1ED064A91ED075AD1ED085A91ED096AEF
:108B8800D1ED0A6A91ED0B7AB4EE672AF1EE10FA8C
:108B9800F4EE672A14BF01230023F1EE10FAB4EEB5
:108BA800673A18BF43F00103F1EE10FAF4EE673AA2
:108BB80018BF43F00103F1EE10FAB4EE674A18BF8C
:108BC80043F00103F1EE10FAF4EE674A18BF43F0E0
:108BD8000103F1EE10FAB4EE675A18BF43F001032F
:108BE800F1EE10FAF4EE675A18BF43F00103F1EE04
:108BF80010FAB4EE676A18BF43F00103F1EE10FAF9
:108C0800F4EE676A18BF43F00103F1EE10FAB4EE10
:108C1800677A18BF43F00103F1EE10FA18BF43F06A
:108C28000103002B40F0468491ED007AB4EE677A98
:108C3800F1EE10FA40F03E84584DD4F898102B68A5
:108C4800994200F23E843B78012B3FF4D9A994F86D
:108C58009720002A3FF4D4A90B2B0DD801229A4063
:108C680040F6030112EA01060BD112F4C06F03D0DB
:108C7800093B012B40F2CD87474B2A685A600B23EA
:108C88003B70002384F89730FFF7BAB9F9F764FD11
:108C98000790FEF780BD594604220CA821F0E0FE9B
:108CA8009DF83330AB2B04BF02236B76FFF7D5B9A1
:108CB8003068FAF725FA49463A201EF09BFB4946E8
:108CC800834604220CA821F0CBFEBBF1000F07D08D
:108CD8001EF0E8FB1EF0BEFB95F82420FFF778B8DD
:108CE8001EF0E0FB0C9B1BBAC3F38073AB76FFF757
:108CF800DBB99FED2E7AF4EEC76AF1EE10FA44BFA5
:108D08009FED2B7A77EE666A91E69FED2A7AD5ED8C
:108D1800037A77EE877AC5ED037AFEF710BE1D4A0F
:108D280041F2B513D35C002B00F0818794F897309B
:108D380001223A70002B3FF463A9A2E7F7EE006A1C
:108D4800FFF71CB8F7EE006AFEF79FBF1A49D1F883
:108D580000C0BCF936E0FFF7D2BB07EE906ADFED42
:108D6800176AB8EEE77A66EEA65A9FED155A9FED98
:108D7800156ADFED157AA5EE856A26EEA55AE5EEA9
:108D8800867AE5EE276A26EE870A5EE5048F0020DC
:108D9800542B0020E0740020682B0020B86A0020C3
:108DA800686C0020DC370020E0360020DB0FC9BFEC
:108DB800DB0F49C000000000843E002084F9223FF8
:108DC80092E741B99730083C15A82ABEF0930020D5
:108DD800B4F91420A179A8EB020686EAE670A0EBA4
:108DE800E670884240F376829045C8BF494207EE54
:108DF800901A95ED037AA361F8EEE77A012077EEF1
:108E0800277A2077C5ED037AFEF78ABD9F4B1B783A
:108E1800002B00F071831A200BF084FE002840F02C
:108E28006B8394F89730002B40F0668309233B70DE
:108E38000EF054FEB2787EE61A200BF073FE00287E
:108E4800F6D0934B1B88002BF2D1924B45201D681E
:108E580022F0A4FE0E2022F0A1FE28460EF0C0FA51
:108E6800059D28460EF0BCFA8B4A4FF480510A2320
:108E7800284611803B700EF02FFBD9E7874D22F072
:108E88000DFE874A6B68126864339342C0F09E8572
:108E9800B27850E6022A00F03884814B7F491B687B
:108EA8004B60804800230B6003210360397042E661
:108EB8007D4B1B78D9077FF53EAE802023F01EFC42
:108EC80008B11DF0A9FC0EF013FFB27833E622F0CA
:108ED800E5FD764B002105208DE80300A3F108028B
:108EE800029153200EF01AFE0028D1D16B4BB278B4
:108EF800186008233B701EE622F0D0FD6C4A0292EF
:108F0800A2F10C03292101930091A2F10A03502137
:108F1800163A49200EF002FE0028B9D15F4BB2780C
:108F280018604FF0FF31596007233B7003E622F0C9
:108F3800B5FD604B93ED000A29F03EFD5E4B93EDC5
:108F4800000A804629F038FD8146402022F088FD3D
:108F580000289DD1514D594A2B6892F801E0492BC0
:108F680000F26385DFE813F0F006FD06F6061D073C
:108F780016070F070807BD07B407A6079F07950739
:108F88008E078007230784087D08720867085C0835
:108F9800510846083B083008250814080408F40757
:108FA800E407D407C407090AF909E909E109D1095D
:108FB800C909C109B909B109A909A00997098E09FF
:108FC80086097E0975096C0964095C0954094C090C
:108FD8004609D808D108CA08C308BB08B308A008BE
:108FE800990892088B08E306DC06D506CE06C70664
:108FF800C006B906B20678067206660603236B70C9
:10900800FEF7F6BF2B690622652BAA7032D92A789B
:10901800032A14BF6FF0FF026FF07F02A3F165030C
:1090280003EA020303F1010314BF4FF480728022A4
:109038009A422B611ED23268EE6802329F1997421B
:1090480080F0AD851E4A6E60D16FAF60490203FBA8
:1090580001F30521166042F81C3C42F8183CA9703F
:10906800AA681849012026F0ABFA012840F00885C3
:109078000623AB700021144825F016FE012840F0A5
:10908800FF84AB780133DBB2AB7057E4E02B0020F0
:10909800CC290020D0290020C2290020682B0020DC
:1090A800B86A0020046C0020EB3C0020A45203089E
:1090B800C6500308DC290020D0370020683E002075
:1090C80074860020E4740020508600202A782B7DC6
:1090D800DFF8D493DB4ECDF81090032A14BF4FF479
:1090E80080784FF0800847461A46002A47D0012A60
:1090F800FBD1D5496B68096832684FEA412E4FF0B9
:1091080000094FF0FF31B1FBFEFE1EEB030049F1F1
:1091180000014FF00009494502F1020208BF9042E0
:109128009046CA4938BF03EB0E0202201EF008FB26
:10913800032800F2FD8101A353F820F0F97F00080D
:1091480055910008F97F000855910008D5F804E00A
:10915800AA682B69A2EB0E01994284BFC5F80CE0FE
:10916800296103283FF44EAF0132B2FBF7F107FB48
:10917800112109B13A44521A00216A6029753268EE
:109188000499023200201EF0DBFA032800F2D08195
:1091980001A353F820F000BFF97F00084D920008A2
:1091A800F97F00080D90000841F27013EB5C002B6A
:1091B8003EF41EAFA6481FF015FBFEF719BFA54BDE
:1091C80000930320A87030230522A349A04826F065
:1091D80065F9FEF70DBF00230DF130094946184621
:1091E80009221EF06DF901287EF402AF0C9A92F85C
:1091F800FE31552B00F09E8141F2B4120221012369
:10920800A9546B70FEF7F4BE0DF1300941F2FC165B
:109218004946A859002309221EF052F901287EF474
:10922800E7AE00230C9A2B70B2F80B30B3F5007F31
:1092380000F0508441F2B41203210123A9546B7049
:10924800FEF7D6BE6A6885F814B00132AA6050E706
:1092580004212C2023F096FB032183464E2023F083
:1092680091FB0C210490362023F08CFB049B421CBC
:1092780002339A4009FA0BF9A2FB0901420A42EAB1
:10928800C152EA63FEF740BE74481FF0ABFAFEF71E
:1092980089BF73481FF0A6FAFEF77EBF71481FF01A
:1092A800A1FAFEF785BFBCF838109FED6F7A07EE7C
:1092B800901AF8EEE77A6D4967EE877AC1ED007A81
:1092C800FEF744BBB0EE677AFFF71BB8F0EE477ABB
:1092D800FFF72DB8217F19B1654923770B68236201
:1092E80023691344B3F5FA6FA8BF4FF4FA63B3F5D3
:1092F8007A7FB8BF4FF47A7307EE903AF8EEE77AC0
:10930800C5ED037AFEF70CBB237F002B3FF4DDAAE3
:10931800574B84F828201B6822772362FFF7D5BAB9
:1093280007EE905ADFED536A9FED537A84F8885020
:10933800F8EEE77A67EEA67A77EE876ABDEEE66A18
:1093480016EE103A2033402B40F28981DFED4B6A4C
:109358004B4BBDEEE77AC3ED006A17EE103A2033A7
:10936800402B00F2C3819FED477AF4EEC77AF1EE05
:1093780010FA40F31F84DFED445A9FED446A01E080
:10938800F0EE477AF4EEC67AF1EE10FA37EEE57AA7
:10939800F6DCDFED3F7AB4EEE77AF1EE10FA40F151
:1093A8000684DFED395A9FED3B6A01E0B0EE677A3B
:1093B800B4EEC67AF1EE10FA77EE257AF6D49FED80
:1093C8002E7AF4EEC77AF1EE10FA40F392819FED0F
:1093D8002D7A77EE677A67EEA75A9FED2F5A9FEDA1
:1093E8002F6A9FED2F7AA5EE856A27EEA55AA5EE7E
:1093F800867AE5EE077AC4ED237AFFF726B995ED6C
:10940800000A0493069229F0D7FA2649DFF89CC08F
:10941800D1F8EC10DFF898E0069AAEF800008CFB63
:10942800013CC917C1EBAC1107EE901AF8EEE77AC8
:10943800049BFDEEE77A17EE901AAEF80210FEF7DD
:10944800DDBA00BFE8860020F0860020E87400201E
:1094580050860020FDE90208FC7A03088485002074
:1094680098860020C88500206F12833A28000020C3
:109478000C94002035FA8E3CDB0FC93F0000000039
:1094880020000020DB0F4940DB0FC940E4CB164128
:10949800DB0F49C0E4CB16C192E741B99730083CCD
:1094A80015A82ABE94090020E4740020D34D621048
:1094B80088680020A04B1B6803F59C530833C4F848
:1094C80098303B78012B7EF49BAD94F89730002BB5
:1094D8007EF496AD032A00F0CE830EF009FC01233A
:1094E80084F89730FEF78CBDF0EE476AFFF793BA21
:1094F800B0EE667AFFF779BA05980DF0EDFF97E4BC
:1095080085F82430FEF774BD8B4BEE681B686B61E1
:10951800072385F82430002E3EF46AAD2B692A68AB
:1095280069680120B04795F82420531EFEF757BDFF
:109538002A7DDAE592F8FF31AA2B7FF45DAED2F8E6
:10954800C6314BB192F8C211A1F10B0001282DD9F7
:1095580001F0F701062929D0D2F8D6314BB192F89B
:10956800D211A1F10B00012820D901F0F701062939
:109578001CD0D2F8E6314BB192F8E211A1F10B0000
:10958800012813D901F0F70106290FD0D2F8F631D6
:10959800002B3FF431AE92F8F221A2F10B01012920
:1095A80004D902F0F702062A7FF426AE41F2FC1134
:1095B80001226B50AA7029E6DFED607AF4EEE76AC3
:1095C800F1EE10FA40F36683DFED5D5A9FED5D6AB8
:1095D80001E0F0EE676AF4EEC66AF1EE10FA76EE94
:1095E800E57AF6DCDFED586AF4EEE67AF1EE10FA89
:1095F80040F14D83DFED525A9FED546A01E0F0EEE1
:10960800667AF4EEC67AF1EE10FA77EEA56AF6D429
:10961800DFED4F7AF4EEE76AF1EE10FA05DDDFEDE3
:10962800477A77EEE66AFFF79EBBDFED4A7AF4EEFB
:10963800E76AF1EE10FA44BFDFED437A77EEE66AA7
:10964800FFF791BB444B1B78002B40F0EA81434B5A
:109658001B8B07EE903AF8EEE77AFFF77EBAF4EE46
:10966800C77AF1EE10FA40F3A982DFED355A9FED83
:10967800356A01E0F0EE476AF4EEC66AF1EE10FAD8
:1096880036EEE57AF6DCDFED306AB4EEE67AF1EE36
:1096980010FA40F18982DFED2A5A9FED2C6A01E029
:1096A800B0EE667AB4EEC67AF1EE10FA77EE256A75
:1096B800F6D49FED277AF4EEC76AF1EE10FA40F37C
:1096C800C2819FED1E7A77EE666A66EEA65A9FED16
:1096D800245A9FED246A9FED247AA5EE856A26EE2A
:1096E800A55AA5EE867AE5EE076A31E6DFED1F7A20
:1096F80081E69FED187AF4EEC77AF1EE10FA44BFCE
:109708009FED117A77EE677A65E6DFF8648098F85E
:109718001430052B3FF6BCAB01A252F823F000BF72
:1097280091990008998E000815990008DB970008A0
:1097380011980008CF990008B86A0020DB0F49404B
:10974800DB0FC940E4CB1641DB0F49C0E4CB16C19F
:10975800DB0FC93FDB0FC9BFA85900208059002083
:1097680092E741B99730083C15A82ABE00000000CE
:10977800F0930020D8F8042092F91A104B1C5C468C
:109788000AD0C44B01F5817103EB0113FF20D9798D
:109798006FF30001D971907692F91B104D1C15D00A
:1097A800BC4D01F5817105EB011305EB0115DB7962
:1097B800E979C3F34503012BC6BF03F1FF33DBB2DD
:1097C8000023FF2063F34601E971D076032388F86C
:1097D8001430B148D8F804100378002B7FF458AB44
:1097E800002900F05A8291F82830002B7FF450AB02
:1097F8002838442228F0D8FE0021D8F8040025F0A3
:1098080007FB0023C8F80430D8F81050DFF8A8A2E6
:10981800DFF8A8E2DFF8A8C2A04B05F1010BAAFB0C
:109828000B59ACFB0B5CAEFB0BE506959C4DA5FB01
:109838000BE50895069D0FCBAD090995089D4FEAE4
:10984800D90E4FEA5C1C6D0B0DF13009CDF810C034
:109858000695AAFB0EC5CC46ACE80700049A8CF81E
:109868000030AAFB02020998D20801460892ED08C6
:10987800AAFB0112069905EB8505AEEB4505AAFB87
:10988800011AD108089A089501EB8101049DA0EB03
:1098980041014FEADA0A069802EB8202A5EB42027E
:1098A8000AEB8A0A7B4D41F2A4030EEB8E0EA0EB65
:1098B8004A0A0898EB5CABEB4E0B303001F1300EE6
:1098C8000BF1300B30320AF1300A01218DF83600E5
:1098D8008DF837B08DF835208DF834E08DF833A049
:1098E80088F81410002B00F0708141F2E803EB5C5B
:1098F800002B00F0698141F22C13EB5C002B00F087
:10990800C481042388F81430FFF7C2BA654DDFF824
:10991800B491DFF8B4A1A3460BAA2946D8F80400ED
:1099280025F03CF9012849464FF0030240F04981EF
:109938000B9C2046002C3FF41DAF2378002B3FF4EE
:1099480019AF2BF0B8F9032251460028E4D104F1ED
:1099580008002BF0B0F903460028DDD154F8030FB6
:109968000C9022798DF834200CA88DF8353028F029
:10997800F3FDD8F81030984203D90CA828F0ECFD74
:109988000346C8F81030C7E7424D6B78032B7FF4C5
:109998007FAA41F2A4020123AA5C88F81430002AA5
:1099A80000F0928141F2E802AA5C002A00F07D8171
:1099B80041F22C13EB5C002B00F07681002388F831
:1099C8001430FFF765BAB278FFF767BA402022F083
:1099D80047F800287FF45CAA2B68DFF8F080DFF8EE
:1099E800F0A04FF040090DE022F0D8F8DAF8002096
:1099F8002B68013A0133B9F10109CAF800202B603C
:109A080000F09C8118F803301846002BECD1002395
:109A18004FF0FF322B6004236A603B70B278FFF787
:109A28008AB8DFED217AFFF798B822F075F8002898
:109A38003FF42EAA1D4BB2784FF4805119800A23A7
:109A48003B70FFF778B89FED1A7AF4EEC76AF1EE2B
:109A580010FA44BF9FED177A77EE666A35E600F094
:109A6800C480042385F82430FEF728BB0021D8F8E9
:109A7800000025F0CDF900287FF445A8FFF708BAC3
:109A880002287EF4B5AA41F2B4120123AB546B70DC
:109A9800FEF7AEBAE0740020C0860020DC7F030821
:109AA8005917B7D1F893002000000000C229002000
:109AB800DB0FC9BFDB0F49C0CDCCCCCCD34D621076
:109AC8001F85EB51107B0308147B030850500308D3
:109AD800046C0020137C022B7FF4ACAB92F8FE31AF
:109AE800552B7FF4A7AB92F8FF31AA2B7FF4A2ABDA
:109AF800D189AF59B14B0F441F60567B41F21020FA
:109B0800731E7F2B2E503FF695AB734236EA030344
:109B18007FF490AB41F218207302013B2B50D08A9E
:109B280000B9506ADFF83CE341F20423E850B2F888
:109B380011305B0103F2FF135B12CEF80030B2F86C
:109B480013C0BCF1000F01D1D2F820C04000194465
:109B58000144ACEB010141F2082E40F6F47CB1FB64
:109B6800F6F1614545F80E1040F281804FF6F47623
:109B7800B14278D903212970D26A91493B441844EB
:109B880041F20C2641F21C230978A851EA5009B980
:109B98001EF0FAFDAB780133AB70FEF729BA24F05A
:109BA80047FF2B69FFF74EBAF0EE476A81E5F0EE02
:109BB800477A04E4B0EE677AFFF7EBBBB0EE667A5B
:109BC80061E55C46FFF764B90B4603EB031305EB4D
:109BD800830000F585507B4B009349463C232022A7
:109BE800043025F05BFCFFF753B91DF075FB022824
:109BF8007EF466AAFEF762BA734D286819F0F4FD80
:109C0800724B1B780022022B2A603BD0B278FEF7F9
:109C180090BF452021F0C2FFFF2021F0BFFF6C4814
:109C280021F08EFF304621F0B9FFFFF725B8022258
:109C3800FEF784BF674B68491A68684828F078FAC5
:109C48002B68B27801332B60FEF775BF92786249B2
:109C5800634828F06DFAF3E7624B5F495A8A624815
:109C680028F066FAECE702222A70002285E7012331
:109C78002B70FFF7DFBA802022F040FD00287EF429
:109C8800BFA92AE41CF0E0FDC0E702239DE7F0EE3F
:109C9800676ABDE4F0EE667AA4E41EF075FD00285C
:109CA8007FF4AAADFFF7F4B80223442202FB035362
:109CB80003F585504D4B0093102213234C49043073
:109CC80025F0ECFBFFF7E4B81346EEE7454B4249B5
:109CD8001A88484828F02CFAB2E7424B3E499A784D
:109CE800454828F025FAABE73E4B3B491A794348EB
:109CF80028F01EFAA4E79AF808203749404828F0C7
:109D080017FA9DE7BAF8242033493E4828F010FA9C
:109D180096E79AF8202030493B4828F009FA8FE75F
:109D28009AF81E202C49394828F002FA88E794F856
:109D380094202949364828F0FBF981E718F80330C0
:109D4800002B7FF4A5A862E6324A3349334828F04D
:109D5800EFF975E7324B334A3349344828F0E8F9CC
:109D68006EE7334A334B019200932A4A324B334908
:109D7800334828F0DDF963E71A4B1749DA8A314886
:109D880028F0D6F95CE7174B13499A8A2E4828F031
:109D9800CFF955E7737832782C492D4828F0C8F95F
:109DA8004EE72C4A1C492C4828F0C2F948E72B4BAF
:109DB80009491A682A4828F0BBF941E7E0860020DB
:109DC800C08600206BAF0208086C0020712B0020B1
:109DD800D07F0308008F0020AC7B0308C47F0308F2
:109DE800B87F030880590020A47F030825BA020819
:109DF800087B0308947F0308807F03086C7F0308AF
:109E0800587F03083C7F0308207F03080C7F030862
:109E1800F47E0308187B0308247B0308287B0308C7
:109E28004C79030840790308747B03087C7B03089A
:109E3800647B030858790308387B0308407B0308D0
:109E4800507B0308BC7B0308B07B0308987B03089E
:109E5800A07B03086C3E00208C7B0308484C002044
:109E6800387C030800870020AE4B5B79012B7FF418
:109E7800E7AEB4F99030B4F99220AB49AB4828F07A
:109E880057F9DDE6AA4BAB491A88AB4828F050F9D8
:109E9800D6E6A448A9498378427800780090A84873
:109EA80028F046F9CCE6A74B1B68D80409D40C2344
:109EB8002B60C5E6A44B9F491A8AA44828F038F9B4
:109EC800BEE6A34B9B491A78A24828F031F9B7E6B9
:109ED8001FFA89F31FFA88F293499F4828F028F956
:109EE800AEE64FF07E529D499D4828F021F9A7E63D
:109EF8009C4B9D49D3F800E09C489EF80D309EF895
:109F08000C209EF80EE0CDF800E028F011F997E655
:109F1800944B9549D3F800E095489EF80A309EF88E
:109F280009209EF80BE0CDF800E028F001F987E65B
:109F38008C4B8D49D3F800E08E489EF807309EF888
:109F480006209EF808E0CDF800E028F0F1F877E662
:109F5800844B8549D3F800E087489EF804309EF882
:109F680003209EF805E0CDF800E028F0E1F867E668
:109F78007C4B7D49D3F800E080489EF801309EF87C
:109F880000209EF802E0CDF800E028F0D1F857E66E
:109F98007B4B75497B480C2202FB0E3E9EF806302F
:109FA8009EF805209EF807E0CDF800E028F0C0F8FC
:109FB80046E6734A744975480C2303FB0E2EBEF817
:109FC8000A2028F0B5F83BE66D4A6F4970480C2323
:109FD80003FB0E2E9EF8082028F0AAF830E6684AFF
:109FE80069496C480C2303FB0E2E9EF8042028F0C8
:109FF8009FF825E6624A644967480C2303FB0E2E46
:10A008009EF8032028F094F81AE65D4A5E496348F2
:10A018000C2303FB0E2E9EF8092028F089F80FE682
:10A02800574A59495E480C2303FB0E2E9EF801201F
:10A0380028F07EF804E6524A53495A480C2303FB99
:10A048000E2E9EF8022028F073F8F9E50C2303FB86
:10A058000EFE4B4B4C4913F80E20534828F068F875
:10A06800EEE5524B48491A78514828F061F8E7E57F
:10A07800504B45499A78504828F05AF8E0E54F4B3C
:10A088004149DA784E4828F053F8D9E54D4B3E4916
:10A098001A784D4828F04CF8D2E54C4B3A49DA7812
:10A0A8004B4828F045F8CBE5484B9FED4A7A1B888A
:10A0B8003549494807EE903AF8EEE77A67EE877A2D
:10A0C800FDEEE77A17EE902A28F032F8B8E5394A1B
:10A0D8001549138A4148928928F02AF8B0E5354A8B
:10A0E8001149D3893E48528928F022F8A8E5314B16
:10A0F80025495A793B4828F01BF8A1E52D4B224900
:10A108001A79394828F014F89AE52A4B1E49DA7862
:10A11800364828F00DF893E562791B49344828F051
:10A1280007F88DE5DC930020DC7B0308287C030816
:10A13800D829002038AA0308207C0308047C0308D7
:10A14800107C0308D4290020083B0020F07B03087A
:10A15800DF8D0020F87B0308E47B0308C87B030835
:10A16800D07B0308843E0020C07C0308F87C0308E9
:10A17800F07C0308E87C0308DC7C0308D47C030833
:10A18800E43A0020CC7C0308AC7B0308B07C0308CD
:10A19800A47C0308987C0308907C0308847C03084B
:10A1A800787C0308707C0308687C0308308C0020E6
:10A1B800547C030810440020447C0308F82B00203A
:10A1C800E47E0308082C0020D47E03081829002008
:10A1D800C47E03080000C842B87E0308A47E0308B2
:10A1E800947E0308847E0308707E0308647E030857
:10A1F800547E030822796949694827F099FF1FE5C9
:10A20800684B66491B6868489A8D27F091FF17E5E7
:10A21800644B62491B6865485A8D27F089FF0FE532
:10A22800604B5E491B686248DA8F27F081FF07E5BB
:10A238005C4B5A491B685F489A8F27F079FFFFE407
:10A24800584B56491B685C4893F83B2027F070FF31
:10A25800F6E4544B51491B68584893F83A2027F0C4
:10A2680067FFEDE44F4B4D491B6855481A8F27F09F
:10A278005FFFE5E44B4B49491B685248DA8E27F0EB
:10A2880057FFDDE4474B45491B684F4893F830209A
:10A2980027F04EFFD4E4434B40491B684B4893F8E2
:10A2A8002F2027F045FFCBE43E4B3C491B6848482C
:10A2B80093F8282027F03CFFC2E43A4B37491B6843
:10A2C8004448DA8C27F034FFBAE4364B33491B682C
:10A2D80041489A8C27F02CFFB2E4324B2F491B6877
:10A2E8003E485A8C27F024FFAAE42E4B2B491B68C2
:10A2F8003B481A8C27F01CFFA2E42A4B27491B680D
:10A3080038489A7F27F014FF9AE4264B3649D3F849
:10A3180000E036489EF81C309EF81B209EF81DE091
:10A32800CDF800E027F004FF8AE41E4B1B491B68A8
:10A338002F481A7E27F0FCFE82E41A4B2A49D3F8EC
:10A3480000E02C489EF816309EF815209EF817E07D
:10A35800CDF800E027F0ECFE72E4124B2249D3F866
:10A3680000E025489EF813309EF812209EF814E06D
:10A37800CDF800E027F0DCFE62E40A4B1A49D3F876
:10A3880000E01E489EF810309EF80F209EF811E05D
:10A39800CDF800E027F0CCFE52E400BFAC7B030808
:10A3A800587E0308843E0020407E0308307E030860
:10A3B800247E0308147E0308FC7D0308E07D03085F
:10A3C800CC7D0308B47D0308A07D0308907D0308B5
:10A3D800807D03086C7D03085C7D0308507D0308BD
:10A3E800407D03082C7D0308C07C0308247D0308F6
:10A3F8001C7D0308107D0308087D0308007D030801
:10A408002DE9F04F9A4A9B49137895B00446099074
:10A4180000F59C4020300C900860002B00F07C84F4
:10A42800954909688C4240F29680944905910968DB
:10A438009348944CDFF888B20391013B137001F400
:10A44800805302900893002B40F09480029B5B7D20
:10A45800002B40F06283039B1E0400F11086039BCF
:10A46800DD050BD5099A884BDFF858A29A429AF86D
:10A47800022000F2CD87002A40F0CE87834B049358
:10A48800834D039B13F4805740F06783029BBBF90D
:10A4980006605B8B9E42B4BF002601267D4B1B687D
:10A4A80013F0805373D0049A127812F0010275D019
:10A4B80002987949808C91ED037A07EE900AF8EEBC
:10A4C800E77AB4EEE77AF1EE10FA80F2B086002E61
:10A4D80069D194F8A410002965D1704870490068C2
:10A4E80090F830004FF0000EC1F800E0C1F804E029
:10A4F800C1F808E06B49002856D10870002A57D0E7
:10A50800039AD10654D5684A1278D20650D4002F3F
:10A518004ED1002B4CD1039B5B0249D495F800C067
:10A52800BCF1000F01F05785604B9B78002E41F07D
:10A538008F853BB15E4A5F4B12681B689B1A002BE4
:10A54800C1F29D85102019F077FE012384F8A5300B
:10A5580095F800C02EE0494B05931B680393484AC1
:10A56800484C029203F48053DFF854B10893002B4F
:10A578003FF46CAF00214748FAF71AF900287FF436
:10A5880065AF10F0E1FB059B1B6803935EE7039A38
:10A59800500288D4049A127802F00102002184F84B
:10A5A800A410002E99D03F4901200870002AA7D195
:10A5B80095F800C0029ABBF900E0508B918BBBF96B
:10A5C80002208645CCBF8027002747F040038E45F0
:10A5D800A8BF3B469B0843F080078242C8BF3B4662
:10A5E80043F040078A42B4BF3A461A469208BBF97C
:10A5F80004E0BBF9067042F080038645C8BF1A46DE
:10A6080042F040038E45A8BF13469B0843F08002E2
:10A618008742D4BF1846104640F0400294F8A6304E
:10A628008F42ACBF014611468B4200F018840023CC
:10A6380084F8A61084F8A730BCF1000F00F0A585B7
:10A64800059B1D4A1B68039203F00403002B40F08E
:10A658000B830DF14808194D0023C8F8043005F1A3
:10A668005009129340F6330A192740F283362EE038
:10A67800902F00200C2E00208C2F0020686C0020CA
:10A68800805E0020441F0020404B4C00EB3C002023
:10A698002C0000201C94002074690020843E0020B7
:10A6A800A028002028260020D8930020241F00205E
:10A6B800B86A002054300020D4510020902B00208C
:10A6C800AC880020303E002004354D4520D0AA78C3
:10A6D800EB789A4217FB0260F6D26978043117FBCF
:10A6E80003623BF911305345A8BF5346B3F5617F68
:10A6F800B8BF4FF461739842E6DA9A42E4DB2978EE
:10A708002329E1D840460435F6F798FE4D45DED1B9
:10A71800AB4B98E803001E78AA4B83E80300002E91
:10A7280000F032820121A748FAF742F8002840F0E9
:10A738000C81059B1B68DC0500F10281A24C238873
:10A748001DB225F00105AFB2BB42278000F0FB83A4
:10A758009E4D02260F204FF014094FF0FF082E706F
:10A7680085F8019085F8028019F066FD3146954814
:10A778002788FAF71DF8002840F0958727F002038C
:10A788009BB2BB4223800AD0904B1421FF220225A2
:10A798000F201D7059709A7019F04EFD2788DFF848
:10A7A80058A28B4B9AF8001002935868BB0708BF51
:10A7B80081F00201C1F34001F8F7AEFC039B1B686E
:10A7C80013F00A0F24D005217E48F9F7F1FF00287D
:10A7D80000F0C68425886F0740F1E886794806218D
:10A7E800F9F7E6FF002800F0A8846E0640F1FB8622
:10A7F80007217448F9F7DCFF50B1764B764AB3F974
:10A808000430764982FB0302DB17C3EBA2030B80FB
:10A818000C216C48F9F7CCFF2288002800F0B180A1
:10A8280042F480739A42238009D0684B0225142190
:10A83800FF220F201D7059709A7019F0FDFC684BAB
:10A848001B78082B00F0A9800E2B00F0A680059B32
:10A858001B685D0542D5634B1B79002B58D014212A
:10A868005848F9F7A5FF002856D11FF061FA0120D2
:10A8780019F006FC90B3DFF8848100254FF0CC096D
:10A8880002E0DDB2022D29D809FB05F76B1C58F848
:10A898000760002EF5D1C378534A90F9020052F8A8
:10A8A80023300196032200920121324618F0C6FF98
:10A8B800034605EB450000EB0010059353B1314604
:10A8C80008EB8000CC222AF084F9059B48F8073071
:10A8D8000135EDB218F014FA0028D3D1049B1B7887
:10A8E800D80740F18D804149414A01230B7013700C
:10A8F800029B9AF80010186801F00101F8F70CFCA7
:10A90800039B1B685B0700F1EB8015B0BDE8F08F77
:10A91800049B1B78D907A8D53C2021F0EFFE00281E
:10A92800DCD01BF079FF3C2021F08AFE0028D5D02E
:10A938001BF072FF3C2021F083FE0028F1D1CDE707
:10A948002C4BDB78002B3FF4F9AE039B1B68980770
:10A958007FF5F4AE1C4C2788F9073FF50FAF47F099
:10A9680001039F4223803FF409AF184B1421FF22B3
:10A9780002250F201D7059709A7019F05DFC278808
:10A98800FCE622F480739BB29A4223807FF44DAF99
:10A99800134B1B78082B7FF457AF228822F0400313
:10A9A8009BB29A4223803FF452AF084B02251421F0
:10A9B800FF220F201D7059709A7019F03DFC46E770
:10A9C800DE3A00201C940020283E00200438002095
:10A9D800486B0020603E0020676666669A1E00206D
:10A9E8008C2B002034690020D06F0308EC3C002039
:10A9F800C41E0020303E0020446B00206438002034
:10AA0800AA4B93F80090B9F1000F5FD1DFF80083EB
:10AA1800A74F18F8030C3E784146A8F103050AF041
:10AA280057F8002800F0D482002E40F0268305F164
:10AA3800080168790AF04CF8002841F0D1819D4955
:10AA4800A87A0AF045F8002800F0D582022E41F0D5
:10AA5800CB819949E87B0AF03BF8002841F0B081A6
:10AA68009649287D0AF034F8002800F0D582042E93
:10AA780041F0AA819249687E0AF02AF8002841F03C
:10AA8800A7819049A87F0AF023F8002800F0D58212
:10AA9800062E41F0A1818C4995F823000AF018F898
:10AAA800002840F0E886894995F828000AF010F84F
:10AAB800002800F0D582082E40F0F386844995F8E6
:10AAC8002D000AF005F8002840F0D582814B0122BC
:10AAD8001A700AF05AFA039B1B685B077FF515AFDB
:10AAE80003200AF01FF8002800F0F185238813F0EE
:10AAF80008047FF40AAF082019F0ACFC7648774DBB
:10AB08007749784A784BBBF8066000682E80086061
:10AB180014601C6015B0BDE8F08F029A013BD27D2D
:10AB28003BF91330002A40F04983A3F57A73B3F553
:10AB38007A7FA8BF4FF47A7323EAE37307EE903A5B
:10AB48009FED6A7AF8EEE77A67EE877A684AFCEE54
:10AB5800E77A17EE903A138081E41D216548F9F7EA
:10AB680027FE00287FF492AC634A029BD2881B8B95
:10AB7800BBF90660991A8E4240F32F8613449E4211
:10AB8800B4BF0026012689E4DFF888915B4F09F1FC
:10AB98005A054FF00108494619F8010C09F098FFC9
:10ABA800F8B199F8040099F8023099F803E000EB3D
:10ABB800400104EB8101013BD1F8B42003EB4303CE
:10ABC8003B4493420DD094F8E02081F8B0E008FAB5
:10ABD80000F022EA0000C1F8B430C1F8B86084F887
:10ABE800E00009F10609A945D5D14549454A464B32
:10ABF8000968D2F8009093F800A0444D0691002609
:10AC08006B685BB31F784FB3AA68A9EB0202002AEE
:10AC18000ADB94F8E0200121B14022EA010209F59B
:10AC2800FA7184F8E020A960BAF1000F16D02A78EA
:10AC380059780432D2B2002940F0FE8202993BF9D9
:10AC48001220098B01F1C800824240F39A8594F8DA
:10AC5800E0209B783241D10740F1FC850136042E73
:10AC680005F10C05CCD15DE594F8AB3053B1049BEC
:10AC78001B78D80706D5029BBBF906205B8B9A4246
:10AC880000F3DA8511211B48F9F792FD002800F03E
:10AC9800B68294F8AE302BB994F8A93013B93223A0
:10ACA800A4F8AC30012384F8AE30D2E4EC3C0020A8
:10ACB80024000020D7310020DC310020E1310020C1
:10ACC800E6310020EB310020F0310020F531002082
:10ACD800FA310020C41E00200C940020A41E00207D
:10ACE800B01E0020A81E0020A01E0020AAF1823F4E
:10ACF800089400201C940020DC370020C45203086C
:10AD080078260020B86A0020FD3D0020F41F0020AE
:10AD1800CD310020E5300020994C9A4B26780293DB
:10AD2800994F002E00F06082B6B1DFF89492DFF8F8
:10AD380094B2DFF85482CA460025072D4046E9B28E
:10AD48007B6841F3D180984700B20135AE422BF8B9
:10AD5800020F0AF1040AF0D18C4B05931A4609999F
:10AD68008B4B12680392A3FB013E42F2010313408E
:10AD78004FEA9E1E079300F033828648864A874B27
:10AD880000788749069012781A70069B08702BB1D4
:10AD9800824B93F800B08BF001030693814A029925
:10ADA800127838781090B1F82680088D91F822C072
:10ADB8000B92098B0B9A119194F829107A4B0E90EB
:10ADC80008461146A3FB01135B0803EB4303D31AA0
:10ADD800DBB20D93039B2578744EDFF8ECB1DFF8F6
:10ADE800EC91CDF810800F220CF1040C03F4805381
:10ADF80084F828200A945FFA8CFC109C0F92AA46CB
:10AE080008930021804610972DB9A44599BFE246C2
:10AE18006546A2462546A94280F29482069B002BED
:10AE280000F04682624B049833F9112097B28742AA
:10AE38004FEA410303D30E98874240F2118259F832
:10AE48002120964580F03E823BF90320079F002F82
:10AE580040F00E822BF8032001310636D4E794F82F
:10AE6800A790B9F1F90F00F2DB8109F101095FFA46
:10AE780089F984F8A79084F8A610BCF1000F00F0B7
:10AE88008581B9F1140F7FF4DBAB5F2940F0918124
:10AE9800049E337813F0010300F04E870FF054FF3F
:10AEA800337803F00103002B7FF4CAAB94F8A62093
:10AEB800572A00F0C786059B1B6813F0040302D0CD
:10AEC8005A2A00F0F2845D2A00F027875B2A00F0F6
:10AED8002F875E2A00F0C484562A00F089872B78D1
:10AEE8002BB16F2A00F09F87324B00211960972AF7
:10AEF80000F08D87A72A00F092840021BB2A1291C6
:10AF080000F0CD87B72A00F0AA87BE2A00F0CA87CA
:10AF1800BD2A00F0C987792A00F0DF877A2A00F075
:10AF2800D5879E2A00F0CB879D2A00F0C087AE2ADD
:10AF380001F03D80AD2A7FF483ABFF21002015F09E
:10AF480074F8FFF77DBB02211B48F9F731FC002894
:10AF58003FF414AC2580BA073FF521AC47F0020353
:10AF6800BB4223803FF41BAC144B02201421FF2268
:10AF780018700F2059709A7019F05EF927880EE43E
:10AF8800441F0020805E0020903B0020686C002059
:10AF9800D34D6210E82D0020840100208501002097
:10AFA800FD3D0020912F0020ABAAAAAA701F002007
:10AFB800481F0020583000201C940020043800202E
:10AFC800F82F0020461F0020AC880020942F002076
:10AFD80008F10501687909F07BFD00283FF42FADE1
:10AFE800012E40F0FD8605F10D01A87A09F070FDEB
:10AFF800002840F0F986C249E87B09F069FD00287D
:10B008003FF42EAD032E40F0DB86BE49287D09F0C3
:10B018005FFD002840F0D886BB49687E09F058FDDE
:10B0280000283FF42EAD052E40F0D286B749A87F00
:10B0380009F04EFD002840F0CF86B54995F8230069
:10B0480009F046FD00283FF42EAD072E40F013848A
:10B05800B04995F8280009F03BFD002840F021840C
:10B06800AD4995F82D0009F033FD00283FF42EADC9
:10B07800092E3FF42BAD4FF009094B46FEE3D4F8F7
:10B088008C30099AD31A002BFFF6E9A9A34A94F841
:10B098009030517CA24A029D32F811200C98A97D6B
:10B0A800C4F88C00013303F00F0384F89030234474
:10B0B80092B292FBF1F283F8942094F8940094F8F9
:10B0C800951094F8962094F8973001440A4494F81F
:10B0D800980094F899101344184494F89A2094F816
:10B0E8009B3001440A4494F89C0094F89D10134442
:10B0F800184494F89E2094F89F3001440A4494F828
:10B10800A00094F8A1101344184494F8A23094F8BD
:10B11800A32001440B441A4442F30B12642AE97D2C
:10B12800A8BF642213B209B1C2F1640307EE903AD2
:10B138009FED7C7AF8EEE77A06E525F040039BB2AE
:10B14800AB4223803FF454AB774B02251421FF22F6
:10B158000F201D7059709A7019F06EF8FFF748BBF0
:10B16800238823F00405ADB2AB4225803FF436AB0B
:10B178006D4B02251421FF220F201D7059709A7003
:10B1880019F05AF82588FFF729BBE14600216748DE
:10B19800F9F70EFBB8B1002384F8A8300FF050FC83
:10B1A80094F8A730142B7FF44BAA2B78002B40F08F
:10B1B8004787049B1B7803F0010374E6C3F53B63E0
:10B1C80008331BB2B1E4049B594A1B781060DF07AF
:10B1D80000F11385B9F1140F3FF468AEFFF730BAE8
:10B1E800544B1B780693D2E593F822303E7804330B
:10B1F800DBB2B3428EBF267023701E4694E594F8E6
:10B20800A930002B3FF425AA049B1B7813F00103F7
:10B2180002BF012284F8A93084F8AA20FFF719BADE
:10B2280084F8A630BCF1000FB0D0FFF709BA0121AD
:10B2380084F8A410FFF7B7B9012900F0238594F822
:10B24800E0200123B34001361343042E84F8E03094
:10B2580005F10C057FF4D4ACFFF764BA1A464B002D
:10B268000EF5967749F82170079F002F3FF4F2AD4D
:10B278000D985F1807440A9800EB4707BA85B8F19C
:10B28800000F03D10B9802287FF6E4ADB6F80280D0
:10B298003288B78842441744274A3FB282FB0702E4
:10B2A8002648A2EBE772C75212B24FF00108D1E567
:10B2B800049B002BD2D059F8212096454FEA410330
:10B2C800FFF4C2AD1E4A1E48D25CC718002A00F01F
:10B2D8009281022A40F05B817A7802EB820202EBCB
:10B2E800820202F2EE2292B20329DFBF012000FAA5
:10B2F80001F70F98B843CEBF12B212B20F90A5E56E
:10B30800DC310020E1310020E6310020EB31002063
:10B31800F0310020F5310020FA310020C06A002009
:10B32800DC6A002014AE2341043800201C9400205D
:10B3380058300020FD3D002056555555B81F0020B7
:10B348002C3000200F990A9CB14B109F84F800A064
:10B358000F2942460CBF0122002284F8298084F874
:10B3680028101A7006D11B21AA48F9F721FA0028DB
:10B3780000F0C584A848A94B82681968A84BC16029
:10B388008A1A012119704368A64E9A42029A3170AE
:10B3980088BF002392F8226088BF80F82130089B7C
:10B3A8003878B2F826C0B2F818E00436F6B2002BA6
:10B3B80000F0508186429C4A40F2C1819B4E17465C
:10B3C80000210DB982460546A94218DA12F8113053
:10B3D80083B1022B0CD17B7803EB830303EB83034C
:10B3E80003F2EE239BB226F8023B01310237E8E76D
:10B3F8003388F8E7CBB2032BFAD87346F3E784F81F
:10B4080000A00B9B8A4A01331370089BFFF71BB8F7
:10B4180012B901228AF80220864B04931D789AF803
:10B42800218005F001031B20039309F07BFBB8F191
:10B43800010F079000F0D48105F0020306939AF8F3
:10B4480020207D4DDFF808927C4E744F052A00F2CB
:10B458009580DFE802F08579032F3E51B8F1010F9E
:10B4680004BF05238AF82030039B002B00F09C8042
:10B47800029B3868B3F91810B9F80230002261F35A
:10B488000F0263F31F42002361F30F0361F31F43AD
:10B49800DAF81410CBF804208842CBF8003040F2D8
:10B4A80021810323069347F230520323CAF81C2054
:10B4B8008AF82030338843F0020333800FF044FCCD
:10B4C8003A68DAF81C3013440422CAF818308AF8AB
:10B4D8002020B8F1010F40F024843B68DAF81820E6
:10B4E8009A424BD2287818B909F01CFB002845D19C
:10B4F800338823F0020333803A68B9F806306421B0
:10B5080001FB03234FF4806000228AF820208AF888
:10B518000320CAF8103018F085FF9AF8202095E724
:10B5280009F006FB012800F04184079B002B40F03E
:10B538005A81B8F1010F21D03B68DAF810209A42FD
:10B5480028D301238AF82030B8F1010FD4D099F814
:10B558000830012B1ED011F0FFFE9AF8202075E765
:10B56800039B002BDCD1079B4FF48060002B00F07D
:10B57800AB8018F06FFF0022CAF81020069B002B42
:10B5880040F0AC80059B1B680393FEF77BBF3BF83C
:10B598000320A9E611F0E0FE032240F6B8338AF84A
:10B5A8002020CAF81C3085E73B687CE745F0040397
:10B5B8009D4223800AD0224B02251421FF220F200E
:10B5C8001D7059709A7018F037FE25881D4B1E4A59
:10B5D800B3F904301D4982FB0302DB17C3EBA20356
:10B5E8000B80FFF7FBB845F04003AB4223807FF4A4
:10B5F800ABADFFF7FDB8CAB2022A40F2FB82032ABC
:10B60800C5D1119A0898049F002808BF3A466BE6EE
:10B618008E3B00201C940020303E0020B86A002099
:10B6280084010020850100202C300020AC880020F7
:10B63800912F0020EB3C00202C00002024940020B7
:10B6480004380020603E002067666666901E002071
:10B65800F437002086421946B04A4BD8B0481746FE
:10B668000DB9B24635468D427FF7C9AE12F8113092
:10B6780083B1022B0CD17B7803EB830303EB8303A9
:10B6880003F2EE239BB220F8023B01310237E7E7D1
:10B698000388F8E7CBB2022B03D9032BF8D1634612
:10B6A800F1E77346EFE727F001039BB2BB42238023
:10B6B8003FF451AC0F202E7085F8019085F8028078
:10B6C80018F0BAFD278846E418F0ACFE53E70820C6
:10B6D80018F0A8FEFFF719B903230693069818F087
:10B6E800ABFD4FE7B8F1010FF6D103239AF82020FC
:10B6F8000693ABE68A4E17460DB982460546A9421F
:10B70800BFF67DAE12F8113083B1022B0CD17B78D5
:10B7180003EB830303EB830303F2EE239BB226F8C8
:10B72800023B01310237E7E73388F8E7CBB2022B57
:10B7380003D9032BF8D16346F1E77346EFE778485E
:10B74800174600210DB9B24635468D427FF757AEF0
:10B7580012F8113083B1022B0CD17B7803EB8303F1
:10B7680003EB830303F2EE239BB220F8023B013183
:10B778000237E7E70388F8E7CBB2032BFAD873461A
:10B78800F3E7C8398A423DDA94F8E0209B783241E1
:10B79800D2073FF563AAC3F10008012018F02AFE7A
:10B7A8007A1E162A00F2E780DFE812F0D801EC01D1
:10B7B800C101390100021102AE019B01860171012C
:10B7C8005C01E500390149011102AE019B01250127
:10B7D8001101FD00E800A300D2000126FEF75EBEBD
:10B7E800002306932BE699F80430002B3FF4A1AE12
:10B7F80011F0B2FD03224FF47A738AF82020CAF8B8
:10B808001C3057E694F8E0300122B24023EA0203E4
:10B8180009F5FA7284F8E030AA60FFF71FBA4149C7
:10B82800059B0A781B6842F004020A7003F00403BF
:10B838003D4A0392FEF70ABF00213C48F8F7B8FFDB
:10B8480000287FF41FAA322384F8AB00A4F8AC3098
:10B85800FFF718BA9846002B0CBF012002209DE77D
:10B86800334B02220320334D33492A700B6018F002
:10B87800C1FDFEF7E5BE4FF007094B4603EB830316
:10B888001D4487F80090A978687812F031FE049B6F
:10B898002A4A1B7801211170DA077FF51AA9FFF7E8
:10B8A80027B84FF008094B46E8E794F8A920002A82
:10B8B80040F0A78394F8AB2082F0010284F8AB2013
:10B8C800002A40F099831E49096811F4003104D018
:10B8D8001C490979002940F0AE830A461A48855C5C
:10B8E8000D2D02F10C0200F0498301311529F6D122
:10B8F8009EE7D4F8E400154B90F83B109A78414441
:10B90800FE29A8BFFE2121EAE17180F83B10002A38
:10B9180040F0C28322F012F991E400BF2C300020DD
:10B92800AC880020D8930020D45100201C9400201B
:10B93800848E0020683E0020843E0020C41E002023
:10B94800DC300020DC93002080570308E8930020B7
:10B95800D4F8E400B74B90F83A109A784144642937
:10B96800A8BF642121EAE17180F83A10002AD1D0F9
:10B97800172009F00FF9D4F8E400CBE7069AAD4B8D
:10B9880051784144B1F5967FA8BF4FF4967121EAEA
:10B99800E17151709B78002BEDD0152009F0FAF871
:10B9A800D4F8E400B6E7D4F8E4008178A14B414428
:10B9B800C829A8BFC82121EAE17181709B78002BB2
:10B9C800A8D0142009F0E6F8D4F8E400A2E7D4F8E7
:10B9D800E4004178974B4144C829A8BFC82121EA0F
:10B9E800E17141709B78002B94D0132009F0D2F8B4
:10B9F800D4F8E4008EE7D4F8E40001788D4B414494
:10BA0800C829A8BFC82121EAE17101709B78002BE1
:10BA180080D0122009F0BEF8D4F8E4007AE706983E
:10BA2800844B81799A7841446429A8BF642121EA2A
:10BA3800E1718171002A40F0F4820D2F9BD00698A5
:10BA48007C4B41799A7841446429A8BF642121EA52
:10BA5800E1714171002A8ED00E2009F09BF8D4F8CC
:10BA6800E40057E7D4F8E400724B017A9A7841442D
:10BA7800C829A8BFC82121EAE1710172002A3FF450
:10BA880049AF0B2009F086F8D4F8E40042E7D4F86F
:10BA9800E400684BC1799A784144C829A8BFC821F5
:10BAA80021EAE171C171002A3FF434AF0A2009F09C
:10BAB80071F8D4F8E4002DE7D4F8E4005D4B8179FF
:10BAC8009A784144C829A8BFC82121EAE171817147
:10BAD800002A3FF41FAF092009F05CF8D4F8E4000D
:10BAE80018E7D4F8E400534B41799A784144C829BF
:10BAF800A8BFC82121EAE1714171002A40F08B8278
:10BB0800112F7FF452AF05E7D4F8E400494B0179CF
:10BB18009A784144C829A8BFC82121EAE171017176
:10BB2800002A40F0B382102F7FF453AFF2E6069A52
:10BB380017794744642FA8BF642727EAE777177166
:10BB480009F042F83B4B9B78002B3FF414AF0320DD
:10BB5800394609F01FF8D4F8E400DBE6069A354BBD
:10BB680011784144FA29A8BFFA2121EAE17111703C
:10BB78009B78002B3FF4FFAE012009F00BF8D4F8B6
:10BB8800E400C7E6069A2B4B917841446429A8BF84
:10BB9800642121EAE17191709B78002B3FF4EBAEB0
:10BBA800022008F0F7FFD4F8E400B3E60698214B2A
:10BBB800C1799A78414481F30801C171002A3FF4A0
:10BBC800DAAE052008F0E6FFD4F8E400A2E6D4F8DF
:10BBD800E400184BC1789A784144C829A8BFC82105
:10BBE80021EAE171C170002A40F01F820F2F7FF413
:10BBF80004AF8FE6119AFFF777BB0F4B1B78002B2A
:10BC08003EF41EAD0D4BDB78002B7EF419AD94F895
:10BC1800A8300133DBB2032B84F8A8307EF610ADD0
:10BC2800074B5B7813B9002E7EF40AAD0FF08CF841
:10BC3800FFF7B6BAE8930020FD3D0020303E002013
:10BC4800241F0020BA4ABB4B039210461A68BA490F
:10BC58004FF47A73B3FBF2F3C3EB431203EB8203A3
:10BC68000268DB005507A1F8A83055BF059B059B66
:10BC78001B68B24A42BF1B680A21118003F0040303
:10BC8800FEF7E4BC3BF912209978B2F5617F4FF4D6
:10BC9800966393FBF1F3C0F2818040F63301914241
:10BCA800A8BF11460C2FA1F5617191FBF3F800F0C4
:10BCB800BE80182F7FF4C3AA5FFA88F1C8290B4603
:10BCC800A8BFC823D4F8E400C27DDFB297423FF48E
:10BCD800B6AA9B1A9A4AC77548BF0733DB109278F1
:10BCE8005F1CFFB23AB9002F3FF4A9AA384618F0F2
:10BCF80081FBFFF7A4BA182008F04CFFF3E791493D
:10BD0800914BCA681B688B609B1AC82B7FF679AB6E
:10BD1800012381F82130FFF774BB8C4B00220120EE
:10BD2800A1E53968DAF81C200A44CAF8182025E485
:10BD3800874B0122022096E5864A1268960304D5AD
:10BD4800854A1279002A40F03A81844819461A46F1
:10BD5800465C0B2E01F10C0107D00132152AF7D1F0
:10BD6800002284F8A720FFF79EB87D4ED6F800E0A1
:10BD78005100BEF1000F07D08F1800EB87079EF81F
:10BD880001E07F787745EBD20A44764F764900EB9D
:10BD980082020020326038800860E1E70C2F5BD017
:10BDA800182F7FF44CAA00210B468BE73A68B9F8A4
:10BDB8000630642101FB0323CAF81030FFF7B5BB36
:10BDC8004FF003094B4659E54FF004094B4655E53A
:10BDD8004FF005094B4651E54FF006094B464DE536
:10BDE8004FF001094B4649E54FF002094B4645E53E
:10BDF8000DF08CFCF8F752F80DF070FCF7F770FEB8
:10BE0800012018F0F7FA94F8A620FFF768B8059B08
:10BE1800564A1B684FF4C8711180454A039203F0D3
:10BE28000403FEF713BC0EF00BFEFEF709BC5FFA25
:10BE380088F74F4B5B78BB423FF401AA38460FF0B6
:10BE480003FC3F4B9B7823B15FFA88F10C2008F084
:10BE5800A1FE0137FFB246E70027B846E9E70B46DF
:10BE68004FF6FE71434A32485589039090892B4416
:10BE78000144538191810DF049FCF8F70FF80DF05A
:10BE88002DFCF7F72DFE012018F0B4FA059B1B686E
:10BE9800002203F0040384F8A720FEF7D7BB0B4663
:10BEA8000221DFE70223DDE74FF6FE73DAE7002120
:10BEB800FF2014F0BAF894F8A620FFF738B801204C
:10BEC80014F0B3F894F8A620FFF72EB82A4A137A8C
:10BED80043F001031372FEF7B3BB274A137A23F02A
:10BEE80001031372FEF7ACBB029A515D9847032D0C
:10BEF8001BDC40F2EE2240F6CA0C00283EF425AFC7
:10BF080039F825E0BAF802104FF47A73A0EB0E0066
:10BF180003FB00F0A1EB0E0190FBF1F018449042F6
:10BF2800B8BF10466045A8BF604600B2FEF70DBF17
:10BF3800D4510020484C002024440020942600209E
:10BF4800E8930020303E0020B86A0020F08D0020E1
:10BF58003A8E0020DC300020DC9300208057030854
:10BF6800D82500206E260020702600209626002066
:10BF7800683E002018290020743B0020494E37688D
:10BF88004A003FB1551800EB85057F786D78BD42B2
:10BF9800BFF44EAC0A4400EB8202434F434D32607B
:10BFA8000021434A398029600392FEF74FBB0121E3
:10BFB800002014F03AF894F8A620FEF7BBBF3D4ADB
:10BFC8001278002A7FF4C1AE18F01AF9049B1B7886
:10BFD80003F00103C4E6002E3EF4B4AA94F8A5C009
:10BFE800BCF1000F3EF4E6AA18F00AF995F800C073
:10BFF80084F8A570FEF7DEBA0C2018F01DF9FEF7DC
:10C008001FBB0122002184F8AA20294A84F8A9101C
:10C018000392FEF71BBB112008F0BCFDD4F8E40026
:10C028006EE50D2008F0B6FD07E50F2008F0B2FD1B
:10C03800D4F8E400DAE51F49097829B111464DE43E
:10C0480094F8A610FEF721BF18F0DAF8FEF7F8BA50
:10C058003BB11949194A09684FF47A7000FB031378
:10C06800136094F8A530002B3EF4A4AA18F0C8F881
:10C07800002384F8A53095F800C0FEF79BBA0EF0AF
:10C0880063FE002384F8A530FEF792BA102008F06A
:10C0980081FDD4F8E40046E5162008F07BFDD4F8CD
:10C0A800E40037E4D82500206E2600207026002002
:10C0B800D451002073690020B86A00205430002051
:10C0C800F8B55D4B1B78DB072DD55C4B5C4D1C78B8
:10C0D8005C4E012C49D079D3022C1BD06B7A7BB1F2
:10C0E800EB886BB1584B1B7853B119F0E7FF002868
:10C0F8007CD0AB7A83422CBF01230023337000E04D
:10C10800337852492A7A9C4238BF1C460C70002A60
:10C1180053D1F8BD4E494F4A098812889142DDD95A
:10C1280001241C70DAE74A4B4B48454D1988EC78D6
:10C13800B0F8E830A142A1EB030303F1020223D3D4
:10C148002B788B4220D33D4B1C78032C51D03D4E8D
:10C15800424A1278022A04D13B4F414A3F78D7809D
:10C168009480012CA0F8E810B5D13A4A38491288D1
:10C17800E87A0988121A914235DD3A4A12888A42C9
:10C18800ACD200241C70A9E7B1EB440FDBDC2B4BCD
:10C198001C78032CDBD0042AD9D82A4EDFF8A8C093
:10C1A800DFF8C0E02B4F0022032434701C708CF899
:10C1B8000020AEF800203A80CAE7012C36D0022CC5
:10C1C80010D10720BDE8F84018F036B8254A2049B4
:10C1D8001288E87A0988121A91423FF77FAF012442
:10C1E8001C707BE7F8BD02241C7077E702233370CC
:10C1F80087E7042AABD82A7891FBF2F20132082AA1
:10C20800DFF844E06C78AE78164FA8BF08228EF8A5
:10C21800002092B216FB02F614FB02F20D4C3E808F
:10C22800084E2280002434701C7091E70820BDE875
:10C23800F84018F001B800BFEB3C0020A85F0020D0
:10C24800DC930020AE5F0020736900201894002062
:10C258001C690020AC5F0020441F00208568002076
:10C2680088680020AA5F00202DE9F04FBC4B1E789B
:10C278008BB0002E40F0BC80BA4BBB4C1D78DFF869
:10C2880014A3DFF81493DFF8148305F00105A4F173
:10C298000A0B54F80A3CBBB1CC2707FB06B7184673
:10C2A800F6F7B8FC80B154F80A0CF6F7ABFC14F8B2
:10C2B800023C8BB9242831D0F5B154F80A3C184611
:10C2C800F6F7A8FC0028EED10136032E04F1CC04C1
:10C2D800DFD10BB0BDE8F08F012B23D0022B2BD080
:10C2E800032B37D0042B67D0052B40D0062B4FD01B
:10C2F80054F80A2C1346D2E754F80A3C23281A4665
:10C3080000F08881994991F832108142C7D1984B41
:10C31800CAF80090C3F80C801346C0E7012304F85C
:10C32800023CCAE74D2854F80A2C0CBF022300230C
:10C3380004F8023C1346B2E700233C2804F8023C08
:10C3480045D03E28D4D10122032304F8012C04F857
:10C35800023CB2E7C02814D80022042304F8050CD4
:10C3680004F8040C04F8062C04F8023CA5E714F8B9
:10C37800063C14F8052C9A422FD814F8043C834242
:10C3880003D0002304F8023C97E7062304F8023C94
:10C3980014F801ECBEF1000F00F08C81BEF1010F22
:10C3A80000F0D08101360023032E04F8023C04F18A
:10C3B800CC047FF46EAF8CE714F8043C04F8030C4B
:10C3C8005840052304F8040C04F8023C75E70322DE
:10C3D80004F8013C04F8022C6FE714F8042CF9184F
:10C3E8004240013304F8042C04F8063C887264E7E0
:10C3F800604B186800283FF46CAFF7F719FB5E4BE9
:10C408005E4D03F5947A5E4B1868F6F703FC002836
:10C418003FF45FAF5A4B1868F6F7F4FB09281BD0B6
:10C428003F2819D02B68002B67D1042800F0B2816F
:10C438000C2800F0E8807F28E5D0A0F12002D2B2D5
:10C448005E2AE0D80BB92028DDD04E495A1CC854C2
:10C458002A6007F01FFAD6E72C68002C5BD1264625
:10C46800DFF8148100E0984608F10803002E08BFA1
:10C4780046465345F7D3002E6DD03068D8F80020D3
:10C48800075D135D9F42204402EB040140F07E816A
:10C498003C4F04F1FF3EBE4422460BB9FD2A7FD92A
:10C4A8000EF8013F01322A6010F8013F11F801CF60
:10C4B8009C45F2D00AB1B04512D0334807F0F2F9E2
:10C4C800B04508D356F8080B07F0ECF9092007F037
:10C4D800E1F94645F6D92D4807F0E4F92A68002421
:10C4E800944290D22A4E264416F8010F07F0D2F94A
:10C4F8002B6801349C42F7D385E70C2800F0838031
:10C508000A2854D00D2852D07F2800F00881FF2B2C
:10C518003FF679AF91E7184FDFF868B04FF00008A1
:10C5280007F59479464602E008374F450DD2224672
:10C538003968584628F098FB0028F5D1B846002EEF
:10C54800F2D13E4608374F45F1D3002E95D1B8F1C8
:10C55800000F3FF458AF0C4807F0A4F9B2E700BF4A
:10C56800DE3A0020EB3C00206E380020DC4300203F
:10C5780000ED00E0B426002070550308B82700201D
:10C58800B0260020B8260020D0800308D8800308F1
:10C59800B7260020FC9F0020EFBEADDE0400FA05A0
:10C5A800511C2020B85429607B540A4683E77D4FEC
:10C5B80007F0E5F93846232128F040FB002800F071
:10C5C800E780C01B286078B1431EF95C202940F041
:10C5D800E780FA1804E012F8011D202953D1034618
:10C5E800581E002BF7D12B604FF4807200216D4844
:10C5F80028F0EFFA6C4B1B78002B3FF46AAE6B48BF
:10C6080007F050F9FFE66A4807F04CF9674807F069
:10C6180049F9F8E667496848C978684ADFF8D0E117
:10C62800C2F8EC30003118BF012101706449C2F82A
:10C63800F0104021C2F8F43082F8F81082F8F9506E
:10C64800604961480B60F032CEF80020564A012359
:10C65800137007F075FE554807F024F95B4A5C49EA
:10C66800138891F8321043F080032329138005BF03
:10C67800584A14F8023C14F8023CC2F80C8008BF6F
:10C68800CAF8009032E62B60534C464E002204F55F
:10C698009479FA5402E008344C4573D22168304644
:10C6A80009F0C0FE0028F6D04C456BD26368984765
:10C6B800002398E7494BADF822E00FCB0DF1280C89
:10C6C80002AF87E80F004CF824ED14F8051C14F8A5
:10C6D800033C069404EB010E624639464FF0010C08
:10C6E80006A8CDF81CE0ADF820308DF824C0F8F786
:10C6F800CBFEE8B9019F002304F8023C002F3FF469
:10C70800E3AD54F80A0C16F0D1FF013654F80A0CC0
:10C71800B847032E04F1CC047FF4BBADD9E5013B47
:10C72800204A2F482B600021D15407F0BBF86AE655
:10C73800029A2C4B03923946A4F10A00029319F08D
:10C74800CBFED7E714F8053C14F8032C06942344D1
:10C7580007936E2A4FF0000308930993ADF8202041
:10C768007FF420AE631C06A80693F7F7B1FD0746D1
:10C7780006A8F7F7ADFD06A8F7F7AAFD1A4B1F6044
:10C7880058600FE6194807F08DF891E7224691E6C0
:10C79800286818E7034809F0D3F80BB0BDE8F08F14
:10C7A800034671E7B8260020DE3A0020D880030847
:10C7B800E0800308683E002070600020441F0020CD
:10C7C80049050008B02600200C81030824940020A5
:10C7D800DC43002000ED00E0705503080C5303080B
:10C7E80008810308E0950020F85F0020EC8003082A
:10C7F800B42600202DE9F04F2DED028B8FB00646B0
:10C808001DF096FA9C4B1F7827B10FB0BDEC028B38
:10C81800BDE8F08FDFF8C0B2DBF800305905F4D579
:10C82800964B974D1B78002B40F05C81954B1B78FD
:10C83800002B6BD0944C954AD4F86431F31A934288
:10C8480001F24B8094F86C81B8F1000F31D1904F10
:10C858003868F6F7DFF9C0B201280ED9022841F08E
:10C86800EE838C4B1A78002A41F0EB85D4F87021BE
:10C87800B21AB2F57A6F81F00E87D4F87431002BB2
:10C8880044D094F86C31BBB9834B1B689B78012169
:10C898001E3B00228B4284F86C1184F8802141F2FF
:10C8A80035863868022104301DF03AF994F8783159
:10C8B8000FE0D4F874314BB3D4F87C3140F6B7327A
:10C8C800F31A934222D994F87831002B01F0E882C8
:10C8D8006F4F013BDBB284F87831002B01F0718097
:10C8E800D4F8741194F8802111F801EB94F881318F
:10C8F800C4F8741172440133386884F88021714691
:10C9080084F88131F6F78AF9C4F87C61634B2F68A3
:10C918001B7853B1DFF8C481D8F8000028B1604B08
:10C928001B78013B012B41F25B805E4B1B7863B1A6
:10C938005D4F3B684BB1544CD5F80090D4F8B832F1
:10C94800A9EB0303632B00F22987584C2378022BA9
:10C9580001F08782DFF8888198F80030032B01F016
:10C968001C80534B1B7873B1524F3B685BB1464CEC
:10C97800F5F7F2FED4F8C032009044F61F62C31AED
:10C98800934200F283814C4B1B78002B4BD14B4BCD
:10C998001B7843B13C4CD4F8103403F5C333A033AF
:10C9A8009E4280F05B87464B1B78002B3FF42DAFEF
:10C9B800354E444C444D06F231472068F6F72AF9C3
:10C9C80000283FF422AF2068F6F71CF92B78804640
:10C9D8005A1E33B120682A70F6F71CF90028F2D1E4
:10C9E80013E703223946781E28F0D9F896F8303430
:10C9F80096F8312486F8338483F47F4383F0FF0369
:10CA08009B1A1FFA88F89BB2B8EB132FD5D196F86A
:10CA18003224DBB29A42D0D1781E1CF093FF2B78D7
:10CA280018442870C9E7294C2278002A40F0F68675
:10CA3800154CD4F8083403F5C333A0339E42A6D36B
:10CA4800234A94F80C34C4F80864D55CE90701F16A
:10CA5800F483AA0701F1B0836B0701F1BC821D4A78
:10CA680094F80C341178013393FBF1F201FB123383
:10CA780084F80C348BE700BFDE3A0020E069002020
:10CA8800B86A0020EA690020802000203F0D0300DA
:10CA9800846900202500002088690020EC690020B6
:10CAA800F4690020FC69002004870020422F002040
:10CAB800046A0020086A0020706A00207E6A00204C
:10CAC8000E6A0020146A0020186A0020D869002025
:10CAD800786A00207D6A0020686C00203069002098
:10CAE800050200205E4C2A68D4F85C31D31A7C2BEE
:10CAF8007FF69CAE94F86031DFF888919FED598AF3
:10CB0800C4F85C21013384F860314FF024084046B2
:10CB18001DF0BAF8544BF9EC016A1B8A07EE103A7B
:10CB2800F8EEE66AB8EEC77A08F10108C6EE877A29
:10CB38005FFA88F867EE887AFDEEE77ACDED007A3D
:10CB4800BDF900A05FFA8AF01DF074F8CAF3072057
:10CB58001DF070F8B8F1270FD9D130201DF094F8E6
:10CB6800424BDFF82481D3F800905FFA89F01DF07A
:10CB780061F8C9F307201DF05DF8D8F800005E21C0
:10CB8800F6F74CF894F860319A072DD1D4F85C2167
:10CB980041F288339A4201F24F8514201DF074F84F
:10CBA800334B344AB3F9043082FB03124FEAE3797A
:10CBB800C9EBA2090FFA89F95FFA89F01DF03AF872
:10CBC800C9F307201DF036F81C201DF05DF8002081
:10CBD8001DF030F800201DF02DF85E21D8F8000077
:10CBE800F6F71CF894F8603113F0070901F0A083F8
:10CBF800282B7FF41BAE00271720D5F8009084F867
:10CC080060711DF041F838461DF014F81A4B1B4CA2
:10CC1800A3FB09239B0BA4FB03125209C2EB0212CC
:10CC2800A3EB8203D8B21DF005F818201DF02CF8EC
:10CC3800134BA3FB09239B09A4FB03125209C2EB64
:10CC48000212A3EB8203D8B21CF0F4FF38461CF0A2
:10CC5800F1FFD8F800005E21F5F7E0FFE6E500BF38
:10CC68008020002000007A44083B0020883E0020F5
:10CC7800603E00206766666673B2E74589888888E3
:10CC8800D34D62103C3B00208C69002094F8C632DA
:10CC9800002B41F07D81E34B1A6802F00803002B5A
:10CCA80048F603414AF60B404BF60F4349F607484E
:10CCB80004BF0346884612F0040F4FF0190118BF4D
:10CCC8009846920684F8C61203D548F4804848F07E
:10CCD8002008D54B1A79C8F309010191002A41F0BF
:10CCE8003D855B79002B41F073869A4664204FF0AE
:10CCF800FF330A464FF00009CDF81880CDF81C80A4
:10CD08000892ADF826A0ADF828308DF83600ADF8B9
:10CD18002490CDF82A90CDF82E90CDF832900DF1D0
:10CD2800180CBCE80F00DFF810E384F85190AEE867
:10CD38000F009CE80F00AEE807002EF8023B714692
:10CD48004FF0010C1B0C4FF0FE0E1F20C82201F8FB
:10CD58001E3984F84EE084F8522084F853C084F8D1
:10CD68004F0094F8D60284F8500080F0F10383EA6B
:10CD78000313DAB2130983F0E70343EA022383EAD1
:10CD8800C2031BB283EA0312D2B2C3F3072383EAB6
:10CD9800121343EA022383EAC2031BB283F0C802D8
:10CDA80082EA0212D2B2C3F3072383EA121343EAD8
:10CDB800022383EAC2031BB283EA0C0E8EEA0E1E1C
:10CDC8005FFA8EFEC3F3072282EA1E1242EA0E229F
:10CDD800604482EACE0E84F8D602A4F84CE001F151
:10CDE8001F0011F8013B83EA0E0383EA0313DBB249
:10CDF8001A0982EA1E2242EA032282EAC3031BB20C
:10CE08001FFA83FE8142A4F84CE0EAD183F07C0348
:10CE180083EA0313DBB21A0982EA1E2E8EEA032E76
:10CE28008EEAC30E0FFA8EFE1FFA8EF34FEA132A0C
:10CE38005FFA8EFEA4F84C30DFF8009284F874A0F4
:10CE480004F16E0384F873E004F14E0C0193DCF8EE
:10CE58000C30DCF80000DCF80410DCF80820C846C8
:10CE6800A8E80F00019B0CF1100C9C45C146EED1BF
:10CE7800DCF80000C8F80000DFF8C4819CF8043032
:10CE880089F8043008F1270984F825E384F826A3F3
:10CE980018F8011F3868F5F7C1FEC145F8D194F8B4
:10CEA800C722002A41F0798060492B6808780A2156
:10CEB80084F8C712002801F07581DFF888C10128BD
:10CEC800BCF80010059141F29E85BCF80210029151
:10CED800022801F05F84BCF804100391032801F0D4
:10CEE800B985BCF806100191042801F0AD85052824
:10CEF800BCF8081001F0A3850628BCF80AA001F0C8
:10CF08009A850728BCF80CE001F06A85BCF80E90F9
:10CF180094F8D6220693104680F0300383EA031370
:10CF2800DBB20490424A9DF810C0128884F850C0C1
:10CF3800180980F07A0040EA032080EAC3033D48DC
:10CF4800C2EB022280FB02C01044D217C2EB60225F
:10CF580005988DF82D204FF0000860F30F0803980E
:10CF68004FF0000C60F30F0C00201BB261F30F00B0
:10CF780000216EF30F0183EA031EC3F30723039313
:10CF8800029B63F31F48019BCDF81C8063F31F4C81
:10CF9800039BCDF820C05FFA8EFE6AF31F4069F349
:10CFA8001F4183EA1E134FF0000A09900A918DF879
:10CFB8002CA043EA0E2C0DF11809B9E80F008CEAF1
:10CFC800CE0E0FFA8EFE8EF0C808DFF86CC084F81B
:10CFD80051A088EA08185FFA88F8CEF3072EACE863
:10CFE8000F008EEA181E4EEA082399E8030083EA28
:10CFF800C8080FFA88F383F023024CF8040B82EA7E
:10D008000210C0B2C3F3072282EA1012049B2CF864
:10D01800141942EA0022591C82EAC0004FF0230882
:10D02800162211E0D4510020DC930020903B002010
:10D038000894002003082080D420002080230020AA
:10D048007F230020AC8800204FF0FE0EC82384F810
:10D05800D612A4F84C000CEB020184F8538084F833
:10D068004EE084F84F2084F852301CF8013B4340CE
:10D0780083EA0313DBB21A0982EA102242EA032286
:10D0880082EAC3031BB298B28C45A4F84C00ECD1D9
:10D0980083F0F40383EA0313DBB24FEA131E8EEA2C
:10D0A800102E8EEA032E8EEAC30EA0460FFA8EFECD
:10D0B8001FFA8EF958F84E0FDFF818C4A4F84C90F0
:10D0C8004FEA192A5FFA8EFE84F86AE084F86BA0AA
:10D0D800D8F80410D8F80820D8F80C30ACE80F00BD
:10D0E800D8F81000D8F81410D8F8182004F21D3910
:10D0F800ACE8070004F2FF2884F81DA384F81CE3B9
:10D1080018F8011F3868F5F789FDC145F8D194F87A
:10D11800CEE2BEF1000F40F04A87E64B94F8D6C243
:10D12800B3F90010B3F90220B3F904309FEDE26AB5
:10D1380084F851E007EE103A2B6806938CF06A03E6
:10D1480083EA031306EE901AD9B20B0983F0D503CC
:10D1580043EA012383EAC1031BB283EA0311524263
:10D16800C9B207EE902AC3F3072383EA111343EAEF
:10D178000123F8EEE77AF8EEE66AB8EEC77A83EAB2
:10D18800C1031BB267EE867A66EE866A27EE067AD8
:10D19800002083F0C805CDED087ACDED076A8DED46
:10D1A800097A0A900B900C9085EA05150DF118097B
:10D1B800EDB2C3F30728B9E80F0088EA151848EA62
:10D1C800052888EAC505DFF810832DB2A8E80F0006
:10D1D80085F01E0E99E807008EEA0E13DBB2C5F340
:10D1E800072E8EEA131E4EEA032E88E807008EEA01
:10D1F800C30EA8F110051C20C8214FF005091E23F5
:10D208004FF0FE080CF1010284F8521084F8CE9217
:10D2180084F8533084F84E8084F84F00291884F835
:10D2280050C0A4F84CE084F8D62215F8013B83EAF4
:10D238000E0383EA0313DBB21A0982EA1E2242EACA
:10D24800032282EAC3031BB21FFA83FE8D42A4F8AD
:10D258004CE0EAD183F0270383EA0313DBB21A090F
:10D2680082EA1E2E8EEA032E8EEAC30E0FFA8EFE77
:10D278001FFA8EF34FEA13295FFA8EFEDFF8548205
:10D28800A4F84C3084F8719084F870E004F14E0CE6
:10D2980004F16E0ADCF80000DCF80410DCF8082061
:10D2A800DCF80C3045460FC50CF1100CD445A846E7
:10D2B800F0D1824DBCF80030A8F8003005F1240800
:10D2C80084F822E384F8239315F8011F3868F5F7EA
:10D2D800A5FC4545F8D194F8CF320293002B40F0D5
:10D2E8006186774B1B68052213F0140F84F8CF2250
:10D2F80040F0B686DFED737A94F8D6826D4B724AA9
:10D30800B3F90410B2F90620704D7148CDED087AD2
:10D3180088F0220383EA03135FFA83FE4FEA1E13A1
:10D3280083F05903B2F5FA6F43EA0E2383EACE037A
:10D33800A8BF4FF4FA621BB2B2F57A7F83EA031EE4
:10D34800B8BF4FF47A725FFA8EFE4FF0640CA2F504
:10D358007A72C3F307230CFB02F283EA1E1385FBE0
:10D36800025980FB0150D21743EA0E25C9174FF026
:10D37800000AC2EBA912C1EBA00185EACE050DF1A6
:10D38800180CADF82A20ADF82810CDF818A0CDF863
:10D398001CA0CDF824A02DB285F0C80ECDF804C08D
:10D3A800BCE80F008EEA0E1E5FFA8EFEC5F3072555
:10D3B80085EA1E15DFF82091DCF800C084F850805B
:10D3C80045EA0E25A9E80F0085EACE0212B282F0DE
:10D3D8004A0383EA0313DBB2C2F3072282EA131279
:10D3E80049F810C942EA03224A2082EAC3034FF0EF
:10D3F800140E002508F101084FF0FE0C84F85300C4
:10D40800C82084F8515084F8D682A4F84C304A4693
:10D4180009EB0E0184F84EC084F84FE084F85200FE
:10D428001D4612F8010B684080EA0010C0B20309DB
:10D4380083EA152343EA002383EAC00000B285B2D9
:10D448008A42A4F84C50ECD180F0140080EA001015
:10D45800C0B24FEA101E8EEA152E8EEA002E8EEA12
:10D46800C00E25460FFA8EFE1FFA8EF855F84E0F9D
:10D47800DFF860C0A4F84C804FEA182A5FFA8EFEE5
:10D4880084F869A084F868E06968EB68AA68ACE881
:10D498000F00286969692B8BACE8030004F2FF25AB
:10D4A800ACF80030A84684F81BA384F81AE304F209
:10D4B8001B3A13E0603E002088C3E43A7F23002033
:10D4C800D451002000000000AC880020D34D621029
:10D4D8006766666680230020D420002018F8011FA4
:10D4E8003868F5F79BFBC245F8D1D14BD14A1B7878
:10D4F8001278013B12F00100DBB214BFC0224022B7
:10D50800172B04D8CC490B4493F824300293CB4B07
:10D5180019888B071ABF002342F01002012311F467
:10D52800027F18BF022311F0100F18BF062311F055
:10D53800200F18BF1023002841F07680032194F8AB
:10D54800D6E206938EF0460383EA0313D8B20309A2
:10D5580083F0920343EA002383EAC0031BB283EA01
:10D568000310C0B2C3F3072888EA101848EA002855
:10D5780088EAC0080FFA88F888F0C80C9DF80800F7
:10D588008DF81C008CEA0C1C00235FFA8CFC8DF8CB
:10D598001E200320019A8DF81D30C8F307288DF846
:10D5A8001F108DF8200088EA1C1807CA48EA0C28C2
:10D5B80088EACC0C0FFA8CFC8CEA0C18A9E803005A
:10D5C8005FFA88F8CCF3072181EA181141EA0821AB
:10D5D80081EAC80894F854C089F800200FFA88F244
:10D5E8008CEA020C8CEA0C1C5FFA8CFCC2F3072252
:10D5F80082EA1C1242EA0C2294F8550094F856105C
:10D6080094F8579094F8588084F8533082EACC0202
:10D6180012B2504080EA0010C0B2C2F3072282EA78
:10D62800101242EA002282EAC00212B2514081EA94
:10D638000111C9B2C2F3072282EA111242EA012299
:10D6480082EAC10212B289EA020989EA09195FFA73
:10D6580089F9C2F3072282EA191242EA092282EA08
:10D66800C90212B288EA020888EA08185FFA88F83C
:10D67800C2F3072282EA181242EA082294F859C033
:10D6880094F85A0094F85B1094F85C9084F8513040
:10D6980082EAC80212B28CEA020C8CEA0C1C5FFA0D
:10D6A8008CFCC2F3072282EA1C1242EA0C2282EAAC
:10D6B800CC0212B2504080EA0010C0B2C2F3072276
:10D6C80082EA101242EA002282EAC00212B25140F3
:10D6D80081EA0111C9B2C2F3072282EA111242EAB1
:10D6E800012282EAC10213B289EA030282EA021223
:10D6F800D2B2C3F3072383EA121343EA022383EA6D
:10D70800C2031BB283F0320282EA0212D2B2C3F31E
:10D71800072383EA121343EA022383EAC2031BB2F4
:10D728009AB24FF0FE0CDFF8288184F850E0092007
:10D73800C8210EF1010EDBB284F84EC04FEA122C5C
:10D7480084F84F0084F8521084F8D6E2A4F84C20EC
:10D7580084F85EC084F85D30D8F80000D8F804106A
:10D76800D8F80820B8F80CA008F2B22EAEE80700E6
:10D7780008F2C2288EF80290AEF800A084F810C310
:10D7880084F80F3315F8011F3868F5F747FAA845EC
:10D79800F8D1009BC4F8C032FFF7F5B8DFF8B4A0A1
:10D7A800DFF8B48041201CF06DF9BAF9023088FB2B
:10D7B8000320DB17C3EBA00080B21CF049F9BAF9CB
:10D7C800003088FB0320DB17C3EBA00080B21CF0FD
:10D7D8003FF9BAF9043088FB0320DB17C3EBA0003C
:10D7E80080B21CF035F9164B38681978F5F716FA37
:10D7F80094F8BC3213F0010800F04084114AC4F8D0
:10D80800B8920133DBB2A2FB0312D20802EB820208
:10D81800A3EB420384F8BC32FFF797B80A4B0B49D5
:10D828001868F5F7CBF900232370FFF701B900BF9B
:10D838008C2B0020EB3C00201C530308283E0020C2
:10D84800CC890020CDCCCCCC746A0020B4690020EF
:10D85800CE200020603E00206766666694F8143487
:10D86800C84AC4F8106402EB8302D26B42B30EAD0F
:10D8780004F21B43C44E45F8203D002104F22D4319
:10D888003180079380211523A52784F81A34284668
:10D8980084F8191484F81874904728463188F6F7E4
:10D8A80053FD069DB94804F583616D1A152DA8BF6F
:10D8B80015252A4624F078FEB54A94F814341570D4
:10D8C800B44A013382FB0312A2EBE37202EB420279
:10D8D8009B1A84F81434FFF766B8AF4BAF4AD4F8F4
:10D8E80068112868128893F80BE0AD4B401A4FF482
:10D8F8007A71D7B201FB0EF1120A9F771F75884221
:10D908004FF00007DA775A759F701F7180F05583C2
:10D91800A44AA549DFF8A4E21268DFF89CC20F68A0
:10D928008868DCF80010C4F864618EFB028CD2179A
:10D93800C2EB6C12DFF888C28EFB018E8CFB079855
:10D948008CFB009CC017C0EBAC0002F5FA724FEAE2
:10D95800E17C92B2CCEB6E1CFF1701F5EA4EC7EBE7
:10D96800A8070EF1300E9A76120A0CF1780C4FEADD
:10D978002E2E3031DA764FEA272802121F7783F8E5
:10D988001D8083F8200083F8212083F824C083F8C1
:10D9980023E083F82210FEF755BF844F38680368E8
:10D9A8005B69984700283EF4DCAF386803680121BA
:10D9B8009B6998470222002388F800202370FEF70D
:10D9C800D0BF94F8801194F8813138684A1C01332B
:10D9D80084F8802184F88131F5F720F9FEF794BFA7
:10D9E800734CDFF8E0914FF0000A0BE01B2B00F0BE
:10D9F8004B820D2B00F014824FF0010389F801309F
:10DA0800D8F80000F5F706F9002837D0D8F8000054
:10DA1800F5F7F8F883B27E2B2A6828D099F8012008
:10DA2800002AEDD194F882110029DFD07D2B00F077
:10DA38000B8294F886E1BEF1000F04D080F0200339
:10DA4800DBB284F886214A1CD2B2092A635484F8CE
:10DA5800822100F0ED81082AD2D8B4F88421134439
:10DA680003EB132303F0FF03A4F88431C8E784F819
:10DA780082A184F883A189F801A0C1E794F88731CD
:10DA88002BB1637884F88701302B00F05D8594F81A
:10DA980083213C4BDFF83091DFF830C1DFF830A14B
:10DAA8004FF0010E002A3EF440AF2968C91B012936
:10DAB80000F2B18194F89C82B8F1000F40F0FB812C
:10DAC80094F8B41233F8110010B984F8B4E2E9E715
:10DAD8000131B0F5826F84F8B41200F0E2801ED9EB
:10DAE800B0F5E26F00F0C38034D9B0F5046F00F0F0
:10DAF800CC80B0F5116F00F02781B0F5E46FD1D17B
:10DB08002C4AD76B118A642303FB07F393FBF1F1CB
:10DB18001BF0ECFF002384F88331FEF706BFB0F555
:10DB2800007F00F02B8155D8B0F5807F00F0498147
:10DB3800B0F5887FB6D1D9F800104907B2D51E4B89
:10DB48004FF4887019681BF0D1FF002384F88331E3
:10DB5800FEF7EBBEB0F5C06F00F02381B0F5E06FC3
:10DB6800A0D1144A506B118A642303FB00F34FF4CD
:10DB7800E06093FBF1F11BF0B9FF002384F88331D7
:10DB8800FEF7D3BE1C5303081A690020CC2C0020D2
:10DB9800E12C002056555555346900201C69002099
:10DBA8001C6A00200C94002020690020E02F00202F
:10DBB80080200020083B0020883E00201F85EB5174
:10DBC8006766666625000020D4510020DC9300209B
:10DBD80073690020B0F5047F00F00381B0F5806F11
:10DBE8007FF460AF94F8B5320133DBB2032B00F257
:10DBF800328142F2107184F8B53201FB03F1BE4B59
:10DC08001B88002B40F025810131BC4B1B78D807BD
:10DC1800BB4B1B8848BF0431DA0748BF0A31980755
:10DC280048BF14311A0648BF2831D80548BF2831E3
:10DC38005A0748BF6431180748BFC8319A0548BF1A
:10DC480001F5C871980648BF01F57A71DA0648BF30
:10DC580001F5FA61580648BF01F57A614FF4806012
:10DC68001BF044FF002384F88331FEF75EBEA54A0B
:10DC7800976B118A642303FB07F393FBF1F11BF005
:10DC880035FF84F88381FEF750BE9F4BB3F904102B
:10DC980001EB810149001BF029FF84F88381FEF71D
:10DCA80044BED9F8001011F020087FF4FBAEDBF871
:10DCB8000010090600F132849449097B00293FF4D9
:10DCC800F1AE94F8B612032900F22986DFE801F0D4
:10DCD800322819028E4B1B6859799A79DB7901F140
:10DCE800407101EB022101EB0341002384F8B632B5
:10DCF8004FF482601BF0FAFE002384F88331FEF7AC
:10DD080014BE844B1A68137A507992781B0403EB7B
:10DD1800002313444A1C84F8B62203EB0161E7E7A9
:10DD28007C4B1A68D379107952781B0403EB0023D3
:10DD38001344EFE7774B1A689379D07812781B046D
:10DD480003EB00231344E5E79CF8041000293FF493
:10DD5800A9AE9AF8001000293FF4A4AE6E4B1B88B8
:10DD680003EB83035B004FF4116093FBF1F11BF0AD
:10DD7800BDFE002384F88331FEF7D7BD9CF805105B
:10DD880000293FF48FAE654B65491B6881FB032171
:10DD9800DB17C3EBA1011BF0A9FE84F88381FEF712
:10DDA800C4BD9CF8051000293FF47CAE5B4B4FF4D2
:10DDB800C06099681BF09AFE002384F88331FEF74F
:10DDC800B4BDD9F8001048077FF56CAE554B4FF439
:10DDD800807019681BF08AFE002384F88331FEF7EF
:10DDE800A4BD9CF8041000293FF45CAE9AF800002A
:10DDF80000283FF457AE454B5B7B002B00F01084A6
:10DE0800454B198891FBF0F101EB810149004FF472
:10DE180004701BF06BFE002384F88331FEF785BD88
:10DE28004FF0010284F882212370A4F88411E7E5F9
:10DE3800B4F88421C2F1FF0293427FF4DDAD4FF0C4
:10DE4800010384F88731D7E54FF0010384F8863160
:10DE5800D6E50231D9E6012384F8B53242F21071D1
:10DE6800CDE6F4F779FC304B1A6840F6B833801ADF
:10DE7800984200F2EB802D4F3B793A2B00F0E78275
:10DE880000232370FEF76DBDD8F80000F4F7C2FE3A
:10DE980000287FF4B1AD4FF0010384F88331AFE57A
:10DEA800C4F8743184F86C31214F1BF06DFE94F87E
:10DEB8007831FEF70EBDD4F88C32DFF8789094F8FC
:10DEC800B2224B4500F00484511C94F8B3E2D4F814
:10DED80090C284F8B21202F00F028DF818200DF1EA
:10DEE8001902ACEB0301002940F30D8506A9019145
:10DEF8000DF11E0723E000BF24940020EB3C002016
:10DF0800283E0020083B0020603E002034690020A5
:10DF180078260020843E00201C690020206900200B
:10DF2800676666660C940020482F0020302F00207A
:10DF3800846900200C220020002840F39C800133D3
:10DF4800C4F88C3213F8011C02F8011BBA42ACEB7E
:10DF5800030081EA0E0EEFD384F8B3E200F0D9840F
:10DF6800501CB84282F800E005D20EAB9A1A1B3A50
:10DF7800002126F02EFE019932201BF09BFD4FF068
:10DF88000008002384F89C8284F88331FEF7CDBC16
:10DF9800013B84F8C632FEF782BF013A84F8C722F3
:10DFA800FFF7B5B8013B84F8CF32FFF7F2BB0EF1AB
:10DFB800FF3E84F8CEE2FFF78EB9C64A2968127888
:10DFC800C4F86811013A012A3FF6A2AC10210222D6
:10DFD80099701A719CE4C04AC04B12680793A3F168
:10DFE800240800202121D50003F8240C88F8021009
:10DFF80040F10A83BA490327BA4B1B88580500F138
:10E008000083DA0700F1C38303F00203B64A002B4A
:10E018001CBF03271146B54D3A46284624F0C4FADA
:10E028007B190EA80133A91E40F8203D00225B1A77
:10E038007A5588F801301BF039FEFEF710BD1BF049
:10E0480093FDAB4B01221A70FEF717BCA94AB2F830
:10E05800BE3200210133A2F8BE322170FEF781BC26
:10E06800A54B9FEDA67AD3ED007AF8EEE77A67EE36
:10E07800877AFFF741B984F8B3E271E7994B1B88B7
:10E08800DA0515D4D80600F18D83990600F1378496
:10E098005A0600F17784180700F19684D90700F131
:10E0A800758413F0020F0CBF4FF004084FF00C08F2
:10E0B800934B944A1B78D27803F001030AB143F0DA
:10E0C8000203532000931BF0DDFC8F4A128802EBF9
:10E0D800820202EB8202900080B21BF0B9FC0020A1
:10E0E8001BF0B6FC894A8A4912883868C2EBC2120A
:10E0F800520081FB023111444FEAE27ACAEB612AED
:10E108005FFA8AFA5146F4F789FD824B38681A7823
:10E11800009B48EA03087F4B8AEA020A002183F839
:10E1280000A0F4F77BFD41463868F4F777FD794B9A
:10E13800784A1B78386888EA0303DBB219461370FB
:10E14800F4F76CFD94F8BC32002B7FF457AB4F20EA
:10E158001BF098FC1EF058FB1EF056FB1EF054FBFB
:10E1680001213868F4F75AFD6B4A6A4B92F800802F
:10E178001B78684A386808F00108414683F00103B3
:10E188001370F4F74BFD634B38681B7888EA030873
:10E19800604B414683F80080F4F740FD94F8BC32A8
:10E1A800FFF72CBB864682460146019003900290F9
:10E1B80005908146FEF7ACBE484B534907930EAF16
:10E1C800A3F1210047F8200D4FF0080E4FF000088A
:10E1D8000A2003F822EC03F8230C03F8248C3846B1
:10E1E8000988F6F78BF84D4B4D491B6881FB0321D5
:10E1F800DB17C3EBA101384689B2F6F77FF8494B24
:10E20800B3F8069017F05AFF069B5A1C069283F83B
:10E218000080069B4FEA1922591C06911A70069B2A
:10E228005A1C069283F80090069B5A1C0692187096
:10E2380038461BF03BFDFEF70FBCDFF8F0809FED82
:10E248003A8AB8F90230254A079207EE903AF8EE72
:10E25800E77A0EAF67EE887AA2F12403FDEEE77A3B
:10E26800A2F12101002047F8201D02F8240C082201
:10E27800CDED007A5A701E229A70BDF8001038460B
:10E28800F6F73CF8B8F9003007EE903AF8EEE77A7E
:10E29800384667EE887AFDEEE77ACDED007ABDF86C
:10E2A8000010F6F72BF8B8F9043007EE903AF8EEBC
:10E2B800E77A384667EE887AFDEEE77ACDED007AA0
:10E2C800BDF80010F6F71AF838461BF0EFFCFEF719
:10E2D800C0BB00BF189400201C940020B469002023
:10E2E8001C810308283E00202C8103089369002024
:10E2F80025000020802000200C9400200AD7233C11
:10E30800EB3C0020303E00201C69002008940020CF
:10E3180003082080CC890020D893002020690020A1
:10E3280067666666DC93002058A08B41603E00203B
:10E3380002201BF0A9FCFF201BF08EFA0378FF2BAC
:10E3480000F0CB8290F901004FEAE0795FFA89F991
:10E35800C0B21BF06FFC48461BF06CFC03201BF09E
:10E3680093FCFF201BF078FA0378DFF8DC93FF2B8F
:10E378001BBFB0F908A05FFA8AF74FF0000ACAF38A
:10E38800072A38461BF056FC50461BF053FC99F8F8
:10E398000430002B40F009820DF118094946DD4888
:10E3A8001BF00CFC13201BF06FFCBDF91870F8B2C1
:10E3B8001BF040FCC7F307201BF03CFC1B201BF0A4
:10E3C80063FCBDF91A70F8B21BF034FCC7F30720E0
:10E3D8001BF030FC23201BF057FC4E201BF02AFCBE
:10E3E80000201BF027FC4946CA481BF0E7FB122017
:10E3F8001BF04AFCBDF91870F8B21BF01BFCC7F300
:10E4080007201BF017FC1A201BF03EFCBDF91A7000
:10E41800F8B21BF00FFCC7F307201BF00BFC2220FF
:10E428001BF032FC45201BF005FC00201BF002FC11
:10E438005E21D8F80000F4F7F1FB94F86031FEF79C
:10E44800D7BBC4F8706183F80080FEF716BABB78B2
:10E45800DBB103F1FF3C5FFA8CFC0CF1010CBC440E
:10E46800BE4600221EF8013B534083EA0313DBB289
:10E47800120AD90042EA0322F44581EA131382EA18
:10E488000302EFD1002A7FF4FBACA34BDFF8BCC238
:10E49800D3F800E0A14BA2491B68DEF83080A14AFE
:10E4A800CCF83830A04B0988CCF81810CCF86800A4
:10E4B8001168B3F8BE029268CCF82810CCF848204E
:10E4C800CCF85800B8F1000F00F06C82D8F804308E
:10E4D800DEF840108B423BBFDEF80C205B1A5B1A5B
:10E4E8009B18002B7EF436AADEF80030DFF8608235
:10E4F8009B697046022198470423F87888F8003011
:10E5080023F042FE03232370FEF726BA022138685F
:10E51800F4F774FB94F87831FEF7DBB91023042282
:10E52800184606A98DF81A808DF81B808DF81C8076
:10E538008DF81D808DF818308DF819201BF0BAFA67
:10E5480084F88381FEF7F1B9A3785A09012A40F0CB
:10E55800B28103F00F0C13F0100300F0C081DFF854
:10E56800F481E37894F804E0A4F8AA0208EB030124
:10E578008EEA030084F888214346C4F8A082C4F8D0
:10E58800A412A8F1070284F8B002A4F8A8E294F84B
:10E59800B002DFF8C48186460CE012F8011BC4F80B
:10E5A800A002424581EA0E0E197007D2D4F8A412CF
:10E5B800D4F8A032994203F10100EED1424584F823
:10E5C800B0E200F03182127894F8B0329A4200F04A
:10E5D800B181564BC4F88C3200220133B4F8A8122A
:10E5E800C4F8903284F8882101234FF6F672A4F813
:10E5F800941284F88C3184F89C32A4F89622FFF7A0
:10E6080046BA03274A4906E5DBF80030494A4A4931
:10E6180003F48003834216BF114604270327EBE463
:10E628003F4B1988FFF7F0BB4449C97800290CBF54
:10E6380004210521FEF783BFDFF8E0A010201BF0BE
:10E6480023FB3F4ADAF8003082FB0329DB17C3EBD0
:10E6580069195FFA89F01BF0EDFAC9F307201BF07E
:10E66800E9FA21201BF010FBDAF80020344B83FB79
:10E67800023AD3176421C3EB6A1301FB1323002B5F
:10E68800D8BF5B421BB2D8B21BF0D4FA00201BF0F3
:10E69800D1FAFEF782BA012238681A70F4F7B2FA92
:10E6A80080463868F4F7AEFA18F07F0F7EF4E5A8D4
:10E6B8008E287EF4E2A894F86C31002B7EF4F9A839
:10E6C800204BC4F874312D2384F87831FEF7DCB878
:10E6D800B4F99612D4F890C294F894E2501C02F05F
:10E6E8000F0242F010020029B8BF42F020028DF854
:10E6F8001820ACEB090282EA0E0E5FFA8EFE8DF846
:10E70800192084F8B20284F8B3E20DF11A02FFF777
:10E71800E8BB00BF80969800E02F00200C940020F2
:10E728001C69002020690020802000200C22002085
:10E73800208103081C81030814810308303E00204F
:10E748001F85EB511C6A0020DC93002094010020F7
:10E75800050200208C20002088200020C1495A7919
:10E768000B8803EB830303EB83034FEA830A1FFA47
:10E778008AFA002A00F05C81BB4B1B681BB202932B
:10E7880017F09CFC029B019A40B2FEF7B3BAB74956
:10E79800042740E496469246114601920392914618
:10E7A800FEF7B6BB4FF0340882E4DFF8D8A29AF837
:10E7B8000020002A3FF4F0ADB4F86271A94B009232
:10E7C8001B883F016421BFB201FB03235100B3FB47
:10E7D800F1F347EA0327BFB2C3F303231F4306201D
:10E7E8001BF052FAF8B21BF025FA380A1BF022FA8D
:10E7F800B4F862319B4A9E491788009A01339BB24C
:10E8080093FBF2F002FB1033487AA4F86231012836
:10E8180000F0EF804B7B6E2202FB07F7152297FB77
:10E82800F2F7002B40F0DF803A201BF02DFABFB240
:10E838004FF0640AB7FBFAF293B2D8B20192009390
:10E848001BF0F8F9009B180A1BF0F4F93B201BF0A9
:10E858001BFA019A0AFB127080B20A23053090FB5A
:10E86800F3F0C0B21BF0E6F900201BF0E3F9DFF883
:10E87800F8A128201BF008FA0A23DAF8007097FBA1
:10E88800F3F7F8B21BF0D6F9C7F307201BF0D2F95B
:10E8980004201BF0F9F9B9F80630002B7AD1DAF820
:10E8A800087087F31007F8B21BF0C4F9C7F3072004
:10E8B8001BF0C0F970E56F4B6F4AC4F88C32591CD5
:10E8C800012384F8880184F88C01C4F89012C4F8F4
:10E8D800942284F89C32FFF7DAB8484639E594F870
:10E8E8008821002A3FF4D3A894F8B122013202F01B
:10E8F8000F02624562D084F88831FFF7C8B84FF03C
:10E908002408FFF7D5BB06AB01930DF11E07FFF7EF
:10E9180027BB019932201BF0CDF8FFF732BB4B1C07
:10E92800DBB2042B84F8B6324FEA01617FF4E0A928
:10E93800FFF7DBB9514BD4F8A022C4F8A4224FF05A
:10E94800000E03F52072114603F5C079C4F8902231
:10E9580003F525707246C4F8A032C4F894E2C4F8EE
:10E968008C9284F888E1F6F78FFD013054D0D4F802
:10E978008C32C4F890320123C4F88C9284F89C320B
:10E98800FFF785B84FF01008FFF792BB4FF0080863
:10E99800FFF78EBB17F092FB1BF04CF900201BF021
:10E9A80049F9F9E4DEF81C10DEF8203099423BBF43
:10E9B800DEF80C205218CB1AD31A92E5D4F8A41218
:10E9C800D4F8A0322E4AE2E54FF02008FFF770BBDA
:10E9D800254B9246B3F9003064200A46FEF78AB9FF
:10E9E8009146FEF795BABFB29AF8003097FBF3F755
:10E9F8001AE739201BF048F9F8B21BF01BF9380A5E
:10EA08001BF018F933E79646924611460192039295
:10EA180002929146FEF77CBAD4F88C320222591C35
:10EA2800C4F88C121A70A2E784F8B1C2FFF72FB8A5
:10EA38004FF0FF33A2E696469146FEF769BA96462E
:10EA480092469146FEF764BA96469246114691461A
:10EA5800FEF75EBA96469246114601929146FEF737
:10EA680057BA00BF1C6900202069002024810308D0
:10EA7800346900200C2200200000F6FF8C200020C2
:10EA880083200020736900202DE9F04FDFF808B1DA
:10EA98002DED0C8B9BF8003099B0012B039001F001
:10EAA8002C82DFF8F8A09AF80021002A41F034827D
:10EAB800072B01F03B824FF00009344C6368204675
:10EAC800984700286ED0B4F8A860002284F849203E
:10EAD800002E40F09182B4F92450E16AB4F926007E
:10EAE800226BB4F92830691AA16329490091821A66
:10EAF800606BE2630D461B1A94F84A10236404F114
:10EB0800380009F087FB2B6813F0005302F0C68128
:10EB1800D4ED0F5AD4ED0E7A1E4A9AED416ADAED19
:10EB2800426A9AED437ADAF810311268B8EEE58A4B
:10EB3800D4ED105AF8EEE77AF8EEE58A013377EE6D
:10EB4800867A38EE268A78EE878A9342CAED417A29
:10EB58008AED428ACAED438ACAF8103101F0A486C8
:10EB68009BF80060142E02F0AA870023DAF81851E7
:10EB78000193062D02F25482DFE815F0DB14C71466
:10EB8800F21122171A16B1169E1500BF2444002050
:10EB9800686C0020D851002085680020B42400202B
:10EBA800DDF804909BF80080B8F1070F00F0DB82D5
:10EBB8009AF828310593002B40F0E182CD4B5B7920
:10EBC800002B40F0148201239BF800208AF828319A
:10EBD800072A02F07F8200230793C74BDAED4C9A8D
:10EBE80093ED007AC54AC64B1268C64FDAED4B8AD8
:10EBF800DFF89493DFEDC4AA9FEDC49A9FEDC4BAE1
:10EC0800DFEDC4CA9FEDC4AADFEDC4BADFF87C8388
:10EC1800C34E0493F7EE007A37EEE98A002428EE13
:10EC2800078A0292B4EEE78AF1EE10FA88BFB0EED6
:10EC3800678A019325460097BA4B2344D3ED007A9F
:10EC4800B94BF5EE407A2344F1EE10FA93ED00CA81
:10EC580017D0B64B234493ED007A7CEE476AB0EEAA
:10EC6800E66AF4EEC67AF1EE10FA08D5F5EEC06A57
:10EC7800F1EE10FACCBF37EE87CA37EE67CA83EDDC
:10EC880000CAAB4B1F88BB0700F08182022D04F03D
:10EC980028850299A74B91F8322007EE102A91F89F
:10ECA80031202344D3ED006A5342B8EEC77A07EE09
:10ECB800903A27EE267AF8EEE77AB4EEE77AF1EEA4
:10ECC80010FA0AD407EE902AF8EE677AF4EEC77ABB
:10ECD800F1EE10FA88BFF0EE477A974B0693974A01
:10ECE80003EB450332F91510B3F90A30C81A07EED9
:10ECF800100AB8EEC77AF807E7EE497A40F1988229
:10ED08008F4F97ED00CA27EE8CCA9AF86471E7B165
:10ED18008B4FDAF8680197ED007A8A4F5B1A07EE95
:10ED2800903A039B396827EE097AF8EEE77A1F1ABA
:10ED38008F4227EE87CA01F3AF81F7EE007AF4EE2F
:10ED4800E79AF1EE10FA01F173817F4B2344D3ED7A
:10ED5800007A019BD3ED01DA009B68EEA77A3CEEBE
:10ED68006DDA67EE8D7AC3ED007A784BD9ED006ADB
:10ED780093ED007A764BD6ED007A26EE877A234417
:10ED880067EE086A93ED007A26EE877AF0EE676AF6
:10ED9800E7EE0D6AB0EE667A9AED4C6AF7EE006A15
:10EDA800B4EEE66AF1EE10FAACBF0123002343B1DA
:10EDB800F0EEE77AF0EEC76AF4EEE76AF1EE10FAE1
:10EDC80001D586ED007A022D04F08484614A624BF5
:10EDD80052F825001B68B0EE6D0A98475F4A604BF1
:10EDE80052F825001B689847029B93F83A30632B2A
:10EDF80004D84F4B1B88002B01F06081F0EE6C7A31
:10EE0800584B99ED007A37EEC00A2344D3ED007AC7
:10EE180083ED000A029B30EE670A93F8482080EEE3
:10EE280007CADAB1F7EE007AF4EEE79AF1EE10FAD3
:10EE380014DB4D4BD3ED007AB0EECC7AB4EEE77A22
:10EE4800F1EE10FA0ADD494BD3ED007AB0EECDDAD7
:10EE5800B4EEE7DAF1EE10FA01F38E81444B9AF83A
:10EE680074212344D3ED007A68EEA77A27EE8CCA82
:10EE780088ED00CA32B9009BC6ED00CAC3ED00CACE
:10EE8800C8ED00CA009B04330093019B043404338B
:10EE98000C2C05F1010508F1040806F1040601939C
:10EEA8007FF4CAAE9BF80030072B02F0CD80012B0F
:10EEB80002F00081002304932E4B00931A460F4B57
:10EEC80012681B680192114693F82F2011F48053A1
:10EED800069300F05182284B02931B78274807902D
:10EEE80013F0010F264B0393198B264B90ED037AF1
:10EEF8004EE000BF10440020888C0020843E002093
:10EF0800484C00209428002000009642CDCCCC3DEF
:10EF1800AE47813F000000000000C84200003443B3
:10EF2800A02800207C8C0020E8250020F425002063
:10EF3800283E00200026002018290020603E0020DE
:10EF4800648C00208C8C0020388C00202800002045
:10EF5800448C002000320020FC3100206432002064
:10EF680060320020202600209C8C0020988C0020F5
:10EF7800508C0020686C0020EB3C00207469002055
:10EF8800805E0020DC370020348C0020AC28002074
:10EF9800DB8808BFAAF87C11C81A07EE900AF8EEB9
:10EFA800E77AB4EEE77AF1EE10FA42F26780CC180D
:10EFB80006EE904AF8EEE66AB4EEE67AF1EE10FA5A
:10EFC80081F23B84BAF87C31984283F24681D54B72
:10EFD800D54993ED004AD1ED004AD44BCAED604AB9
:10EFE8008AED614AD3ED006ADFEDD17AE0E1D14BD9
:10EFF8001B78013BDBB2E7E5CF49D04B4978049356
:10F0080000911B68CE4F9BF80080B7F906004FF4BB
:10F018007A71B1FBF3F3C3EB431503EB8503DD0012
:10F02800ADB2AE4202F02F86E16FB4F924E0236E50
:10F038004A1C07EE90EA7344012AE2672366F8EE59
:10F04800E77A02F02A86D4ED1B5AD4ED1D6A07EE42
:10F05800102A37EEE56AB8EEC75A012E86EE057A11
:10F0680037EE257A77EEC77A84ED1C7AE6EE276AC2
:10F0780084ED1B7AF0EE667AC4ED1E6AC4ED1D6A53
:10F0880003F04A81D4F89010B4F926E0636E4A1C64
:10F0980007EE90EA7344012AC4F890206366F8EEFC
:10F0A800E77A02F01286D4ED205AD4ED226A07EEF0
:10F0B800102A37EEE56AB8EEC75A012E86EE057AB1
:10F0C80037EE257A77EEC77A84ED217AE6EE276A5D
:10F0D80084ED207AF0EE667AC4ED236AC4ED226AE4
:10F0E80003F03C81D4F8A410B4F928E0A36E4A1CBC
:10F0F80007EE90EA7344012AC4F8A420A366F8EE48
:10F10800E77A02F0FB85D4ED255AD4ED276A07EE9D
:10F11800102A37EEE56AB8EEC75A012E86EE057A50
:10F1280037EE257A77EEC77A84ED267AE6EE276AF7
:10F1380084ED257AF0EE667AC4ED286AC4ED276A74
:10F1480003F02E81F880B4F8A8309BF80080013BCA
:10F15800A4F8A83004990023B8F1070F4B608B601E
:10F16800CB607FF425ADF3F7F7FA754F9AF828319D
:10F178000593A0EB09003880002B3FF41FAD013B3D
:10F188008AF8283119B0BDEC0C8BBDE8F08F9AF8DD
:10F19800643163B1022D04F0A7826A4B06936A4A70
:10F1A80003EB450332F91510B3F90A30B0E5674BA4
:10F1B800234493ED000A019BD3ED01DA009B28EE6E
:10F1C800800A3CEE6DDA022D20EE0D0A83ED000A6E
:10F1D8007FF4CBAD5E4A5F4B10681B6898475E4B67
:10F1E800D9ED006A93ED007A5C4BD6ED007A1A7877
:10F1F8005B4B83ED020A5B4B26EE877A234427EEAE
:10F20800087A93ED006A27EE067AF0EE676AE7EE71
:10F218000D6A012AB0EE667A02D0192A7FF4BCADD5
:10F22800B4EEEADAF1EE10FACCBF01230023BEE512
:10F23800DAED566A9AED577AB2F900E0B2F902703F
:10F24800B4EEE67AF1EE10FA8EEAEE7087EAE77C21
:10F258004CBFB7EE007AF7EE006AA0EBEE70ACEBAD
:10F26800E77C4CBF77EE665A76EEC75A604540F3A6
:10F278004587BEF1000FD6BFCEF1000007EE10EAB9
:10F2880007EE100A384FB8EEC77A3F7827EE097AAA
:10F29800002F00F04387354F97ED005AB5EEC05A5E
:10F2A800F1EE10FA41F35886314FD7ED004AF5EEEA
:10F2B800C04AF1EE10FA41F34F8634EEC77AB7EE42
:10F2C800006AC7EE246A75EEC65AF4EEC66A65EEA1
:10F2D8008A5AF1EE10FA85EE857A88BFF0EE466A12
:10F2E800F5EEC06AF1EE10FA37EE067AB8BFF0EE26
:10F2F8006C6A66EE876AF4EEC66AF1EE10FA88BFA9
:10F30800F0EE466AF5EEC06AF1EE10FAB8BFF0EE1C
:10F318006C6A184F97ED007A67EE877AA7EEA6CA4F
:10F32800F3E400BFD4370020D0370020EC370020AA
:10F3380000000000308C002010440020484C0020C1
:10F348008868002018290020603E0020388C0020A2
:10F35800C4360020D8360020280000202C8C00203D
:10F3680094280020448C0020708C00206C8C002095
:10F37800748C0020688C0020E24B03935B8BE2497D
:10F38800079107EE903AE14B91ED037AE04993ED4E
:10F39800004AE04BD1ED004AD3ED006ADE4B8AED1E
:10F3A800614AF8EEE77A029377EE677ACAED604A27
:10F3B800C7EEA62AD949DA4B91ED008AD949DFED83
:10F3C800DA6A91ED005AD9499FEDD96AD1ED005A10
:10F3D80093ED007AF7EE007AF4EEE72A38EE058A24
:10F3E800F1EE10FA88BFF0EE672A38EE258AF4EEBF
:10F3F800E62AF1EE10FA28EE066AB8BFF0EE662AA1
:10F40800F1EE476A34EEC43AB4EEE66AF1EE10FA69
:10F41800CAED622A8AED643A00F16B85B4EEC76AD8
:10F42800F1EE10FA88BFB0EE476ABC4BDFEDC07A48
:10F43800D3ED018ABB4B93ED015ABC4B78EE858A1C
:10F44800D3ED015A78EEA58A68EEA77AF4EEE76A5A
:10F45800F1EE10FA08DCB4EEE77AF1EE10FA8CBFA0
:10F46800F0EE676AF0EE476AAC4BDFEDB17A93EDE8
:10F47800029AAC4BD3ED025AAE4B39EE259A93ED76
:10F48800007A69EE277AF1EE475AF4EEE57AF1EE62
:10F4980010FA08D4F4EEC77AF1EE10FA8CBFF0EE49
:10F4A800475AF0EE675A002A41F08982F7EE007A4F
:10F4B800A14B5A789AF89431002AA04AFFEE003AF4
:10F4C800B7EE007A127814BFB0EE472AB0EE632A7E
:10F4D800002B14BFB0EE635AB0EE475A002A02F070
:10F4E8005B84F4EEC77AF1EE10FA65EE825A944B1B
:10F4F80041F3128393ED027A93ED011AD3ED031AC7
:10F508009FED892A26EE877A67EE853AA6EE017A7C
:10F51800A5EEA17A27EE237AB4EEC27AF1EE10FABC
:10F52800B4BFF0EE427AF0EE477A8DED0C7A88BFE0
:10F53800B0EE427A012A00F0BE8193ED065AD3ED6F
:10F54800051A93ED072A26EE855AA6EE215AA5EE4E
:10F55800825A25EE235AB4EEC57AF1EE10FAF4EE8B
:10F56800C57A8CBFB0EE452AB0EE472AF1EE10FA04
:10F5780058BFB0EE427AB8BFF0EE457A022A8DED58
:10F588000D5A00F0988193ED0A5AD3ED091A93EDBC
:10F598000B2A26EE855AA6EE215AA5EE825A25EEAA
:10F5A800235AB4EEC57AF1EE10FAF4EEC57A8CBFA0
:10F5B800B0EE452AB0EE472AF1EE10FA58BFB0EE89
:10F5C800427AB8BFF0EE457A032A8DED0E5A00F064
:10F5D800728193ED0E5AD3ED0D1A93ED0F2A26EE94
:10F5E800855AA6EE215AA5EE825A25EE235AB4EE84
:10F5F800C57AF1EE10FAF4EEC57A8CBFB0EE452A62
:10F60800B0EE472AF1EE10FA58BFB0EE427AB8BF12
:10F61800F0EE457A042A8DED0F5A00F04C8193EDF7
:10F62800125AD3ED111A93ED132A26EE855AA6EE37
:10F63800215AA5EE825A25EE235AB4EEC57AF1EE88
:10F6480010FAF4EEC57A8CBFB0EE452AB0EE472A20
:10F65800F1EE10FA58BFB0EE427AB8BFF0EE457A34
:10F66800052A8DED105A00F0268193ED165AD3ED38
:10F67800151A93ED172A26EE855AA6EE215AA5EEFD
:10F68800825A25EE235AB4EEC57AF1EE10FAF4EE5A
:10F69800C57A8CBFB0EE452AB0EE472AF1EE10FAD3
:10F6A80058BFB0EE427AB8BFF0EE457A062A8DED23
:10F6B800115A00F0008193ED1A5AD3ED191A93EDFF
:10F6C8001B2A26EE855AA6EE215AA5EE825A25EE69
:10F6D800235AB4EEC57AF1EE10FAF4EEC57A8CBF6F
:10F6E800B0EE452AB0EE472AF1EE10FA58BFB0EE58
:10F6F800427AB8BFF0EE457A072A8DED125A00F02B
:10F70800DA801FE0805E002074690020DC29002078
:10F71800D0370020E4370020EB3C0020942800205C
:10F72800A08C0020A028002000000000AC280020A9
:10F738006F12833AA48C00208C2B0020756800205F
:10F748001037002093ED1E5AD3ED1D1A93ED1F2A92
:10F7580026EE855AA6EE215AA5EE825A25EE235AA0
:10F76800B4EEC57AF1EE10FAF4EEC57A8CBFB0EEBD
:10F77800452AB0EE472AF1EE10FA58BFB0EE427AA9
:10F78800B8BFF0EE457A082A8DED135A00F0938041
:10F7980093ED225AD3ED211A93ED232A26EE855AAA
:10F7A800A6EE215AA5EE825A25EE235AB4EEC57A62
:10F7B800F1EE10FAF4EEC57A8CBFB0EE452AB0EE41
:10F7C800472AF1EE10FA58BFB0EE427AB8BFF0EE11
:10F7D800457A092A8DED145A6DD093ED265AD3ED4A
:10F7E800251A93ED272A26EE855AA6EE215AA5EE6C
:10F7F800825A25EE235AB4EEC57AF1EE10FAF4EEE9
:10F80800C57A8CBFB0EE452AB0EE472AF1EE10FA61
:10F8180058BFB0EE427AB8BFF0EE457A0A2A8DEDAD
:10F82800155A48D093ED2A5AD3ED291A93ED2B2A6D
:10F8380026EE855AA6EE215AA5EE825A25EE235ABF
:10F84800B4EEC57AF1EE10FAF4EEC57A8CBFB0EEDC
:10F85800452AB0EE472AF1EE10FA8DED165A58BF38
:10F86800B0EE427AA8BFB0EE675A0B2A02F0F184D4
:10F87800D3ED2E7AD3ED2D1A93ED2F2A66EEA77AC3
:10F88800E1EE867AE2EE257A67EEA37AF4EEC77A9D
:10F89800F1EE10FAF4EEC57A8CBFF0EE476AF0EE9E
:10F8A800676AF1EE10FACDED177A98BFB0EE667A76
:10F8B800B8BFF0EE457A77EEC77AF7EE006AF4EE55
:10F8C800E67AF1EE10FACAED4C7A42F3B28486EE8B
:10F8D800A77A012ADDED0C7A67EE877ACDED0C7AEE
:10F8E80055D0DDED0D7A67EE877A022ACDED0D7AD7
:10F8F8004DD0DDED0E7A67EE877A032ACDED0E7ACC
:10F9080045D0DDED0F7A67EE877A042ACDED0F7AC0
:10F918003DD0DDED107A67EE877A052ACDED107AB5
:10F9280035D0DDED117A67EE877A062ACDED117AAA
:10F938002DD0DDED127A67EE877A072ACDED127A9F
:10F9480025D0DDED137A67EE877A082ACDED137A94
:10F958001DD0DDED147A67EE877A092ACDED147A89
:10F9680015D0DDED157A67EE877A0A2ACDED157A7E
:10F978000DD0DDED167A67EE877A0B2ACDED167A73
:10F9880005D0DDED177A27EE877A8DED177AE14BF2
:10F99800196811F0805100F0AC834FF07C53CAF81D
:10F9A8008831002A02F0F281029BDB4E1F78DB4C83
:10F9B800DB48DC4DD6ED005A9AF88C31039EE4788A
:10F9C8000078B5F90650DAED626A768B07F0010C1B
:10F9D800019F07F0100E07F48007002B40F0AB8260
:10F9E800BEF1000F00F0AE85BCF1000F42F07E833F
:10F9F800002C42F05A84CC4BDDED0C7A93ED007A62
:10FA0800CA48E7EE267ABDEEE47A17EE101AB0EE91
:10FA1800447AA3EE277A0D46F0EE477AFDEEE77AB0
:10FA2800BDEEC47A17EE906A17EE104AB142A8BF2D
:10FA38003546B442C8BF254607EE905AF8EEE77A35
:10FA4800012AC0ED007A00F04D8193ED047ADDEDD6
:10FA58000D7AE7EE267AB0EE447AA3EE277AFDEE29
:10FA6800C77A17EE906A17EE905A8E42A8BF0D46D5
:10FA7800A642B8BF254607EE905AF8EEE77A022A62
:10FA8800C0ED017A00F02E8193ED087ADDED0E7A53
:10FA9800E7EE267AB0EE447AA3EE277AFDEEC77A2F
:10FAA80017EE906A17EE905A8E42A8BF0D46A642EE
:10FAB800B8BF254607EE905AF8EEE77A032AC0ED5C
:10FAC800027A00F00F8193ED0C7ADDED0F7AE7EE04
:10FAD800267AB0EE447AA3EE277AFDEEC77A17EEBF
:10FAE800906A17EE905A8E42A8BF0D46A642B8BF3C
:10FAF800254607EE905AF8EEE77A042AC0ED037A15
:10FB080000F0F08093ED107ADDED107AE7EE267ABA
:10FB1800B0EE447AA3EE277AFDEEC77A17EE906A24
:10FB280017EE905A8E42A8BF0D46A642B8BF25468A
:10FB380007EE905AF8EEE77A052AC0ED047A00F04D
:10FB4800D18093ED147ADDED117AE7EE267AB0EEE6
:10FB5800447AA3EE277AFDEEC77A17EE906A17EE7D
:10FB6800905A8E42A8BF0D46A642B8BF254607EE5A
:10FB7800905AF8EEE77A062AC0ED057A00F0B280CE
:10FB880093ED187ADDED127AE7EE267AB0EE447A34
:10FB9800A3EE277AFDEEC77A17EE906A17EE905A11
:10FBA8008E42A8BF0D46A642B8BF254607EE905A1A
:10FBB800F8EEE77A072AC0ED067A00F0938093ED15
:10FBC8001C7ADDED137AE7EE267AB0EE447AA3EEDE
:10FBD800277AFDEEC77A17EE906A17EE905A8E4292
:10FBE800A8BF0D46A642B8BF254607EE905AF8EEC4
:10FBF800E77A082AC0ED077A74D093ED207ADDED14
:10FC0800147AE7EE267AB0EE447AA3EE277AFDEE70
:10FC1800C77A17EE906A17EE905A8E42A8BF0D4623
:10FC2800A642B8BF254607EE905AF8EEE77A092AA9
:10FC3800C0ED087A56D093ED247ADDED157AE7EE1B
:10FC4800267AB0EE447AA3EE277AFDEEC77A17EE4D
:10FC5800906A17EE905A8E42A8BF0D46A642B8BFCA
:10FC6800254607EE905AF8EEE77A0A2AC0ED097A97
:10FC780038D093ED287ADDED167AE7EE267AB0EEE5
:10FC8800447AA3EE277AFDEEC77A17EE906A17EE4C
:10FC9800905A8E42A8BF0D46A642B8BF254607EE29
:10FCA800905AF8EEE77A0B2AC0ED0A7A1AD093ED4B
:10FCB8002C7ADDED177AE6EE877AA3EE274AFDEE79
:10FCC800C47A17EE903A9942A8BF19469C42D8BF09
:10FCD8000C4607EE904AF8EEE77AC0ED0B7A002A58
:10FCE80000F0F98392001249104822F05DFC114B94
:10FCF8001B68002B00F0F4830F4B1B78192B22D8BC
:10FD080001220E4902FA03F31940002942F05483F4
:10FD180016E000BF1C940020DC360020303E002096
:10FD2800A8590020AC88002010370020E8280020BF
:10FD3800E0360020288C00202C8C00203241300333
:10FD48001E0301F1AE86AD4DAD4E019B9C061BD541
:10FD5800F37AFF2B04D0AB4A12789A4201F29C86C0
:10FD6800B6F90870F37D2F80FF2B04D0A54A1278CE
:10FD78009A4201F28C86B6F914406C80082004F08F
:10FD8800D1FE002841F0A083B6F90600B5F900E0DD
:10FD9800B5F90270B6F91210B6F91E20B5F904408B
:10FDA800B6F90430B5F906C07045A8BF7046B94227
:10FDB800A8BF3946A242A8BF22469E45A8BF03460F
:10FDC8002B80B6F91030B5F90800BB42C8BF1946F8
:10FDD800B6F92A306980B6F91C10B6F93470634553
:10FDE800A8BF6346A142CCBF0C461446B6F93620DC
:10FDF800AC80B6F92840B5F90A108242A8BF02467D
:10FE0800A445ACBF9C46A446B6F94230B5F90C40AF
:10FE1800A5F806C08B42A8BF0B468742CCBF384620
:10FE28001046B6F94E202881B6F94000B5F90E7093
:10FE3800A242A8BF22468842C8BF0346B6F95A0064
:10FE4800B6F94C106B81B842B6F958306E4EA8BF5F
:10FE580038469F42A8BF0346A142D8BF1146A98190
:10FE6800EB81B38923B3694FDFF8B891DFF890814C
:10FE780007F11004B7F9023000EE103A4846B8EE20
:10FE8800C00AF0F751FD22F097FDB8F90430B8F92F
:10FE9800062000B2984209F12C0908F10C0803DB8E
:10FEA80082421346A8BF034627F8023FA742E1D182
:10FEB800574B1B78013B182B00F2C485DFE813F081
:10FEC800B005C205C205F00AC205C205C2051F0E6B
:10FED800C205C205C205C205C2055F0EC205C2053C
:10FEE800C205C2050E0EF00A500EC205C2055F0E0D
:10FEF800B005B0EE666AFFF798BA464BDFF828A15E
:10FF08001968454A454F9AF80031C96912883980FD
:10FF18007A80002B3EF4CFADF7F730FC00238AF847
:10FF280000319BF80030072B7EF4C5ADF2F714FCC6
:10FF38008146FEF7C2BDBEF1000F00F04B81BCF157
:10FF4800000F42F02181002841F03A82FDEEC47A88
:10FF58000DF1300E17EE906AFDEEE47A0EEB820397
:10FF680017EE907AFDEEE57A2D48DFF8C090CDF8CF
:10FF780024A017EE905AB1EE436A84F001084FFAB4
:10FF880084FC08929A46034693ED007AFEEC017AC7
:10FF9800E7EE267A3A461030B0EE647AA6EE277A73
:10FFA800FDEEC77A17EE903A9F42A8BF1A469D42C7
:10FFB800CCBF002104F00101002914BF11462946D5
:10FFC8009E42CCBF002308F0010307EE901A002BD5
:10FFD80014BF13463346B8EEE77A07EE903AF8EEC8
:10FFE800E77ABCF1000F18BFF0EE477AD645E9EC86
:08FFF800017AC8D1089ADDF876
:020000040801F1
:1000000024A070E6D82800200C8D0020903B002012
:1000100080570020D62800202C8C0020B06A0020B9
:10002000BE2700208868002010370020E4890020C7
:10003000B4240020E8280020069BB2F90070B3F930
:100040000A305A49F81A096880EAE073A3EBE073B2
:100050008B42BEF67EAEB2F90230069AB2F90C209F
:100060009A1A82EAE273A3EBE27399427EF771AEC9
:1000700004994F4BD1ED017A93ED007AF0EEE77AD7
:10008000F4EEC77AF1EE10FA7EF563AED1ED027AA6
:10009000F0EEE77AB4EEE77AF1EE10FA7EF759AEB9
:1000A000444B1A8800238AF86431002A40F0EA831E
:1000B000414A424B1178186881F00101F3F730F89A
:1000C000FEF747BE3E4B3F4A2344D3ED006A92ED14
:1000D000007A3D4B26EE877AF7EE006AB4EEE67AB8
:1000E000D3ED007AF1EE10FA88BFB0EE667A27EE13
:1000F000277A67EE0C7AFEF787BE019B5F023FF519
:1001000050AC52E4002FD6BF784207EE107A07EECB
:10011000100A2E4FB8EEC77A3F7827EE097A002FE3
:100120007FF4BDA82A4FD7ED006AF4EECB6AF1EE5A
:1001300010FA40F1BE87B7EE005A35EE665A9FEDD1
:10014000256A254F3BEEC77A25EE065A97ED006AE1
:10015000E7EE056A26EE867AB5EEC07AF1EE10FA81
:1001600040F2FE86CAEE076AB7EE006A35EEC67A3E
:10017000F0EE465AE7EE265AF0EE656AFFF7BFB892
:1001800001230399CAF86811022A8AF864317EF4BF
:1001900069AE084A1288002A43F0E181064A074BFB
:1001A00011781868F2F7BCFFFEF75CBE908C002057
:1001B000948C0020546B0020566B0020586B00205C
:1001C0000C260020608C00205C8C0020708C0020AD
:1001D000788C0020610BB63B6C8C0020D44BDDED9D
:1001E0000C7A93ED007A002840F09887E7EE267AA3
:1001F000D048B1EE436AB0EE647AA6EE277AF0EE0C
:10020000477ABDEEE47A002C42F0F282FDEEE77A06
:1002100017EE104A17EE906AFDEEC47AB44217EE5C
:10022000901A17EE105AA8BF3546B142C8BF0D4606
:1002300007EE905AF8EEE77A012AC0ED007A00F056
:100240004A8193ED047ADDED0D7AE7EE267AB0EE81
:10025000647AA6EE277AFDEEC77A17EE906A17EE5B
:10026000905AA642A8BF25468E42B8BF0D4607EE5B
:10027000905AF8EEE77A022AC0ED017A00F02B815D
:1002800093ED087ADDED0E7AE7EE267AB0EE647A29
:10029000A6EE277AFDEEC77A17EE906A17EE905A0F
:1002A000A642A8BF25468E42B8BF0D4607EE905A1B
:1002B000F8EEE77A032AC0ED027A00F00C8193EDA4
:1002C0000C7ADDED0F7AE7EE267AB0EE647AA6EED0
:1002D000277AFDEEC77A17EE906A17EE905AA6427B
:1002E000A8BF25468E42B8BF0D4607EE905AF8EEDD
:1002F000E77A042AC0ED037A00F0ED8093ED107ADE
:10030000DDED107AE7EE267AB0EE647AA6EE277A73
:10031000FDEEC77A17EE906A17EE905AA642A8BF74
:1003200025468E42B8BF0D4607EE905AF8EEE77AA2
:10033000052AC0ED047A00F0CE8093ED147ADDED4D
:10034000117AE7EE267AB0EE647AA6EE277AFDEE11
:10035000C77A17EE906A17EE905AA642A8BF2546B4
:100360008E42B8BF0D4607EE905AF8EEE77A062A9D
:10037000C0ED057A00F0AF8093ED187ADDED127ACA
:10038000E7EE267AB0EE647AA6EE277AFDEEC77A1B
:1003900017EE906A17EE905AA642A8BF25468E42E5
:1003A000B8BF0D4607EE905AF8EEE77A072AC0ED7F
:1003B000067A00F0908093ED1C7ADDED137AE7EE7B
:1003C000267AB0EE647AA6EE277AFDEEC77A17EEAB
:1003D000906A17EE905AA642A8BF25468E42B8BF33
:1003E0000D4607EE905AF8EEE77A082AC0ED077A34
:1003F00071D093ED207ADDED147AE7EE267AB0EE37
:10040000647AA6EE277AFDEEC77A17EE906A17EEA9
:10041000905AA642A8BF25468E42B8BF0D4607EEA9
:10042000905AF8EEE77A092AC0ED087A53D093ED96
:10043000247ADDED157AE7EE267AB0EE647AA6EE40
:10044000277AFDEEC77A17EE906A17EE905AA64209
:10045000A8BF25468E42B8BF0D4607EE905AF8EE6B
:10046000E77A0A2AC0ED097A35D093ED287ADDEDD6
:10047000167AE7EE267AB0EE647AA6EE277AFDEEDB
:10048000C77A17EE906A17EE905AA642A8BF254683
:100490008E42B8BF0D4607EE905AF8EEE77A0B2A67
:1004A000C0ED0A7A17D093ED2C7ADDED177AE6EEDF
:1004B000877AE6EE274AFDEEE47A17EE903A9C4200
:1004C000A8BF1C469942D8BF214607EE901AF8EE05
:1004D000E77AC0ED0B7ABCF1000F3FF404AC164B89
:1004E0001B68002B7FF40CAC144B1B7893B1144B9E
:1004F000187860B10F4D134E0024E0B23368B5ECAC
:10050000010A98470E4B187801348442F5DB0E4BF4
:100510001B6898479BF80030072B00F0AB85012340
:100520008AF8003119B0BDEC0C8BBDE8F08F00BF2C
:1005300010370020E8280020288C0020105E0020C2
:10054000756800209C590020A4590020D24BDDED95
:100550000C7A93ED007A002C41F05484E7EE267A71
:10056000CE48BDEEE47A17EE101AB0EE447AA3EE50
:10057000277A0D46F0EE477AFDEEE77ABDEEC47AB3
:1005800017EE906A17EE104AB142A8BF3546B44242
:10059000C8BF254607EE905AF8EEE77A012AC0ED6B
:1005A000007A98D093ED047ADDED0D7AE7EE267AA5
:1005B000B0EE447AA3EE277AFDEEC77A17EE906A82
:1005C00017EE905A8E42A8BF0D46A642B8BF2546E8
:1005D00007EE905AF8EEE77A022AC0ED017A3FF46E
:1005E0007AAF93ED087ADDED0E7AE7EE267AB0EE7B
:1005F000447AA3EE277AFDEEC77A17EE906A17EEDB
:10060000905A8E42A8BF0D46A642B8BF254607EEB7
:10061000905AF8EEE77A032AC0ED027A3FF45BAF16
:1006200093ED0C7ADDED0F7AE7EE267AB0EE447AA0
:10063000A3EE277AFDEEC77A17EE906A17EE905A6E
:100640008E42A8BF0D46A642B8BF254607EE905A77
:10065000F8EEE77A042AC0ED037A3FF43CAF93ED5D
:10066000107ADDED107AE7EE267AB0EE447AA3EE4A
:10067000277AFDEEC77A17EE906A17EE905A8E42EF
:10068000A8BF0D46A642B8BF254607EE905AF8EE21
:10069000E77A052AC0ED047A3FF41DAF93ED147A92
:1006A000DDED117AE7EE267AB0EE447AA3EE277AF2
:1006B000FDEEC77A17EE906A17EE905A8E42A8BFE9
:1006C0000D46A642B8BF254607EE905AF8EEE77AE7
:1006D000062AC0ED057A3FF4FEAE93ED187ADDED03
:1006E000127AE7EE267AB0EE447AA3EE277AFDEE90
:1006F000C77A17EE906A17EE905A8E42A8BF0D4641
:10070000A642B8BF254607EE905AF8EEE77A072AC8
:10071000C0ED067A3FF4DFAE93ED1C7ADDED137A7F
:10072000E7EE267AB0EE447AA3EE277AFDEEC77A9A
:1007300017EE906A17EE905A8E42A8BF0D46A64259
:10074000B8BF254607EE905AF8EEE77A082AC0EDC2
:10075000077A3FF4C0AE93ED207ADDED147AE7EE30
:10076000267AB0EE447AA3EE277AFDEEC77A17EE2A
:10077000906A17EE905A8E42A8BF0D46A642B8BFA7
:10078000254607EE905AF8EEE77A092AC0ED087A76
:100790003FF4A1AE93ED247ADDED157AE7EE267AEB
:1007A000B0EE447AA3EE277AFDEEC77A17EE906A90
:1007B00017EE905A8E42A8BF0D46A642B8BF2546F6
:1007C00007EE905AF8EEE77A0A2AC0ED097A3FF46C
:1007D00082AE93ED287ADDED167AE7EE267AB0EE5A
:1007E000447AA3EE277AFDEEC77A17EE906A17EEE9
:1007F000905A8E42A8BF0D46A642B8BF254607EEC6
:10080000905AF8EEE77A0B2AC0ED0A7A3FF463AE0D
:1008100093ED2C7ADDED177AE6EE877AA3EE274A80
:10082000FDEEC47A17EE903A9942A8BF19469C4251
:10083000D8BF0C4607EE904AF8EEE77AC0ED0B7A87
:1008400049E607EE901AF8EEE77A1548154C90ED58
:10085000004AD4ED004A1448CAED604A06EE903AC8
:1008600077EE677ABCEEC77AF8EEE66A17EE103AD2
:1008700077EEE67A8AED614AAAF87C31D0ED006A1B
:10088000FEF79ABD09494A69002A3EF462AA0A683D
:1008900013604B74FEF75DBA10370020E828002083
:1008A000D4370020D0370020EC3700205C6B0020CC
:1008B00007EE103A9BF800308E4FCAF81061B8EE80
:1008C000C77AF7EE006A132B86EE879AB7F9040011
:1008D000BAF8145194ED080A01F06481864B874AF6
:1008E00093ED001A93ED093A93ED162A93ED1F6AE2
:1008F000D3ED0B1A93ED144AD3ED015AD3ED0A3A16
:1009000093ED0C7A93ED155AD3ED172AD3ED206AA7
:10091000D3ED044AD3ED030A69EE277A69EE288AFB
:1009200029EE088AA7EE813A02EB85060021A2EEA5
:10093000286ACAF80411CAF80811A8EE214AE7EE9D
:10094000A53AA8EE075A93ED1A7AD3ED0F5A93ED14
:10095000021AD3ED0E1A86ED003AE2EEA86A64EEB2
:10096000C34A27EE467A93ED0D2AD3ED192A86ED78
:10097000204AE3EE603A65EEC45A93ED183AC3EDAF
:10098000093AE7EE814AF0EE477AA4EE615AE8EEC2
:10099000025AE2EEC66AE3EE287AC3ED0A4A83ED14
:1009A000145AC3ED155A86ED406AC3ED1F6AC3EDB4
:1009B000207ACAF80C116B1C03F01F03AAF814313B
:1009C000B880FEF7D1B84E4B1A79002A3EF472ADCA
:1009D0004C4A1278002A3EF46DAD1B789FED4A2AEE
:1009E00007EE103A494B07EE902A1B88F8EEE77A9B
:1009F00005EE103AB8EE477AB8EE455A27EE277A58
:100A0000F7EE003AC7EE057AF4EEC27AF1EE10FA8C
:100A100088BFF0EE427AF4EEE37AF1EE10FAB8BF56
:100A2000F0EE637AFEF748BDB37B002B42F06B8497
:100A3000029B1B7813F0010342F06584344A12686C
:100A4000002A02F02186136001230593009B1B6896
:100A5000980633D42F4A1278052A2FD0D9027FF571
:100A600043ADF57B112D3FF63FAD2B4BDDF81480E8
:100A70001C4633F9153000EE103A4046B8EEC00A75
:100A80006F1C05F10E060AF077FD4346FFB25D1BB1
:100A9000F6B2A04600E027467C1C7819122FE4B27B
:100AA000C0B23FF421AD38F9173000EE103AB8EE7D
:100AB000C00A0AF061FDB442EDD115E5059A13466E
:100AC0000233541CDBB21046E4B20593B5F9003092
:100AD00000EE103AB8EEC00A0AF04EFDB5F9023049
:100AE00000EE103A2046B8EEC00A0AF045FD009B21
:100AF0001B68B3E78868002098540020FC51002050
:100B0000DC93002073690020713DAA3F1C6900201E
:100B1000905700202C8C0020AC88002000000000A2
:100B200093ED027A93ED012AD3ED037A5FED053A56
:100B300026EE877AA6EE027AA5EEA77A27EE057A48
:100B4000B4EEE37AF1EE10FAB4BFF0EE637AF0EEB1
:100B5000477A8DED0C7A88BFB0EE637A012A3EF4B5
:100B6000AEAED3ED063AD3ED051A93ED072A66EE45
:100B7000A33AE6EE213AE5EE823A63EE853AB4EE28
:100B8000E37AF1EE10FAF4EEE37A8CBFB0EE632A6A
:100B9000B0EE472AF1EE10FA58BFB0EE427AB8BF75
:100BA000F0EE637A022ACDED0D3A3EF488AED3ED35
:100BB0000A3AD3ED091A93ED0B2A66EEA33AE6EE54
:100BC000213AE5EE823A63EE853AB4EEE37AF1EE4D
:100BD00010FAF4EEE37A8CBFB0EE632AB0EE472A47
:100BE000F1EE10FA58BFB0EE427AB8BFF0EE637A79
:100BF000032ACDED0E3A3EF462AED3ED0E3AD3EDBC
:100C00000D1A93ED0F2A66EEA33AE6EE213AE5EED1
:100C1000823A63EE853AB4EEE37AF1EE10FAF4EE3E
:100C2000E37A8CBFB0EE632AB0EE472AF1EE10FAF9
:100C300058BFB0EE427AB8BFF0EE637A042ACDED29
:100C40000F3A3EF43CAED3ED123AD3ED111A93EDC8
:100C5000132A66EEA33AE6EE213AE5EE823A63EE17
:100C6000853AB4EEE37AF1EE10FAF4EEE37A8CBF53
:100C7000B0EE632AB0EE472AF1EE10FA58BFB0EE9C
:100C8000427AB8BFF0EE637A052ACDED103A3EF411
:100C900016AED3ED163AD3ED151A93ED172A66EE7C
:100CA000A33AE6EE213AE5EE823A63EE853AB4EEF7
:100CB000E37AF1EE10FAF4EEE37A8CBFB0EE632A39
:100CC000B0EE472AF1EE10FA58BFB0EE427AB8BF44
:100CD000F0EE637A062ACDED113A3EF4F0ADD3ED95
:100CE0001A3AD3ED191A93ED1B2A66EEA33AE6EEF3
:100CF000213AE5EE823A63EE853AB4EEE37AF1EE1C
:100D000010FAF4EEE37A8CBFB0EE632AB0EE472A15
:100D1000F1EE10FA58BFB0EE427AB8BFF0EE637A47
:100D2000072ACDED123A3EF4CAADD3ED1E3AD3ED0B
:100D30001D1A93ED1F2A66EEA33AE6EE213AE5EE80
:100D4000823A63EE853AB4EEE37AF1EE10FAF4EE0D
:100D5000E37A8CBFB0EE632AB0EE472AF1EE10FAC8
:100D600058BFB0EE427AB8BFF0EE637A082ACDEDF4
:100D7000133A3EF4A4ADD3ED223AD3ED211A93ED0C
:100D8000232A66EEA33AE6EE213AE5EE823A63EED6
:100D9000853AB4EEE37AF1EE10FAF4EEE37A8CBF22
:100DA000B0EE632AB0EE472AF1EE10FA58BFB0EE6B
:100DB000427AB8BFF0EE637A092ACDED143A3EF4D8
:100DC0007EADD3ED263AD3ED251A93ED272A66EEB4
:100DD000A33AE6EE213AE5EE823A63EE853AB4EEC6
:100DE000E37AF1EE10FAF4EEE37A8CBFB0EE632A08
:100DF000B0EE472AF1EE10FA58BFB0EE427AB8BF13
:100E0000F0EE637A0A2ACDED153A3EF458AD93ED33
:100E10002A2AD3ED291AD3ED2B3A26EE822AA6EE02
:100E2000212AA5EEA32A22EE052AB4EEC27AF1EE1B
:100E300010FAF4EEC27A8CBFF0EE423AF0EE473A86
:100E4000F1EE10FA8DED162A58BFB0EE637AA8BF06
:100E5000B0EE672A0B2A02F03A83D3ED2E7AD3ED57
:100E60002D1AD3ED2F3A66EEA77AE6EE217AE3EE5D
:100E7000A57A67EE857AF4EEC77AF1EE10FAF4EE11
:100E8000C27A8CBFF0EE476AF0EE676AF1EE10FAB4
:100E9000CDED177A98BFB0EE667AB8BFF0EE427A21
:100EA000FEF70DBD904A04920025904E904FDDF85C
:100EB0001080CDF80490A946B6EC018AD4ED087AEA
:100EC000B8EEC88A28EE278AB9F1000F02F0EB834A
:100ED0007BBB9BF80030082B3BD005F5D260B0EE11
:100EE000480A2044D4F88C36984705F5E360D4F8D6
:100EF0001437204498479BF80030032BB0EE408A0B
:100F000022D0D4F8AC30D6F84406B0EE480A984760
:100F100008EB890309F10109B9F1030F05F12C056B
:100F200083ED010A3DF440AE009B1B6803F00053C3
:100F3000C2E705F5F460B0EE480A2044D4F89C37C7
:100F40009847B0EE408AC4E721F03AFD27F819002F
:100F5000D7E7B0EE480A21F033FD27F81900BCE7C7
:100F6000DFED646AFEF7D9B9DFF8A881DAED017A1E
:100F70009AED006AB8F80000D8F8143077EEA77A36
:100F8000F0EE006AB0EE677AA6EE267A01380AEB38
:100F9000C002D6EE267A083A1033F6EE003A27EE73
:100FA000237A67EEA37A8AED207ACAED217ADFF8F8
:100FB00068A157460AF1800192ED027A92ED036A28
:100FC000D7ED036AD7ED027A53ED014A13ED025AC9
:100FD00037EE674A76EEC65A77EE277AE4EE845A01
:100FE0000138A2F10802E5EE047A07F1080703F1DF
:100FF000080336EE267A01F10801E4EE877AE5EE81
:10100000475A67EEA37A25EEA37AC1ED007A81ED07
:10101000017AD1D1142E07D1F1F7A2FB019B344FF5
:10102000C01A7880DAF818512F4B0493324A009B8B
:10103000013582FB05125119EA17C2EBA1021B68A8
:10104000C2EBC202AD1ACAF8185103F000532BE7E5
:10105000F1F786FB9BF80030079A254F801A012B89
:1010600078802CD0072B7DF429AFF1F779FB049021
:10107000FDF726BFF1F774FB049A1D4B801AD88048
:10108000FFF74DBA1D491E481E4B91ED004AD0EDA9
:10109000004A1D491B78CAED604A8AED614AD1EDCC
:1010A000006A13B101238AF88C31DAED627AFEF717
:1010B00083B9164F97ED007AFFF74EB80C4FF1F752
:1010C0004FFB134ADAF8783112680490C31A9A1A5F
:1010D000CAF87801BB80FA80FDF7F2BEF1F740FB59
:1010E0000790FDF77EBD00BF484C00205C44002007
:1010F000886800200000000093244992DC29002029
:10110000D8370020A8590020E83700206C8C002038
:10111000742B0020E4510020B4240020E7EE267A4E
:10112000DF48B1EE436AB0EE647AA6EE277AF0EEBD
:10113000477ABDEEE47A002C41F09686FDEEE77A20
:1011400017EE104A17EE906AFDEEC47AB44217EE1D
:10115000901A17EE105AA8BF3546B142C8BF0D46C7
:1011600007EE905AF8EEE77A012AC0ED007A3FF4D4
:10117000B2A993ED047ADDED0D7AE7EE267AB0EEB2
:10118000647AA6EE277AFDEEC77A17EE906A17EE1C
:10119000905AA642A8BF25468E42B8BF0D4607EE1C
:1011A000905AF8EEE77A022AC0ED017A3FF493A94B
:1011B00093ED087ADDED0E7AE7EE267AB0EE647AEA
:1011C000A6EE277AFDEEC77A17EE906A17EE905AD0
:1011D000A642A8BF25468E42B8BF0D4607EE905ADC
:1011E000F8EEE77A032AC0ED027A3FF474A993ED92
:1011F0000C7ADDED0F7AE7EE267AB0EE647AA7EE90
:10120000C37AFDEEC77A17EE906A17EE905AA6429F
:10121000A8BF25468E42B8BF0D4607EE905AF8EE9D
:10122000E77A042AC0ED037A3FF455A993ED107ACA
:10123000DDED107AE7EE267AB0EE647AA7EEC37A97
:10124000FDEEC77A17EE906A17EE905AA642A8BF35
:1012500025468E42B8BF0D4607EE905AF8EEE77A63
:10126000052AC0ED047A3FF436A993ED147ADDED3A
:10127000117AE7EE267AB0EE647AA7EEC37AFDEE35
:10128000C77A17EE906A17EE905AA642A8BF254675
:101290008E42B8BF0D4607EE905AF8EEE77A062A5E
:1012A000C0ED057A3FF417A993ED187ADDED127AB7
:1012B000E7EE267AB0EE647AA7EEC37AFDEEC77A3F
:1012C00017EE906A17EE905AA642A8BF25468E42A6
:1012D000B8BF0D4607EE905AF8EEE77A072AC0ED40
:1012E000067A3FF4F8A893ED1C7ADDED137AE6EE6A
:1012F000877A2546B0EE647AA6EE277AFDEEC77AA5
:1013000017EE906AB442A8BF3546B142C8BF0D4639
:1013100007EE905AF8EEE77A082AC0ED077A3FF414
:10132000DAA893ED207ADDED147AE6EE877A254689
:10133000B0EE647AA6EE277AFDEEC77A17EE906AD1
:10134000B442A8BF3546B142C8BF0D4607EE905A19
:10135000F8EEE77A092AC0ED087A3FF4BCA893EDCD
:10136000247ADDED157AE6EE877A2546B0EE647ACA
:10137000A6EE277AFDEEC77A17EE906AB442A8BFB0
:101380003546B142C8BF0D4607EE905AF8EEE77AEF
:101390000A2AC0ED097A3FF49EA893ED287ADDED84
:1013A000167AE7EE267A2546B0EE647AA7EEC37A7F
:1013B000FDEEC77A17EE906AB442A8BF3546B14237
:1013C000C8BF0D46FFF767B8FDEEC47A0CA817EE4C
:1013D000906AFDEEE47A00EB820317EE907AFDEE60
:1013E000E57ADFF8C090DFF8B8E0089217EE905A7F
:1013F000B1EE436A84F001084FFA84FC1946CDF837
:1014000024A04B4693ED007AF0EC017AE7EE267AC1
:1014100004F0010309F11009B0EE647AA6EE277A10
:10142000B4EEC74AF1EE10FAD8BF0023002BF0EE5D
:10143000477A18BFB0EE657ABDEEC77AFDEEE77A5F
:1014400017EE102A17EE90AABA4217EE103AA8BF6C
:101450003B469542CCBF002204F00102002A08BF9F
:101460002B46574507EE103A3A46A8BF5246564516
:10147000CCBF002308F00103002B08BF324607EE63
:10148000902AB8EEC77AF8EEE77ABCF1000F18BFE1
:10149000F0EE477A8842EEEC017AB2D1FEF7AEBDAB
:1014A000E828002010370020B84BB5F908101A685A
:1014B00002B111609B69B5F90A2003B11A60009B63
:1014C0001B689A0601F1A58602220592FFF7C6BAAB
:1014D0009AF8B831012B01F02287AD4B96F916002E
:1014E0005A8896F90AE01B88AA4910FB03F31EFBF1
:1014F00002F281FB020C81FB0301D217DB17C2EB66
:101500002C12C3EB21133A441C442A806C80FEF752
:101510003FBCDFF8A082A048D8F80820B8F80C102B
:101520001FF098FE9BF80060142E02F05880DAF845
:1015300018510135CAF8185118E5DFF87882B8F863
:101540000060D8F804E04FEA560C4FEA8C020AEB30
:101550008607F6080AEB020300F09F80103201367E
:101560008E4803EB06163A4410330EF1100507F1CE
:10157000100151ED032A51ED043A10ED043A10ED3B
:10158000032A51ED026A11ED016A10ED020A10ED15
:10159000018A12ED044A12ED035A53ED044A53ED49
:1015A000035A13ED027A53ED017A52ED020A12ED5D
:1015B000011A73EE238A72EE221A40ED048A40ED7E
:1015C000031A70EE268A78EE061A40ED028A40ED84
:1015D000011A74EE848A75EE851A43ED048A43ED90
:1015E000031A77EE208A77EE811A43ED028A43EDE3
:1015F000011A73EE633A75EE655A15ED035A32EE31
:10160000623A74EE644A65EE631A15ED044A23EEFD
:10161000052A64EE652AE3EE041A1033B34224EE81
:10162000843AA3EE842A00F1100005F11005A5EE1E
:10163000853A01F1100102F11002E4EE852A41ED34
:10164000071A01ED082A02ED073A42ED082A55ED86
:10165000055A15ED065A70EE666A38EE466A30EEA7
:10166000C77A71EE677A26EE253A65EEE63A25EE00
:10167000674A67EE054AE6EE053AA6EE853AA7EE1A
:10168000254AE7EEA54A01ED063A41ED053A02ED9D
:10169000064A42ED054A7FF46CAF1FFA8CF572469C
:1016A00029463D4810F0ECFE2946D8F8042038467B
:1016B00010F0E6FE9BF80030142B7FF4B3ACABE4E3
:1016C000374BDAF81CC10493BAF81481C8F120032F
:1016D000D8B2344B08EB4C1703EB8707830801F0B3
:1016E000798701331B0130492C4A029307EB030E23
:1016F00007F1100313ED024A13ED035A13ED016ACB
:1017000013ED047A51ED024A51ED035A51ED016A8D
:1017100051ED047A64EE244A65EE255A66EE266A97
:1017200067EE277A1033734542ED024A42ED035AC1
:1017300042ED016A42ED047A01F1100102F110025A
:10174000D8D1029B1949A3F11002174401EB020EF4
:10175000524410F0030309D0B7EC017AFEEC017A91
:1017600067EE277A013BE2EC017AF5D1B8F1000F80
:1017700041F05585142E7FF459ACF0F7F1FF019B31
:101780000B4FDAF81851C01A78804FE490570020B8
:10179000603E00201F85EB51B4240020C4240020AB
:1017A000484C0020FC5100208C5300207C5300202A
:1017B00088680020E4510020D94B1A78DAF81CE13F
:1017C000D8489FEDD97A4FEACE07C31983ED007A46
:1017D000002A7AD0D549B0EE476AF0EE476A002376
:1017E000F1EC017A013367EEA77A05EE903AB4EE98
:1017F000E77AF1EE10FAF8EEE55AB8BFB0EE677A84
:10180000934276EEA76AA7EEA56AE9D1F5EEC06A23
:10181000C319F1EE10FA83ED007A56DDC6EE265AB2
:10182000C34BC44A1288F7EE007A75EEE75AD3ED3F
:10183000007A65EEA77AFDEEE77A17EE903A812BF3
:1018400041F309839342A8BF134607EE903AF8EE9E
:10185000E77AB94B2C2101FB0E3393ED097AD3EDD6
:10186000003A93ED0A6A93ED014AD3ED046AD3ED91
:10187000034A93ED025AA3EEA77AA4EE276A66EE16
:10188000C76AA7EE646ABDEEC77AE5EE276A17EE6F
:10189000101A812983ED096AC3ED0A6A41F3D882DF
:1018A0008A42A8BF0A4607EE902AF8EEE77AFCEED5
:1018B000E77ACDED027ABDF80830C2199380BEF107
:1018C000000F02D1132E01F05986152E7FF4A2AB22
:1018D00038449A4F838827F81E30994BDAF818510C
:1018E0000493FFF7A3BBDAF81C81954A8D4B049251
:1018F00003EBC803126802929DED027A9B88DFED2C
:10190000917A914AF8EE478A09EE103A643BC82B67
:10191000A8BFC82368EEA78AF8EE497A782BB8BF2B
:10192000782368EEA78A07EE903A2C27B0EE680A73
:1019300007FB0827B8EEE78A21F08EF8B8EEC99ABF
:10194000F0EE409AB0EE680A20F0E8FF38EE097A2F
:1019500079EE487A28EE098A67EE877AB7EE006A50
:1019600088EE277A142EF8EE007A77EE076A60EE9A
:10197000277A89EEA67A77EE065A36EE477AC6EED1
:10198000256A67EEA67A27EE267AC7ED006A87ED0C
:10199000047AC7ED026AC7ED017AC7ED037A01F058
:1019A00036866A4B9BF8006008F1010883FB083C0F
:1019B000ACEBE87C0CEB4C0C0135A8EB0C0CCAF83A
:1019C0001851CAF81CC17FE6DFF8548198F800204E
:1019D000970801F03B86DFF88CC1781C40010CEBC6
:1019E000000E0CF12003ACF1700113ED076A53ED0A
:1019F000056A13ED037A53ED017A53ED025A13EDA4
:101A0000084A53ED064A13ED045A26EE066A66EEBE
:101A1000A66A27EE077A67EEA77AA4EE046A203357
:101A20007345E4EEA46A01F11001A5EE057AE5EE36
:101A3000A57AF1EEC65AB1EEE66AF1EEC76AB1EEEA
:101A4000E77A41ED085A01ED076A41ED066A01EDBA
:101A5000057ACAD1203884440AEB071712F0030331
:101A600018BF0CF1080C0FD05CED017A1CED027A66
:101A700067EEA77A013BE7EE077A0CF1080CB1EEAE
:101A8000E77AA7EC017AEFD1142E01F0B285013587
:101A9000CAF8185192E62E4A32F91340FEF771B98E
:101AA0002B4A32F91370FEF761B9294B294D1A6898
:101AB00059682A609A68DB68EB606960264EAA6004
:101AC000019BFEF747B9F0F74BFE9BF800600190D1
:101AD000142E05BF194FDAF81851DAF818513D8065
:101AE000FDF74BB81D4F002437F9023F00EE103AC6
:101AF000E0B2B8EEC00A013409F03EFD082CF3D183
:101B00000594FEF7A3BF164BB5F906101A6802B18B
:101B100011609B69B5F90820002B7FF4CFACCEE4AF
:101B2000DE510020FC53002000000000B4240020FF
:101B3000E0510020DC51002014540020886800206F
:101B4000484C002027D4D236C44B0020565555555A
:101B5000AC880020D82800200C8D0020D62800203A
:101B600090570020342500209A4F002437F9023B7B
:101B700000EE103AE0B2B8EEC00A013409F0FCFC05
:101B8000042CF3D1BCE7944F002437F9023F00EE58
:101B9000103AE0B2B8EEC00A013409F0EDFC062CB0
:101BA000F3D1ADE78D4EDFF8588296ED004A96ED01
:101BB000097AD6ED014A96ED0A6AD6ED046A96EDE9
:101BC000035AD6ED025A69EE277A08EB8503A7EE91
:101BD000847AA7EEA46A66EEC76AA7EE456AE7EEC6
:101BE000A56A20EE070A86ED096AC6ED0A6A83ED4A
:101BF000007A29EE088A20F0E3FE69EE288AD6ED05
